:020000040800F2
:1000000000060020A102000855100008D50F0008C6
:100010002D100008D50F000801100008A3020008E9
:10002000A3020008A3020008A3020008392A00085E
:10003000A3020008A3020008A3020008A30200080C
:10004000A3020008A3020008A3020008A3020008FC
:10005000A3020008A3020008C13E0008ED3E00080C
:10006000193F0008453F0008713F0008A30200083F
:10007000A3020008A3020008A3020008A3020008CC
:10008000A3020008A3020008A3020008A3020008BC
:10009000A3020008A3020008A30200089D3F000875
:1000A000A3020008A3020008A3020008A30200089C
:1000B000A3020008A3020008A3020008A30200088C
:1000C000A3020008A3020008A3020008A30200087C
:1000D000A3020008A3020008A3020008754000085C
:1000E00001400008A3020008A3020008A3020008C0
:1000F000A3020008A3020008A3020008A30200084C
:10010000A3020008A3020008B1400008A3020008EF
:10011000A302000889400008A3020008A302000807
:10012000A3020008A3020008A3020008A30200081B
:10013000A3020008A3020008A3020008A30200080B
:10014000A3020008A3020008A3020008A3020008FB
:10015000A3020008A3020008A3020008A3020008EB
:10016000A3020008A3020008A3020008A3020008DB
:10017000A3020008A5350008A3020008A302000896
:10018000A3020008A30200089D400008A302000883
:10019000A3020008A3020008A3020008A3020008AB
:1001A000A3020008A3020008A3020008A30200089B
:1001B000A3020008A3020008A3020008A30200088B
:1001C000A3020008A3020008A3020008A30200087B
:1001D000A302000891350008A3020008A30200084A
:1001E000A3020008A3020008A3020008A30200085B
:1001F000A3020008A3020008A3020008A30200084B
:10020000A3020008A3020008A3020008A30200083A
:10021000A3020008A3020008A3020008A30200082A
:10022000A3020008A3020008A3020008A30200081A
:10023000A3020008A3020008A3020008A30200080A
:10024000A3020008A3020008A3020008A3020008FA
:10025000A3020008A3020008A3020008A3020008EA
:10026000A3020008A3020008A3020008A3020008DA
:10027000A3020008A3020008A3020008A3020008CA
:10028000A3020008A3020008A3020008A3020008BA
:10029000A3020008A3020008A3020008A3020008AA
:1002A00002E000F000F8FEE772B63A4880F30888F2
:1002B000394880F3098839484EF60851CEF20001DA
:1002C000086040F20000CCF200004EF63471CEF22D
:1002D00000010860BFF34F8FBFF36F8F40F2000043
:1002E000C0F2F0004EF68851CEF200010860BFF374
:1002F0004F8FBFF36F8F4FF00000E1EE100A4EF604
:100300003C71CEF200010860062080F31488BFF330
:100310006F8F02F04FFC02F0F1FB03F08BFB4FF00C
:1003200055301F491B4A91423CBF41F8040BFAE784
:100330001C49194A91423CBF41F8040BFAE71A499B
:100340001A4A1B4B9A423EBF51F8040B42F8040B69
:10035000F8E700201749184A91423CBF41F8040BC6
:10036000FAE702F009FC03F0E9FB144C144DAC422F
:1003700003DA54F8041B8847F9E700F041F8114C00
:10038000114DAC4203DA54F8041B8847F9E702F038
:10039000F1BB000000060020002200200000000841
:1003A0000000002000060020E04400080022002099
:1003B0005C22002060220020D44F0020A002000810
:1003C000A0020008A0020008A00200082DE9F04FDA
:1003D0002DED108AC1F80CD0D0F80CD0BDEC108AED
:1003E000BDE8F08F002383F311882846A047002042
:1003F00001F006FFFEE701F081FE00DFFEE70000EE
:1004000038B500F0D7FC30B1164B00220E211A721D
:100410005A729972DA7202F0CFFA054602F002FBC4
:100420000446D0B9104B9D4219D001339D4241F290
:10043000883512BF044600250124002002F0C6FAC8
:100440000CB100F059F800F065FD00F0F9FB28460A
:1004500000F004F900F050F8F9E70025EDE7054653
:10046000EBE700BF00220020010007B008B500F054
:10047000B3FBA0F120035842584108BD07B541F233
:100480001203022101A8ADF8043000F0C3FB03B051
:100490005DF804FB202310B583F311881248C3686C
:1004A0000BB101F033FF0023104A4FF47A710E486C
:1004B00001F0F0FE002383F311880D4C236813B183
:1004C0002368013B2360636813B16368013B636089
:1004D000084B1B7833B9636823B9022000F08CFC09
:1004E0003223636010BD00BF602200209504000825
:1004F0007C23002074220020F8B5514B514A1C4641
:100500001968013100F09B8004339342F8D162688E
:100510004D4B9A4240F293804C4B9B6803F1006331
:1005200003F500339A4280F08A80002000F0A2FB9D
:100530000220474B187000F04FFC464B0021D3F8C7
:10054000E820C3F8E810D3F81021C3F81011D3F84D
:100550001021D3F8EC20C3F8EC10D3F81421C3F821
:100560001411D3F81421D3F8F020C3F8F010D3F805
:100570001821C3F81811D3F81821D3F8802042F0BD
:100580000062C3F88020D3F8802022F00062C3F814
:100590008020D3F88020D3F8802042F00072C3F886
:1005A0008020D3F8802022F00072C3F88020D3F896
:1005B000803072B64FF0E023C3F8084DD4E9000450
:1005C000BFF34F8FBFF36F8F234AC2F88410BFF37E
:1005D0004F8F536923F480335361BFF34F8FD2F8A9
:1005E000803043F6E076C3F3C905C3F34E335B01B5
:1005F00003EA060C29464CEA81770139C2F8747285
:10060000F9D2203B13F1200FF2D1BFF34F8FBFF38C
:100610006F8FBFF34F8FBFF36F8F536923F4003396
:1006200053610023C2F85032BFF34F8FBFF36F8F77
:10063000202383F31188854680F308882047F8BD7E
:100640000000020820000208FFFF0108002200202D
:10065000742200200044025800ED00E02DE9F04F24
:1006600093B0A94B2022FF2100900AA89D6800F0BA
:10067000FBFBA64A1378A3B90121A5481170C360FA
:10068000202383F31188C3680BB101F03FFE0023E0
:10069000A04A4FF47A719E4801F0FCFD002383F3D9
:1006A0001188009B9C4A03B1136000239B49009C66
:1006B00098469B461E469A460B705360012000F0F8
:1006C0008BFB24B1944B1B68002B00F0168200209A
:1006D00000F082FA0390039B002BF2DB012000F074
:1006E0006BFB039B213B162BE8D801A252F823F0A9
:1006F0004D0700087507000809080008BD06000836
:10070000BD060008BD0600089D0800086F0A000825
:1007100089090008EB090008130A0008390A0008D3
:10072000BD0600084B0A0008BD060008BD0A000807
:10073000ED070008BD060008010B00085907000876
:10074000ED070008BD060008EB0900080220FFF7CE
:100750008DFE002840F0FB81009B022105A8B8F126
:10076000000F08BF1C4641F21233ADF8143000F000
:1007700051FAA3E74FF47A7000F02EFA071EEBDB74
:100780000220FFF773FE0028E6D0013F052F00F29C
:10079000E081DFE807F0030A0D101336052304217A
:1007A00005A8059300F036FA17E004215648F9E74A
:1007B00004215B48F6E704215A48F3E74FF01C098F
:1007C000484609F1040900F057FA0421059005A8EC
:1007D00000F020FAB9F12C0FF2D101204FF0000AFD
:1007E00000FA07F747EA0B0B5FFA8BFB00F088FB78
:1007F00026B10BF00B030B2B08BF0024FFF73EFEC6
:100800005CE704214848CDE7002EA5D00BF00B0390
:100810000B2BA1D10220FFF729FE074600289BD011
:1008200001203E4E00F026FA4FF000080220307002
:1008300000F0D2FA5FFA88F9484600F02BFA044635
:1008400090B1484608F1010800F034FA0028F1D1CF
:10085000B846044641F21213022105A83E46ADF8FF
:10086000143000F0D7F929E7012325460220337020
:1008700000F0A2FA244B9B68AB4207D9284600F04F
:10088000FBF9013040F068810435F3E70025234B84
:10089000B8463E461D70204B5D60A7E7002E3FF432
:1008A0005BAF0BF00B030B2B7FF456AF02201B4BFF
:1008B000187000F091FA322000F08EF9B0F10009C2
:1008C000FFF64AAF19F003077FF446AF0E4A09EB73
:1008D0000503926893423FF63FAFB9F5807F3FF73B
:1008E0003BAF124BB945019322DD4FF47A7000F013
:1008F00073F90390039A002AFFF62EAF039A01378B
:10090000019B03F8012BEDE7002200207823002053
:1009100060220020950400087C230020742200201F
:1009200004220020082200200C220020782200202F
:10093000C820FFF79BFD074600283FF40DAF1F2D91
:1009400011D8C5F120020AAB25F0030084494A45BD
:10095000184428BF4A46019200F060FA019AFF212C
:100960007F4800F081FA4FEAA903C9F387027C4966
:100970002846019300F080FA064600283FF46AAF4B
:10098000019B05EB830531E70220FFF76FFD00288F
:100990003FF4E2AE00F0AAF900283FF4DDAE0027F4
:1009A000B946704B9B68BB4218D91F2F11D80A9BC0
:1009B00001330ED027F0030312AA134453F8203C4E
:1009C00005934846042205A9043700F045FB8146FB
:1009D000E7E7384600F050F90590F2E7CDF81490BB
:1009E000042105A800F016F900E70023642104A8FB
:1009F000049300F005F900287FF4AEAE0220FFF763
:100A000035FD00283FF4A8AE049800F065F9059084
:100A1000E6E70023642104A8049300F0F1F800281D
:100A20007FF49AAE0220FFF721FD00283FF494AE38
:100A3000049800F053F9EAE70220FFF717FD0028B9
:100A40003FF48AAE00F062F9E1E70220FFF70EFD05
:100A500000283FF481AE05A9142000F05DF9074697
:100A60000421049004A800F0D5F83946B9E73220F3
:100A700000F0B2F8071EFFF66FAEBB077FF46CAE56
:100A8000384A07EB0A03926893423FF665AE0220AC
:100A9000FFF7ECFC00283FF45FAE27F00307574454
:100AA000BA453FF4A3AE50460AF1040A00F0E4F858
:100AB0000421059005A800F0ADF8F1E74FF47A7035
:100AC000FFF7D4FC00283FF447AE00F00FF90028F0
:100AD00044D00A9B01330BD008220AA9002000F061
:100AE000CBF900283AD02022FF210AA800F0BCF957
:100AF000FFF7C4FC1C4801F089FB13B0BDE8F08F80
:100B0000002E3FF429AE0BF00B030B2B7FF424AE29
:100B10000023642105A8059300F072F80746002819
:100B20007FF41AAE0220FFF7A1FC814600283FF4B3
:100B300013AEFFF7A3FC41F2883001F067FB059884
:100B400000F028FA4E463C4600F0DAF9B6E50646D3
:100B50004CE64FF0000AFFE5B8467BE6374679E6FB
:100B60007822002000220020A08601002DE9F84F05
:100B70004FF47A7306460D46002402FB03F7DFF8B4
:100B80005080DFF8509098F900305FFA84FA5A1CD0
:100B900001D0A34210D159F824002A4631460368F7
:100BA000D3F820B03B46D847854205D1074B0120FA
:100BB00083F800A0BDE8F88F0134042CE3D14FF492
:100BC000FA7001F023FB0020F4E700BFC8230020E7
:100BD00010220020B4410008002307B5024601217D
:100BE0000DF107008DF80730FFF7C0FF20B19DF829
:100BF000070003B05DF804FB4FF0FF30F9E7000099
:100C00000A46042108B5FFF7B1FF80F00100C0B229
:100C1000404208BD074B0A4630B41978064B53F8DA
:100C20002140014623682046DD69044BAC4630BCB8
:100C3000604700BFC8230020B4410008A08601001F
:100C400070B50A4E00240A4D01F08EFD30802868F0
:100C50003388834208D901F083FD2B6804440133B3
:100C6000B4F5003F2B60F2D370BD00BFCA23002053
:100C70008423002001F056BE00F1006000F5003032
:100C80000068704700F10060920000F5003001F04C
:100C9000CDBD0000054B1A68054B1B889B1A83428B
:100CA00002D9104401F05CBD00207047842300206D
:100CB000CA23002038B5074D04462868204401F0B7
:100CC00055FD28B928682044BDE8384001F060BDD2
:100CD00038BD00BF842300200020704700F1FF5082
:100CE00000F58F10D0F8000870470000064991F811
:100CF000243033B100230822086A81F82430FFF73A
:100D0000C1BF0120704700BF88230020014B186835
:100D1000704700BF0010005C244BF0B51A68044611
:100D2000234BC2F30B06120C1F885868BE4293F97E
:100D3000085028D09F89BE4206D101200C2505FB12
:100D40000033586893F9085041F201039A421CD0CD
:100D500041F203039A421AD042F201039A4218D098
:100D600042F203039A4208BF5625621E0B46441EF8
:100D70000A4493420FD214F9016F581C6EB1034616
:100D800000F8016CF5E70020D8E75A25EDE7592572
:100D9000EBE75825E9E7184605E02C2482421C7051
:100DA00001D9981C5D70401AF0BD00BF0010005CB6
:100DB0001422002000207047022804D1054B4FF078
:100DC00000629A6170470128FCD1024B4FF08062AB
:100DD000F7E700BF000C0258022804D1054B4FF47E
:100DE00000629A6170470128FCD1024B4FF4806287
:100DF000F7E700BF000C0258022805D1064A5369E4
:100E000083F40063536170470128FCD1024A53699F
:100E100083F48063F6E700BF000C0258002310B58E
:100E2000934203D0CC5CC4540133F9E710BD0000F9
:100E3000013810B510F9013F3BB191F900409C42D7
:100E400003D11AB10131013AF4E71AB191F9002046
:100E5000981A10BD1046FCE703460246D01A12F954
:100E6000011B0029FAD1704702440346934202D085
:100E700003F8011BFAE770472DE9F8431F4D1446AC
:100E80000746884695F8242052BBDFF870909CB343
:100E900095F824302BB92022FF2148462F62FFF716
:100EA000E3FF95F824004146C0F1080205EB8000FD
:100EB000A24228BF2246D6B29200FFF7AFFF95F8B4
:100EC0002430A41B17441E449044E4B2F6B2082E0A
:100ED00085F82460DBD1FFF709FF0028D7D108E0AF
:100EE0002B6A03EB82038342CFD0FFF7FFFE00287B
:100EF000CBD10020BDE8F8830120FBE78823002048
:100F0000024B1A78024B1A70704700BFC8230020AA
:100F100010220020F8B5194C194800F079FC214640
:100F2000174800F0A1FC24681648D4F89020164E0B
:100F3000D2F80438154D43F00203114FC2F80438BB
:100F400001F064F92046124900F09CFDD4F890208D
:100F50000424D2F8043823F00203C2F804384FF412
:100F6000E133336055F8040BB84202D0314600F04B
:100F7000ADFB013C14F0FF04F4D1F8BDC4420008FD
:100F8000C832002040420F00B0230020B4410008C6
:100F9000CC42000838B50B4B04461A780A4B53F87C
:100FA00022500A4B9D420CD0094B002118221846B2
:100FB000FFF75AFF046001462846BDE8384000F0BC
:100FC00085BB38BDC8230020B4410008C8320020CA
:100FD000B023002000B59BB0EFF30981682268467A
:100FE000FFF71CFFEFF30583044B9A6BDA6A9A6AEA
:100FF0009A6A9A6A9A6A9A6A9B6AFEE700ED00E02A
:1010000000B59BB0EFF3098168226846FFF706FF41
:10101000EFF30583044B9A6B9A6A9A6A9A6A9A6A02
:101020009A6A9B6AFEE700BF00ED00E000B59BB046
:10103000EFF3098168226846FFF7F0FEEFF30583BE
:10104000034B5A6B9A6A9A6A9A6A9A6A9B6AFEE793
:1010500000ED00E0FEE7000030B50A44084D914283
:101060000DD011F8013B5840082340F30004013B28
:101070002C4013F0FF0384EA5000F6D1EFE730BDB7
:101080002083B8ED026843681143016003B118473B
:1010900070470000024A136843F0C00313607047B2
:1010A00000480040024A136843F0C00313607047D1
:1010B00000500040024A136843F0C00313607047B9
:1010C0000078004037B5274C274D204600F0F2FA53
:1010D00004F11400009400234FF40072234900F03F
:1010E000B3F94FF40072224904F138000094214B07
:1010F00000F02CFA204BC4E91735204C204600F0B4
:10110000D9FA04F11400009400234FF400721C4932
:1011100000F09AF94FF400721A4904F13800009473
:10112000194B00F013FA194BC4E91735184C204637
:1011300000F0C0FA04F1140000234FF400721549C6
:10114000009400F081F9144B4FF40072134904F13C
:101150003800009400F0FAF9114BC4E9173503B0D8
:1011600030BD00BFCC23002000E1F5051025002094
:10117000102B002095100008004800403824002063
:1011800010270020102D0020A5100008005000405E
:10119000A424002010290020B5100008102F0020E2
:1011A00000780040037C30B5334C002918BF0C4652
:1011B000012B18D1314B98420FD1314BD3F8E82095
:1011C00042F48022C3F8E820D3F8102142F48022B0
:1011D000C3F81021D3F8103105E02A4B98422FD0E4
:1011E000294B984238D02268036EC16D03EB52033D
:1011F0008466B3FBF2F36268150442BF23F007056F
:1012000003F0070343EA4503CB60A36843F04003C0
:101210004B60E36843F001038B6042F4967343F044
:1012200001030B604FF0FF330B62510505D512F03F
:1012300010221DD0B2F1805F1CD080F8643030BD28
:101240000F4BD3F8E82042F48012C3F8E820D3F81B
:10125000102142F48012BBE7094BD3F8E82042F09A
:101260008042C3F8E820D3F8102142F08042AFE773
:101270007F23E2E73F23E0E7C4410008CC230020BE
:101280000044025838240020A42400202DE9F0470F
:10129000C66D05463768F4692107346219D014F029
:1012A000080118BF8021E20748BF41F02001A307D1
:1012B0004FF0200348BF41F04001600748BF41F4B0
:1012C000807183F31188281DFFF7DCFE002383F370
:1012D0001188E2050AD5202383F311884FF40071A9
:1012E000281DFFF7CFFE002383F311884FF020095C
:1012F0004FF0000A14F0200838D13B0616D54FF005
:10130000200905F1380A200610D589F311885046C6
:1013100000F050F9002836DA0821281DFFF7B2FE48
:1013200027F080033360002383F31188790614D5F6
:10133000620612D5202383F31188D5E913239A423C
:1013400008D12B6C33B127F040071021281DFFF77F
:1013500099FE3760002383F31188E30618D5AA6E3F
:101360001369ABB15069BDE8F047184789F311889C
:10137000736A284695F86410194000F0B5F98AF3AD
:101380001188F469B6E7B06288F31188F469BAE7A6
:10139000BDE8F087F8B51546826804460B46AA42B8
:1013A00000D28568A1692669761AB5420BD2184623
:1013B0002A46FFF733FDA3692B44A3612846A3689F
:1013C0005B1BA360F8BD0CD9AF1B18463246FFF774
:1013D00025FD3A46E1683044FFF720FDE3683B44D1
:1013E000EBE718462A46FFF719FDE368E5E700003A
:1013F00083689342F7B50446154600D28568D4E960
:101400000460361AB5420BD22A46FFF707FD63691E
:101410002B4463612846A3685B1BA36003B0F0BD47
:101420000DD93246AF1B0191FFF7F8FC01993A46FE
:10143000E0683144FFF7F2FCE3683B44E9E72A4601
:10144000FFF7ECFCE368E4E710B50A440024C3614D
:10145000029B8460C16002610362C0E90000C0E9D0
:10146000051110BD08B5D0E90532934201D182685B
:1014700082B98268013282605A1C4261197000216F
:10148000D0E904329A4224BFC368436100F0DAFE17
:10149000002008BD4FF0FF30FBE7000070B52023AF
:1014A00004460E4683F31188A568A5B1A368A26916
:1014B000013BA360531CA36115782269934224BFAA
:1014C000E368A361E3690BB120469847002383F3E7
:1014D0001188284607E03146204600F0A3FE002888
:1014E000E2DA85F3118870BD2DE9F74F04460E4608
:1014F00017469846D0F81C904FF0200A8AF31188BE
:101500004FF0000B154665B12A4631462046FFF7DD
:1015100041FF034660B94146204600F083FE0028A3
:10152000F1D0002383F31188781B03B0BDE8F08F5E
:10153000B9F1000F03D001902046C847019B8BF3FF
:101540001188ED1A1E448AF31188DCE7C160C3617B
:10155000009B82600362C0E905111144C0E90000EC
:1015600001617047F8B504460D461646202383F303
:101570001188A768A7B1A368013BA36063695A1CDF
:1015800062611D70D4E904329A4224BFE36863614A
:10159000E3690BB120469847002080F3118807E0EB
:1015A0003146204600F03EFE0028E2DA87F311883B
:1015B000F8BD0000D0E9052310B59A4201D1826838
:1015C0007AB982680021013282605A1C82611C78DB
:1015D00003699A4224BFC368836100F033FE20464A
:1015E00010BD4FF0FF30FBE72DE9F74F04460E46E4
:1015F00017469846D0F81C904FF0200A8AF31188BD
:101600004FF0000B154665B12A4631462046FFF7DC
:10161000EFFE034660B94146204600F003FE002875
:10162000F1D0002383F31188781B03B0BDE8F08F5D
:10163000B9F1000F03D001902046C847019B8BF3FE
:101640001188ED1A1E448AF31188DCE702684368AA
:101650001143016003B11847704700001430FFF7D1
:1016600043BF00004FF0FF331430FFF73DBF0000D1
:101670003830FFF7B9BF00004FF0FF333830FFF7C5
:10168000B3BF00001430FFF709BF00004FF0FF3177
:101690001430FFF703BF00003830FFF763BF0000CE
:1016A0004FF0FF323830FFF75DBF00000020704779
:1016B000FFF708BD044B036000234360C0E9023319
:1016C00001230374704700BFDC41000810B52023DC
:1016D000044683F31188FFF765FD0223237400237A
:1016E00083F3118810BD000038B5C36904460D4668
:1016F0001BB904210844FFF7A9FF294604F114008F
:10170000FFF7B0FE002806DA201D4FF48061BDE827
:101710003840FFF79BBF38BD026843681143016042
:1017200003B118477047000013B5406B00F58054B3
:10173000D4F8A4381A681178042914D1017C02293C
:1017400011D11979012312898B4013420BD101A9C0
:101750004C3002F06FF8D4F8A4480246019B21797E
:10176000206800F0DFF902B010BD0000143001F075
:10177000F1BF00004FF0FF33143001F0EBBF000069
:101780004C3002F0C3B800004FF0FF334C3002F091
:10179000BDB80000143001F0BFBF00004FF0FF31B2
:1017A000143001F0B9BF00004C3002F08FB80000D7
:1017B0004FF0FF324C3002F089B800000020704733
:1017C00010B500F58054D4F8A4381A6811780429AB
:1017D00017D1017C022914D15979012352898B40F8
:1017E00013420ED1143001F051FF024648B1D4F833
:1017F000A4484FF4407361792068BDE8104000F0C0
:101800007FB910BD406BFFF7DBBF000070470000E1
:101810007FB5124B0125042604460360002305749E
:1018200000F1840243602946C0E902330C4B029068
:10183000143001934FF44073009601F003FF094BFD
:1018400004F69442294604F14C000294CDE9006369
:101850004FF4407301F0CAFF04B070BD04420008A9
:1018600005180008291700080A68202383F3118847
:101870000B790B3342F823004B79133342F82300E2
:101880008B7913B10B3342F8230000F58053C3F872
:10189000A41802230374002383F311887047000007
:1018A00038B5037F044613B190F85430ABB9012525
:1018B000201D0221FFF730FF04F114006FF0010139
:1018C000257700F0CBFC04F14C0084F854506FF005
:1018D0000101BDE8384000F0C1BC38BD10B50121A0
:1018E00004460430FFF718FF0023237784F85430B0
:1018F00010BD000038B504460025143001F0BAFED2
:1019000004F14C00257701F089FF201D84F8545024
:101910000121FFF701FF2046BDE83840FFF750BF27
:1019200090F8803003F06003202B06D190F88120DE
:101930000023212A03D81F2A06D800207047222A14
:10194000FBD1C0E91D3303E0034A426707228267E7
:10195000C3670120704700BF2C22002037B500F577
:101960008055D5F8A4381A68117804291AD1017C59
:10197000022917D11979012312898B40134211D101
:1019800000F14C04204602F009F858B101A92046A4
:1019900001F050FFD5F8A4480246019B2179206848
:1019A00000F0C0F803B030BD01F10B03F0B550F802
:1019B000236085B004460D46FEB1202383F31188D1
:1019C00004EB8507301D0821FFF7A6FEFB6806F132
:1019D0004C005B691B681BB1019001F039FF019855
:1019E00003A901F027FF024648B1039B2946204680
:1019F00000F098F8002383F3118805B0F0BDFB6870
:101A00005A691268002AF5D01B8A013B1340F1D1B4
:101A100004F18002EAE70000133138B550F82140A4
:101A2000ECB1202383F3118804F58053D3F8A42864
:101A30001368527903EB8203DB689B695D6845B1EB
:101A400004216018FFF768FE294604F1140001F034
:101A500027FE2046FFF7B4FE002383F3118838BD2C
:101A60007047000001F01AB901234022002110B58F
:101A7000044600F8303BFFF7F7F90023C4E90133CF
:101A800010BD000010B52023044683F311882422E2
:101A9000416000210C30FFF7E7F9204601F020F902
:101AA00002232370002383F3118810BD70B500EB6F
:101AB0008103054650690E461446DA6018B11022BB
:101AC0000021FFF7D1F9A06918B110220021FFF71A
:101AD000CBF931462846BDE8704001F013BA00004A
:101AE00083682022002103F0011310B504468360AF
:101AF0001030FFF7B9F92046BDE8104001F08EBA6A
:101B0000F0B4012500EB810447898D40E4683D4332
:101B1000A469458123600023A2606360F0BC01F0EA
:101B2000ABBA0000F0B4012500EB810407898D40B9
:101B3000E4683D436469058123600023A26063601B
:101B4000F0BC01F021BB000070B502230025044663
:101B5000242203702946C0F888500C3040F8045CF9
:101B6000FFF782F9204684F8705001F05FF963684E
:101B70001B6823B129462046BDE87040184770BD58
:101B8000037880F88C300523037043681B6810B518
:101B900004460BB1042198470023A36010BD000048
:101BA00090F88C20436802701B680BB10521184720
:101BB0007047000070B590F87030044613B10023F0
:101BC00080F8703004F18002204601F04BFA63681F
:101BD0009B68B3B994F8803013F0600535D00021CC
:101BE000204601F0F5FC0021204601F0E5FC636889
:101BF0001B6813B1062120469847062384F87030ED
:101C000070BD204698470028E4D0B4F88630A26F13
:101C10009A4288BFA36794F98030A56F002B4FF0DC
:101C2000200380F20381002D00F0F280092284F865
:101C3000702083F3118800212046D4E91D23FFF78B
:101C400071FF002383F31188DAE794F8812003F011
:101C50007F0343EA022340F20232934200F0C58040
:101C600021D8B3F5807F48D00DD8012B3FD0022B6F
:101C700000F09380002BB2D104F188026267022247
:101C8000A267E367C1E7B3F5817F00F09B80B3F5FE
:101C9000407FA4D194F88230012BA0D1B4F88830D1
:101CA00043F0020332E0B3F5006F4DD017D8B3F51F
:101CB000A06F31D0A3F5C063012B90D86368204694
:101CC00094F882205E6894F88310B4F88430B047AA
:101CD000002884D0436863670368A3671AE0B3F5FC
:101CE000106F36D040F6024293427FF478AF5C4BDF
:101CF00063670223A3670023C3E794F88230012BB4
:101D00007FF46DAFB4F8883023F00203A4F8883074
:101D1000C4E91D55E56778E7B4F88030B3F5A06FE6
:101D20000ED194F88230204684F88A3001F0DCF835
:101D300063681B6813B10121204698470323237071
:101D40000023C4E91D339CE704F18B03636701237F
:101D5000C3E72378042B10D1202383F31188204676
:101D6000FFF7BEFE85F311880321636884F88B506A
:101D700021701B680BB12046984794F88230002BE5
:101D8000DED084F88B300423237063681B68002B3B
:101D9000D6D0022120469847D2E794F884302046D6
:101DA0001D0603F00F010AD501F04EF9012804D0F9
:101DB00002287FF414AF2B4B9AE72B4B98E701F0E6
:101DC00035F9F3E794F88230002B7FF408AF94F8EC
:101DD000843013F00F01B3D01A06204602D501F06B
:101DE0000FFCADE701F000FCAAE794F88230002B6D
:101DF0007FF4F5AE94F8843013F00F01A0D01B06E9
:101E0000204602D501F0E4FB9AE701F0D5FB97E705
:101E1000142284F8702083F311882B462A46294621
:101E20002046FFF76DFE85F31188E9E65DB11522C6
:101E300084F8702083F3118800212046D4E91D2303
:101E4000FFF75EFEFDE60B2284F8702083F3118815
:101E50002B462A4629462046FFF764FEE3E700BFEB
:101E6000344200082C4200083042000838B590F88F
:101E700070300446002B3ED0063BDAB20F2A34D82D
:101E80000F2B32D8DFE803F03731310822323131FD
:101E90003131313131313737856FB0F886309D427D
:101EA00014D2C3681B8AB5FBF3F203FB12556DB95C
:101EB000202383F311882B462A462946FFF732FE5A
:101EC00085F311880A2384F870300EE0142384F817
:101ED0007030202383F31188002320461A461946C8
:101EE000FFF70EFE002383F3118838BDC36F03B1E3
:101EF00098470023E7E70021204601F069FB002115
:101F0000204601F059FB63681B6813B10621204687
:101F100098470623D7E7000010B590F870300446C4
:101F2000142B29D017D8062B05D001D81BB110BD12
:101F3000093B022BFBD80021204601F049FB002180
:101F4000204601F039FB63681B6813B10621204667
:101F50009847062319E0152BE9D10B2380F8703040
:101F6000202383F3118800231A461946FFF7DAFD70
:101F7000002383F31188DAE7C3689B695B68002B51
:101F8000D5D1C36F03B19847002384F87030CEE7F2
:101F9000024B0022C3E900339A60704710310020E1
:101FA000002382680374054B1B6899689142FBD239
:101FB0005A6803604260106058607047103100201A
:101FC00008B5202383F31188037C032B05D0042B51
:101FD0000DD02BB983F3118808BD436900221A6024
:101FE0004FF0FF334361FFF7DBFF0023F2E7D0E957
:101FF000003213605A60F3E7002382680374054BD4
:102000001B6899689142FBD85A680360426010606F
:102010005860704710310020054B19690874186822
:10202000026853601A60186101230374FEF7CEB989
:10203000103100204B1C30B5044687B00A4D10D03B
:102040002B6901A8094A00F025F92046FFF7E4FFB3
:10205000049B13B101A800F059F92B69586907B026
:1020600030BDFFF7D9FFF8E710310020C11F00088D
:1020700038B50C4D044641612B6981689A689142DC
:1020800003D8BDE83840FFF78BBF1846FFF7B4FF11
:1020900001232C61014623742046BDE83840FEF739
:1020A00095B900BF10310020044B1A681B69906875
:1020B0009B68984294BF0020012070471031002097
:1020C00010B5084C236820691A6854602260012208
:1020D00023611A74FFF790FF01462069BDE81040A4
:1020E000FEF774B91031002008B5FFF7DDFF18B115
:1020F000BDE80840FFF7E4BF08BD0000FFF7E0BF00
:10210000FEE7000010B50C4CFFF742FF00F0B4F8FA
:1021100080220A49204600F03BF8012344F8180CBD
:10212000037400F099FC002383F3118862B604481D
:10213000BDE8104000F04CB83831002038420008AB
:102140004842000800F01CB9EFF3118020B9EFF30A
:102150000583202282F311887047000010B530B942
:10216000EFF30584C4F3080414B180F3118810BDA3
:10217000FFF7BAFF84F31188F9E70000034A5168BA
:1021800053685B1A9842FBD8704700BF001000E00C
:1021900082600222028270478368A3F17C0243F8C6
:1021A0000C2C026943F83C2C426943F8382C074A4E
:1021B00043F81C2CC268A3F1180043F8102C02222B
:1021C00003F8082C002203F8072C7047E5030008E9
:1021D00010B5202383F31188FFF7DEFF00210446AA
:1021E000FFF746FF002383F31188204610BD00004F
:1021F000024B1B6958610F20FFF70EBF1031002002
:10220000202383F31188FFF7F3BF000008B50146D0
:10221000202383F311880820FFF70CFF002383F3AA
:10222000118808BD49B1064B42681B6918605A60A5
:10223000136043600420FFF7FDBE4FF0FF3070478E
:10224000103100200368984206D01A68026050607E
:1022500018465961FFF7A4BE7047000038B5044620
:102260000D462068844200D138BD036823605C605D
:102270004561FFF795FEF4E7054B4FF0FF3103F1A1
:102280001402C3E905220022C3E90712704700BF08
:102290001031002070B51C4E05460C46C0E90323E2
:1022A00001F0B2FB334653F8142F9A420DD130623D
:1022B0000A2C2CBF00190A302A60C5E90124C6E99E
:1022C0000555BDE8704001F089BB316A431AE31837
:1022D00038BF1C469368A34202D9081901F08EFB4F
:1022E00073699A6894420CD85A68AC602B606A6033
:1022F00015609A685D60121B9A604FF0FF33F361BE
:1023000070BDA41A1B68ECE71031002038B51B4CD7
:10231000636998420DD08168D0E9003213605A6039
:102320000022C2609A680A449A604FF0FF33E3616A
:1023300038BD03682246002142F8143F93425A6098
:10234000C16003D1BDE8384001F052BB9A68816892
:10235000256A0A449A6001F057FB6369411B9A6839
:102360008A42E5D9AB181D1A206A092D98BF01F1E0
:102370000A02BDE83840104401F040BB1031002093
:102380002DE9F041184C002704F11406656901F0AD
:102390003BFB236AAA68C11A8A4215D81344D5F8B0
:1023A0000C802362D5E9003213605A606369EF60E4
:1023B000B34201D101F01CFB87F311882869C047A3
:1023C000202383F31188E1E76169B14209D0134406
:1023D0001B1ABDE8F0410A2B2CBFC0180A3001F0CF
:1023E0000DBBBDE8F08100BF103100200020704718
:1023F000FEE70000704700004FF0FF30704700001C
:1024000002290CD0032904D00129074818BF002055
:102410007047032A05D8054800EBC20070470448FE
:1024200070470020704700BF284300083C2200206E
:10243000DC42000870B59AB005460846144601A96A
:1024400000F0C2F801A8FEF707FD431C0022C6B247
:102450005B001046C5E9003423700323023404F8FE
:10246000013C01ABD1B202348E4201D81AB070BD2A
:1024700013F8011B013204F8010C04F8021CF1E707
:1024800008B5202383F311880348FFF767FA002378
:1024900083F3118808BD00BFC832002090F8803057
:1024A00003F01F02012A07D190F881200B2A03D1E3
:1024B0000023C0E91D3315E003F06003202B08D191
:1024C000B0F884302BB990F88120212A03D81F2A34
:1024D00004D8FFF725BA222AEBD0FAE7034A42676D
:1024E00007228267C3670120704700BF33220020A4
:1024F00007B5052917D8DFE801F0191603191920C7
:10250000202383F31188104A01210190FFF7CEFAAE
:10251000019802210D4AFFF7C9FA0D48FFF7EAF9C1
:10252000002383F3118803B05DF804FB202383F3B9
:1025300011880748FFF7B4F9F2E7202383F31188E5
:102540000348FFF7CBF9EBE77C420008A042000804
:10255000C832002038B50C4D0C4C2A460C4904F109
:102560000800FFF767FF05F1CA0204F110000949EE
:10257000FFF760FF05F5CA7204F118000649BDE8CF
:102580003840FFF757BF00BFA04B00203C2200207F
:1025900060420008684200087342000870B50446B3
:1025A00008460D46FEF758FCC6B2204601340378B3
:1025B0000BB9184670BD32462946FEF739FC002893
:1025C000F3D10120F6E700002DE9F84F05460C464F
:1025D000FEF742FC2C49C6B22846FFF7DFFF08B1E0
:1025E0000236F6B229492846FFF7D8FF08B110365F
:1025F000F6B2632E0DD8DFF89080DFF89090244F6C
:10260000DFF894A0DFF894B02E7846B92670BDE8C4
:10261000F88F29462046BDE8F84F01F0B5BD252EBC
:102620002ED1072241462846FEF702FC70B9DBF89E
:1026300000300735093444F8093CDBF8043044F82D
:10264000053C9BF8083004F8013CDDE708224946C8
:102650002846FEF7EDFB98B9A21C0E4B1978023202
:102660000909C95D02F8041C13F8011B01F00F01F0
:102670005345C95D02F8031CF0D118340835C3E78F
:10268000013504F8016BBFE74843000873420008B6
:102690005A43000800E8F11F0CE8F11F50430008FE
:1026A000BFF34F8F044B1A695107FCD1D3F81021A7
:1026B0005207F8D1704700BF0020005208B50D4BFB
:1026C0001B78ABB9FFF7ECFF0B4BDA68D10704D5E9
:1026D0000A4A5A6002F188325A60D3F80C21D207B4
:1026E00006D5064AC3F8042102F18832C3F8042152
:1026F00008BD00BFFE4D00200020005223016745A9
:1027000008B5114B1B78F3B9104B1A69510703D563
:10271000DA6842F04002DA60D3F81021520705D59A
:10272000D3F80C2142F04002C3F80C21FFF7B8FFA8
:10273000064BDA6842F00102DA60D3F80C2142F06D
:102740000102C3F80C2108BDFE4D002000200052FC
:102750000F289ABF00F580604004002070470000F9
:102760004FF4003070470000102070470F2808B564
:102770000BD8FFF7EDFF00F500330268013204D1FA
:1027800004308342F9D1012008BD0020FCE700009D
:102790000F2870B5054645D8FFF7D6FC224CFFF749
:1027A0007FFF0646FFF78AFF4FF0FF33072D636177
:1027B000C4F8143120D82361FFF772FF2B0243F0D5
:1027C0002403E360E36843F08003E36023695A076E
:1027D000FCD42846FFF764FF4FF40031FFF7B8FF41
:1027E00000F002F93046FFF78BFFFFF7B7FC2846F1
:1027F000BDE87040FFF7BABFC4F81031FFF750FFD3
:10280000A5F108031B0243F02403C4F80C31D4F8EB
:102810000C3143F08003C4F80C31D4F810315B075D
:10282000FBD4D6E7002070BD002000522DE9F84F00
:1028300040EA020305460C461746D80602D000209F
:10284000BDE8F88F27F01F07DFF8D4B0FFF736FF99
:102850002744BC4203D10120FFF752FFF0E72022BA
:102860002946204601F080FC10B920352034F0E7DD
:102870002B4605F120021E68711CE0D104339A42F8
:10288000F9D1FFF761FC05F17843234AB3F5801FC6
:10289000224B28BF9A4603F1040338BF9046A2F1A9
:1028A000080228BF9846A3F108033ABF9146DA46CA
:1028B0009946FFF7F5FEC8F80060A5EB040CD9F8BF
:1028C000002004F11C0142F00202C9F80020221F7E
:1028D000DAF8006016F00506FAD152F8043F8A4291
:1028E0004CF80230F4D1BFF34F8FFFF7D9FE4FF011
:1028F000FF32C8F80020D9F8002022F00202C9F8FF
:102900000020FFF72BFC20222146284601F02CFC5A
:102910000028AAD030469FE7142000521021005210
:102920001020005210B5084C237828B11BB9FFF7CE
:10293000C5FE0123237010BD002BFCD02070BDE824
:102940001040FFF7DDBE00BFFE4D00200244074BE4
:10295000D2B210B5904200D110BD441C00B253F861
:10296000200041F8040BE0B2F4E700BF50400058EB
:102970000E4B30B51C6F240405D41C6F1C671C6FF4
:1029800044F400441C670A4C02442368D2B243F466
:1029900080732360074B904200D130BD441C51F836
:1029A000045B00B243F82050E0B2F4E70044025860
:1029B000004802585040005807B5012201A90020E4
:1029C000FFF7C4FF019803B05DF804FB13B504469C
:1029D000FFF7F2FFA04205D0012201A900200194D7
:1029E000FFF7C6FF02B010BD0144BFF34F8F064B87
:1029F000884204D3BFF34F8FBFF36F8F7047C3F884
:102A00005C022030F4E700BF00ED00E0034B1A68E1
:102A10001AB9034AD2F8D0241A607047004E002039
:102A20000040025808B5FFF7F1FF024B1868C0F3E9
:102A3000806008BD004E0020EFF30983054968332C
:102A40004A6B22F001024A6383F30988002383F36F
:102A50001188704700EF00E0202080F3118862B6F3
:102A60000D4B0E4AD96821F4E0610904090C0A43B0
:102A70000B49DA60D3F8FC2042F08072C3F8FC20E6
:102A8000084AC2F8B01F116841F00101116010221C
:102A9000DA7783F82200704700ED00E00003FA05C2
:102AA00055CEACC5001000E0202310B583F311888B
:102AB0000E4B5B6813F4006314D0F1EE103AEFF3A1
:102AC00009844FF08073683CE361094BDB6B23663C
:102AD00084F30988FFF7E8FA10B1064BA36110BD33
:102AE000054BFBE783F31188F9E700BF00ED00E039
:102AF00000EF00E0F7030008FA03000870B5BFF329
:102B00004F8FBFF36F8F1A4A0021C2F85012BFF3E4
:102B10004F8FBFF36F8F536943F400335361BFF39B
:102B20004F8FBFF36F8FC2F88410BFF34F8FD2F86F
:102B3000803043F6E074C3F3C900C3F34E335B0146
:102B400003EA0406014646EA81750139C2F860527B
:102B5000F9D2203B13F1200FF2D1BFF34F8F53690D
:102B600043F480335361BFF34F8FBFF36F8F70BD5A
:102B700000ED00E0FEE700000A4B0B480B4A9042D4
:102B80000BD30B4BC11EDA1C121A22F003028B422C
:102B900038BF00220021FEF767B953F8041B40F844
:102BA000041BECE73C450008D44F0020D44F002024
:102BB000D44F00207047000070B5D0E924430022B4
:102BC0004FF0FF359E6804EB42135101D3F8000922
:102BD000002805DAD3F8000940F08040C3F8000966
:102BE000D3F8000B002805DAD3F8000B40F0804042
:102BF000C3F8000B013263189642C3F80859C3F8B2
:102C0000085BE0D24FF00113C4F81C3870BD00001F
:102C100000EB8103D3F80CC02DE9F043DCF814205D
:102C20004E1CD0F89050D2F800E005EB063605EBCC
:102C30004118506870450AD30122D5F8343802FA99
:102C400001F123EA0101C5F83418BDE8F083AEEBC9
:102C50000003BCF81040A34228BF2346D8F8184907
:102C6000A4B2B3EB840FF0D89468A4F1040959F826
:102C7000047F3760A4EB09071F44042FF7D81C44D6
:102C8000034494605360D4E7890141F0200101615D
:102C900003699B06FCD41220FFF770BA10B50A4CEA
:102CA0002046FEF7E1FE094BC4F89030084BC4F80B
:102CB0009430084C2046FEF7D7FE074BC4F89030FE
:102CC000064BC4F8943010BD044E002000000840AC
:102CD00090430008A04E0020000004409C430008E0
:102CE00070B503780546012B5DD1494BD0F8904073
:102CF000984259D1474B0E216520D3F8D82042F095
:102D00000062C3F8D820D3F8002142F00062C3F873
:102D10000021D3F80021D3F8802042F00062C3F8EC
:102D20008020D3F8802022F00062C3F88020D3F8FE
:102D3000803000F071FC384BE360384BC4F8003849
:102D40000023D5F89060C4F8003EC02323604FF400
:102D50000413A3633369002BFCDA01230C203361D5
:102D6000FFF70CFA3369DB07FCD41220FFF706FAF1
:102D70003369002BFCDA00262846A660FFF71CFF0B
:102D80006B68C4F81068DB68C4F81468C4F81C6881
:102D9000002B3AD1224BA3614FF0FF336361A3684C
:102DA00043F00103A36070BD1E4B9842C8D1194B7C
:102DB0000E214D20D3F8D82042F00072C3F8D8205D
:102DC000D3F8002142F00072C3F80021D3F80021AB
:102DD000D3F8802042F00072C3F88020D3F880201E
:102DE00022F00072C3F88020D3F88020D3F8D820D6
:102DF00022F08062C3F8D820D3F8002122F080624C
:102E0000C3F80021D3F8003193E7074BC3E700BFB5
:102E1000044E0020004402584014004003002002E9
:102E2000003C30C0A04E0020083C30C0F8B5D0F8BF
:102E30009040054600214FF000662046FFF724FF32
:102E4000D5F8941000234FF001128F684FF0FF3037
:102E5000C4F83438C4F81C2804EB431201339F42F1
:102E6000C2F80069C2F8006BC2F80809C2F8080B82
:102E7000F2D20B68D5F89020C5F898306362102321
:102E80001361166916F01006FBD11220FFF776F9D0
:102E9000D4F8003823F4FE63C4F80038A36943F47F
:102EA000402343F01003A3610923C4F81038C4F889
:102EB00014380B4BEB604FF0C043C4F8103B094B88
:102EC000C4F8003BC4F81069C4F80039D5F898304C
:102ED00003F1100243F48013C5F89820A362F8BDF3
:102EE0006C43000840800010D0F8902090F88A10C1
:102EF000D2F8003823F4FE6343EA0113C2F8003825
:102F0000704700002DE9F84300EB8103D0F89050A2
:102F10000C468046DA680FFA81F94801166806F017
:102F20000306731E022B05EB41134FF0000194BF03
:102F3000B604384EC3F8101B4FF0010104F1100322
:102F400098BF06F1805601FA03F3916998BF06F520
:102F5000004600293AD0578A04F158013743490105
:102F60006F50D5F81C180B430021C5F81C382B18DE
:102F70000127C3F81019A7405369611E9BB3138A38
:102F8000928B9B08012A88BF5343D8F89820981841
:102F900042EA034301F140022146C8F8980028465E
:102FA00005EB82025360FFF76FFE08EB8900C368F0
:102FB0001B8A43EA845348341E4364012E51D5F8DA
:102FC0001C381F43C5F81C78BDE8F88305EB49178A
:102FD000D7F8001B21F40041C7F8001BD5F81C18D6
:102FE00021EA0303C0E704F13F030B4A28462146C8
:102FF00005EB83035A60FFF747FE05EB4910D0F855
:10300000003923F40043C0F80039D5F81C3823EA0E
:103010000707D7E70080001000040002D0F89420D2
:103020001268C0F89820FFF7C7BD00005831D0F8EB
:10303000903049015B5813F4004004D013F4001F92
:103040000CBF0220012070474831D0F89030490170
:103050005B5813F4004004D013F4001F0CBF02208F
:103060000120704700EB8101CB68196A0B6813607F
:103070004B6853607047000000EB810330B5DD689A
:10308000AA691368D36019B9402B84BF4023136029
:103090006B8A1468D0F890201C4402EB4110013C6C
:1030A00009B2B4FBF3F46343033323F0030343EAAD
:1030B000C44343F0C043C0F8103B2B6803F0030344
:1030C000012B0ED1D2F8083802EB411013F4807FA7
:1030D000D0F8003B14BF43F0805343F00053C0F8D6
:1030E000003B02EB4112D2F8003B43F00443C2F82C
:1030F000003B30BD2DE9F041D0F8906005460C460C
:1031000006EB4113D3F8087B3A07C3F8087B08D5D0
:10311000D6F814381B0704D500EB8103DB685B6825
:103120009847FA071FD5D6F81438DB071BD505EBEF
:103130008403D968CCB98B69488A5A68B2FBF0F627
:1031400000FB16228AB91868DA6890420DD2121A6A
:10315000C3E90024202383F3118821462846FFF782
:103160008BFF84F31188BDE8F081012303FA04F298
:103170006B8923EA02036B81CB68002BF3D02146D5
:103180002846BDE8F041184700EB81034A0170B5BD
:10319000DD68D0F890306C692668E66056BB1A444A
:1031A0004FF40020C2F810092A6802F00302012A35
:1031B0000AB20ED1D3F8080803EB421410F4807F52
:1031C000D4F8000914BF40F0805040F00050C4F81B
:1031D000000903EB4212D2F8000940F00440C2F8A3
:1031E00000090122D3F8340802FA01F10143C3F8BF
:1031F000341870BD19B9402E84BF4020206020686B
:103200001A442E8A8419013CB4FBF6F440EAC44007
:1032100040F00050C6E700002DE9F041D0F8906082
:1032200004460D4606EB4113D3F80879C3F8087934
:10323000FB071CD5D6F81038DA0718D500EB810348
:10324000D3F80CC0DCF81430D3F800E0DA68964507
:103250001BD2A2EB0E024FF000081A60C3F80480E4
:10326000202383F31188FFF78FFF88F311883B0633
:1032700018D50123D6F83428AB40134212D0294682
:103280002046BDE8F041FFF7C3BC012303FA01F279
:10329000038923EA02030381DCF80830002BE6D01F
:1032A0009847E4E7BDE8F0812DE9F84FD0F8905059
:1032B00004466E69AB691E4016F480586E6103D0F7
:1032C000BDE8F84FFEF740BC002E12DAD5F8003EFC
:1032D0009F0705D0D5F8003E23F00303C5F8003E54
:1032E000D5F80438204623F00103C5F80438FEF76A
:1032F00057FC300505D52046FFF75EFC2046FEF75B
:103300003FFCB1040CD5D5F8083813F0060FEB6874
:1033100023F470530CBF43F4105343F4A053EB60F9
:10332000320704D56368DB680BB120469847F30287
:1033300000F1BA80B70226D5D4F8909000274FF05C
:10334000010A09EB4712D2F8003B03F44023B3F51E
:10335000802F11D1D2F8003B002B0DDA62890AFAD6
:1033600007F322EA0303638104EB8703DB68DB686E
:1033700013B13946204698470137D4F89430FFB24C
:103380009B689F42DDD9F00619D5D4F89000026AF7
:10339000C2F30A1702F00F0302F4F012B2F5802F05
:1033A00000F0CC80B2F5402F09D104EB830300225A
:1033B00000F58050DB681B6A974240F0B280300312
:1033C000D5F8185835D5E90303D500212046FFF775
:1033D00091FEAA0303D501212046FFF78BFE6B0364
:1033E00003D502212046FFF785FE2F0303D50321D5
:1033F0002046FFF77FFEE80203D504212046FFF7B1
:1034000079FEA90203D505212046FFF773FE6A0263
:1034100003D506212046FFF76DFE2B0203D50721B9
:103420002046FFF767FEEF0103D508212046FFF78E
:1034300061FE700340F1A980E90703D50021204611
:10344000FFF7EAFEAA0703D501212046FFF7E4FEB5
:103450006B0703D502212046FFF7DEFE2F0703D5B9
:1034600003212046FFF7D8FEEE0603D504212046AF
:10347000FFF7D2FEA80603D505212046FFF7CCFEB4
:10348000690603D506212046FFF7C6FE2A0603D5A6
:1034900007212046FFF7C0FEEB0576D52046082120
:1034A000BDE8F84FFFF7B8BED4F8909000274FF072
:1034B000010AD4F894305FFA87FB9B689B453FF67E
:1034C00039AF09EB4B13D3F8002902F44022B2F5CF
:1034D000802F24D1D3F80029002A20DAD3F800293C
:1034E00042F09042C3F80029D3F80029002AFBDB00
:1034F0005946D4F89000FFF7C7FB22890AFA0BF36C
:1035000022EA0303238104EB8B03DB689B6813B17E
:1035100059462046984759462046FFF779FB013720
:10352000C7E7910701D1D0F80080072A02F1010214
:103530009CBF03F8018B4FEA18283DE704EB830397
:1035400000F58050DA68D2F818C0DCF80820DCE911
:10355000001CA1EB0C0C00218F4208D1DB689B6999
:103560009A683A449A605A683A445A6027E711F0D8
:10357000030F01D1D0F800808C4501F1010184BF17
:1035800002F8018B4FEA1828E6E7BDE8F88F000043
:1035900008B50348FFF788FEBDE80840FFF784BA86
:1035A000044E002008B50348FFF77EFEBDE8084042
:1035B000FFF77ABAA04E0020D0F8903003EB41110B
:1035C000D1F8003B43F40013C1F8003B7047000002
:1035D000D0F8903003EB4111D1F8003943F40013D7
:1035E000C1F8003970470000D0F8903003EB41116A
:1035F000D1F8003B23F40013C1F8003B70470000F2
:10360000D0F8903003EB4111D1F8003923F40013C6
:10361000C1F8003970470000090100F16043012240
:1036200003F56143C9B283F8001300F01F039A4009
:1036300043099B0003F1604303F56143C3F8802114
:103640001A60704730B50433039C0172002104FBFB
:103650000325C160C0E90653049B0363059BC0E9D1
:103660000000C0E90422C0E90842C0E90A1143632E
:1036700030BD00000022416AC260C0E90411C0E907
:103680000A226FF00101FEF7E9BD0000D0E9043223
:10369000934201D1C2680AB9181D704700207047D3
:1036A000036919600021C2680132C260C269134413
:1036B00082699342036124BF436A0361FEF7C2BD7E
:1036C00038B504460D46E3683BB162690020131D1E
:1036D0001268A3621344E36207E0237A33B92946F0
:1036E0002046FEF79FFD0028EDDA38BD6FF001009F
:1036F000FBE70000C368C269013BC3604369134430
:1037000082699342436124BF436A43610023836219
:10371000036B03B11847704770B52023044683F349
:103720001188866A3EB9FFF7CBFF054618B186F3CC
:103730001188284670BDA36AE26A13F8015B9342C0
:10374000A36202D32046FFF7D5FF002383F311883D
:10375000EFE700002DE9F84F04460E46174698465D
:103760004FF0200989F311880025AA46D4F828B023
:10377000BBF1000F09D141462046FFF7A1FF20B160
:103780008BF311882846BDE8F88FD4E90A12A7EB1D
:10379000050B521A934528BF9346BBF1400F1BD926
:1037A000334601F1400251F8040B914243F8040BF7
:1037B000F9D1A36A403640354033A362D4E90A23E5
:1037C0009A4202D32046FFF795FF8AF31188BD4243
:1037D000D8D289F31188C9E730465A46FDF71EFB57
:1037E000A36A5E445D445B44A362E7E710B5029CB4
:1037F0000433017204FB0321C460C0E906130023F3
:10380000C0E90A33039B0363049BC0E90000C0E9DD
:103810000422C0E90842436310BD0000026A6FF051
:103820000101C260426AC0E904220022C0E90A2202
:10383000FEF714BDD0E904239A4201D1C26822B92F
:10384000184650F8043B0B6070470020704700009A
:10385000C3680021C2690133C360436913448269AC
:103860009342436124BF436A4361FEF7EBBC00000F
:1038700038B504460D46E3683BB1236900201A1DA4
:10388000A262E2691344E36207E0237A33B929466E
:103890002046FEF7C7FC0028EDDA38BD6FF00100C6
:1038A000FBE7000003691960C268013AC260C2699F
:1038B000134482699342036124BF436A0361002376
:1038C0008362036B03B118477047000070B5202373
:1038D0000D460446114683F31188866A2EB9FFF718
:1038E000C7FF10B186F3118870BDA36A1D70A36A6B
:1038F000E26A01339342A36204D3E16920460439AA
:10390000FFF7D0FF002080F31188EDE72DE9F84F95
:1039100004460D46904699464FF0200A8AF31188D6
:103920000026B346A76A4FB949462046FFF7A0FFD5
:1039300020B187F311883046BDE8F88FD4E90A0733
:103940003A1AA8EB0607974228BF1746402F1BD903
:1039500005F1400355F8042B9D4240F8042BF9D1A2
:10396000A36A40364033A362D4E90A239A4204D3BF
:10397000E16920460439FFF795FF8BF3118846452E
:10398000D9D28AF31188CDE729463A46FDF746FA9F
:10399000A36A3D443E443B44A362E5E7D0E90423E7
:1039A0009A4217D1C3689BB1836A8BB1043B9B1ABF
:1039B0000ED01360C368013BC360C3691A448369B6
:1039C0009A42026124BF436A036100238362012398
:1039D000184670470023FBE700F0DAB8034B0022DB
:1039E00058631A610222DA60704700BF000C004081
:1039F000014B0022DA607047000C0040014B586315
:103A0000704700BF000C0040014B586A704700BF70
:103A1000000C00404B6843608B688360CB68C360D8
:103A20000B6943614B6903628B6943620B680360F6
:103A30007047000008B53C4B40F2FF713B48D3F89B
:103A400088200A43C3F88820D3F8882022F4FF6234
:103A500022F00702C3F88820D3F88820D3F8E020AA
:103A60000A43C3F8E020D3F808210A43C3F8082129
:103A70002F4AD3F808311146FFF7CCFF00F58060DC
:103A800002F11C01FFF7C6FF00F5806002F138016A
:103A9000FFF7C0FF00F5806002F15401FFF7BAFFA5
:103AA00000F5806002F17001FFF7B4FF00F580605F
:103AB00002F18C01FFF7AEFF00F5806002F1A80172
:103AC000FFF7A8FF00F5806002F1C401FFF7A2FF35
:103AD00000F5806002F1E001FFF79CFF00F58060D7
:103AE00002F1FC01FFF796FF02F58C7100F5806092
:103AF000FFF790FF00F000F90E4BD3F8902242F050
:103B00000102C3F89022D3F8942242F00102C3F8D4
:103B100094220522C3F898204FF06052C3F89C20ED
:103B2000054AC3F8A02008BD00440258000002580E
:103B3000A843000800ED00E01F00080308B500F0EE
:103B4000F3FAFEF7DFFA0F4BD3F8DC2042F0400225
:103B5000C3F8DC20D3F8042122F04002C3F804218A
:103B6000D3F80431084B1A6842F008021A601A6848
:103B700042F004021A60FEF749FFBDE80840FEF774
:103B8000E9BC00BF0044025800180248704700001A
:103B9000114BD3F8E82042F00802C3F8E820D3F82C
:103BA000102142F00802C3F810210C4AD3F810315A
:103BB000D36B43F00803D363C722094B9A624FF0DB
:103BC000FF32DA6200229A615A63DA605A60012297
:103BD0005A611A60704700BF004402580010005C30
:103BE000000C0040094A08B51169D3680B40D9B2EE
:103BF0009B076FEA0101116107D5202383F3118828
:103C0000FEF7A0FA002383F3118808BD000C0040E2
:103C1000384B4FF0FF31D3F88020C3F88010D3F831
:103C200080200022C3F88020D3F88000D3F88400DD
:103C3000C3F88410D3F88400C3F88420D3F8840038
:103C4000D86F40F0FF4040F4FF0040F43F5040F098
:103C50003F00D867D86F20F0FF4020F4FF0020F429
:103C60003F5020F03F00D867D86FD3F888006FEA44
:103C700040506FEA5050C3F88800D3F88800C0F372
:103C80000A00C3F88800D3F88800D3F89000C3F87E
:103C90009010D3F89000C3F89020D3F89000D3F898
:103CA0009400C3F89410D3F89400C3F89420D3F888
:103CB0009400D3F89800C3F89810D3F89800C3F88C
:103CC0009820D3F89800D3F88C00C3F88C10D3F860
:103CD0008C00C3F88C20D3F88C00D3F89C00C3F878
:103CE0009C10D3F89C10C3F89C20D3F89C3000F0B3
:103CF000E7B900BF00440258614B0122C3F8082114
:103D0000604BD3F8F42042F00202C3F8F420D3F859
:103D10001C2142F00202C3F81C210222D3F81C31FC
:103D2000594BDA605A689104FCD5584A1A6001224E
:103D30009A60574ADA6000221A614FF440429A6151
:103D4000514B9A699204FCD51A6842F480721A6049
:103D50004C4B1A6F12F4407F04D04FF480321A6734
:103D600000221A671A6842F001021A60454B1A686D
:103D70005007FCD500221A611A6912F03802FBD1F3
:103D8000012119604FF0804159605A67414ADA6257
:103D9000414A1A611A6842F480321A60394B1A6833
:103DA0009103FCD51A6842F480521A601A68920492
:103DB000FCD53A4A3A499A6200225A631963394952
:103DC000DA6399635A64384A1A64384ADA621A68BC
:103DD00042F0A8521A602B4B1A6802F02852B2F136
:103DE000285FF9D148229A614FF48862DA61402253
:103DF0001A622F4ADA644FF080521A652D4A5A65CA
:103E00002D4A9A6532232D4A1360136803F00F037D
:103E1000022BFAD11B4B1A6942F003021A611A698C
:103E200002F03802182AFAD1D3F8DC2042F000520E
:103E3000C3F8DC20D3F8042142F00052C3F8042177
:103E4000D3F80421D3F8DC2042F08042C3F8DC2010
:103E5000D3F8042142F08042C3F80421D3F80421AE
:103E6000D3F8DC2042F00042C3F8DC20D3F8042170
:103E700042F00042C3F80421D3F80431704700BF78
:103E800000800051004402580048025800C000F071
:103E9000020000010000FF0100889008222040007D
:103EA000630209012C02040047040508FD0BFF0111
:103EB000200000200010E00000010100002000525E
:103EC0004FF0B04208B5D2F8883003F00103C2F8D1
:103ED000883023B1044A13680BB150689847BDE895
:103EE0000840FEF7E1BD00BF544F00204FF0B04244
:103EF00008B5D2F8883003F00203C2F8883023B145
:103F0000044A93680BB1D0689847BDE80840FEF7B3
:103F1000CBBD00BF544F00204FF0B04208B5D2F8DF
:103F2000883003F00403C2F8883023B1044A1369CF
:103F30000BB150699847BDE80840FEF7B5BD00BF1A
:103F4000544F00204FF0B04208B5D2F8883003F04B
:103F50000803C2F8883023B1044A93690BB1D069D1
:103F60009847BDE80840FEF79FBD00BF544F0020B2
:103F70004FF0B04208B5D2F8883003F01003C2F811
:103F8000883023B1044A136A0BB1506A9847BDE8E0
:103F90000840FEF789BD00BF544F00204FF0B043EA
:103FA00010B5D3F8884004F47872C3F88820A306CB
:103FB00004D5124A936A0BB1D06A9847600604D5BB
:103FC0000E4A136B0BB1506B9847210604D50B4A70
:103FD000936B0BB1D06B9847E20504D5074A136C7D
:103FE0000BB1506C9847A30504D5044A936C0BB1F0
:103FF000D06C9847BDE81040FEF756BD544F0020E6
:104000004FF0B04310B5D3F8884004F47C42C3F8B5
:104010008820620504D5164A136D0BB1506D984780
:10402000230504D5124A936D0BB1D06D9847E00477
:1040300004D50F4A136E0BB1506E9847A10404D5F6
:104040000B4A936E0BB1D06E9847620404D5084AB0
:10405000136F0BB1506F9847230404D5044A936F34
:104060000BB1D06F9847BDE81040FEF71DBD00BFF3
:10407000544F002008B50348FDF708F9BDE8084093
:10408000FEF712BDCC23002008B50348FDF7FEF86B
:10409000BDE80840FEF708BD3824002008B50348F5
:1040A000FDF7F4F8BDE80840FEF7FEBCA4240020AC
:1040B00008B5FFF797FDBDE80840FEF7F5BC000026
:1040C000062108B50846FFF7A7FA06210720FFF7E3
:1040D000A3FA06210820FFF79FFA06210920FFF71F
:1040E0009BFA06210A20FFF797FA06211720FFF70F
:1040F00093FA06212820FFF78FFA09217A20FFF78B
:104100008BFA07213220FFF787FA0C212720FFF7CF
:1041100083FA0C213520FFF77FFA0C215220BDE8ED
:104120000840FFF779BA000008B5FFF771FD00F00D
:104130000DF8FDF7BDFAFDF795FCFDF767FBFFF7FE
:1041400025FDBDE80840FFF747BC00000023054AF5
:1041500019460133102BC2E9001102F10802F8D10F
:10416000704700BF544F002010B5013902449042FF
:1041700001D1002005E0037811F8014FA34201D0DE
:10418000181B10BD0130F2E7034611F8012B03F8AC
:10419000012B002AF9D1704753544D333248373F31
:1041A0003F3F0053544D3332483734332F37353384
:1041B00000000000C8320020A42400203824002081
:1041C000CC2300200096000000000000000000004A
:1041D00000000000000000000000000000000000DF
:1041E0007916000865160008A11600088D1600084B
:1041F0009916000885160008711600085D1600085B
:10420000AD160008000000008917000875170008A7
:10421000B11700089D170008A91700089517000896
:10422000811700086D170008BD1700080000000086
:1042300001000000000000006D61696E00000000D8
:1042400069646C65000000004042000850310020A5
:10425000C832002001000000012100080000000019
:10426000486F6C7962726F0025424F415244252D90
:10427000424C002553455249414C250002000000A4
:1042800000000000A9190008191A000840004000A9
:10429000704B0020804B0020020000000000000056
:1042A0000300000000000000611A00080000000088
:1042B00010000000904B00200000000001000000F2
:1042C00000000000044E002001010200F12400085B
:1042D000012400089D2400088124000843000000F8
:1042E000E442000809024300020100C03209040050
:1042F0000001020201000524001001052401000153
:10430000042402020524060001070582030800FFB9
:1043100009040100020A0000000705010240000034
:104320000705810240000000120000003043000831
:10433000120110010200004062315300000201022C
:10434000030100000403090425424F4152442500A3
:104350005069786861776B364300303132333435D9
:1043600036373839414243444546000000000000DA
:10437000B51B00086D1E0008191F00084000400012
:104380003C4F00203C4F0020010000004C4F00201B
:104390008000000040010000080000000001000053
:1043A00000040000080000000000802A0002000055
:1043B000AAAAAAAA00000024FFFF00000000000033
:1043C00000A00A000000000000000000AAAAAAAA9B
:1043D00000000000FFFF00000000000000000000DF
:1043E0000000105600000000AAAAAAAA000000556A
:1043F000FFFF0000000000000000080020015A003C
:10440000000C0000AAAAAAAA10010500FFFF0000E4
:10441000000800007700000010800200000000008B
:10442000AAAAAAAA00400100FFFF00000000007035
:10443000070000000000000000000000AAAAAAAACD
:1044400000000000FFFF000000000000000000006E
:104450000000000000000000AAAAAAAA00000000B4
:10446000FFFF00000000000000000000000000004E
:1044700000000000AAAAAAAA00000000FFFF000096
:10448000000000000000000000000000000000002C
:10449000AAAAAAAA00000000FFFF00000000000076
:1044A000000000000000000000000000AAAAAAAA64
:1044B00000000000FFFF00000000000000000000FE
:1044C0000000000000000000AAAAAAAA0000000044
:1044D000FFFF0000000000000000000000000000DE
:1044E000380000000000000000001E000000000076
:1044F000FF00000000000000984100083F0000009D
:1045000050040000A34100083F0000000096000096
:1045100000000800960000000008000004000000F1
:1045200044430008000000000000000000000000FC
:10453000000000000000000000000000FFFFFFFF7F
:10454000FFFFFFFFFFFFFFFFFFFFFFFFFFFFFFFF7B
:10455000FFFFFFFFFFFFFFFFFFFFFFFFFFFFFFFF6B
:10456000FFFFFFFFFFFFFFFFFFFFFFFFFFFFFFFF5B
:10457000FFFFFFFFFFFFFFFFFFFFFFFFFFFFFFFF4B
:020000040801F1
:020000040802F0
:1000000000060024D90D0208518C0F087103020864
:10001000CD8B0F08C58B0F08C98B0F08DB0D0208AD
:10002000DB0D0208DB0D0208DB0D020811CD1508FF
:10003000DB0D0208DB0D0208DB0D0208DB0D0208F8
:10004000DB0D0208DB0D0208DB0D0208DB0D0208E8
:10005000DB0D0208DB0D0208E952160815531608DD
:10006000415316086D5316089953160839DC1508C4
:1000700061DC15088DDC1508B9DC1508E5DC150810
:100080000DDD150839DD150821D815081D7A0F0872
:10009000057B0F088D7A0F08757B0F08C55316086E
:1000A000DB0D02083D551608DB0D020851551608F8
:1000B00065551608755516088955160869E5150819
:1000C000DDE5150851E61508C5E6150869F41508BB
:1000D0007DF41508B1541608C5541608D9541608ED
:1000E00029541608DB0D0208DB0D0208DB0D02089F
:1000F000DB0D0208DB0D0208DB0D020865DD1508CB
:10010000DB0D0208DB0D02089D551608DB0D020809
:10011000DB0D0208ED541608DB0D0208DB0D0208AA
:1001200091DD1508B9DD1508E5DD150811DE1508A6
:100130003DDE1508DB0D0208DB0D0208DB0D0208B1
:10014000DB0D0208DB0D0208DB0D0208DB0D0208E7
:1001500065DE150891DE1508BDDE15080155160887
:10016000DB0D0208DB0D0208DB0D0208DB0D0208C7
:10017000DB0D0208354F1608DB0D0208DB0D020807
:10018000DB0D0208DB0D0208155516082955160867
:10019000DB0D0208DB0D0208DB0D0208DB0D020897
:1001A000DB0D0208DB0D0208DB0D0208DB0D020887
:1001B000DB0D0208DB0D0208DB0D020839E715082C
:1001C000ADE71508DB0D0208DB0D0208DB0D0208A8
:1001D000DB0D0208214F1608DB0D0208DB0D0208BB
:1001E000DB0D0208DB0D0208DB0D0208DB0D020847
:1001F000DB0D0208DB0D0208DB0D0208DB0D020837
:10020000DB0D0208DB0D0208DB0D0208DB0D020826
:10021000DB0D0208DB0D0208DB0D0208DB0D020816
:10022000DB0D0208DB0D0208DB0D0208DB0D020806
:100230009D541608DB0D0208DB0D020841D8150895
:10024000DB0D0208E9D9150811DA15083DDA1508A1
:1002500069DA150895DA1508C1DA1508EDDA150816
:1002600019DB1508DB0D0208DB0D0208DB0D0208A7
:10027000DB0D0208DB0D0208DB0D0208DB0D0208B6
:10028000DB0D0208DB0D0208DB0D0208DB0D0208A6
:10029000DB0D0208DB0D0208DB0D0208DB0D020896
:1002A000DB0D0208DB0D0208DB0D0208DB0D020886
:1002B000DB0D0208DB0D0208DB0D0208DB0D020876
:1002C000DB0D0208DB0D0208DB0D0208DB0D020866
:1002D000DB0D0208DB0D0208DB0D0208DB0D020856
:1002E0001D5A0208918B030805E4030831710408C4
:1002F000B5E905083D6108082D680808B901090835
:100300000D7E0908A5860908318A090891140A0892
:1003100075410A08A9500A0895F10A08011B0C0842
:1003200081C00C08FDCF0C08F17E0F0831840F0846
:1003300079A30F08A1401108E1921108E1E8110822
:10034000553B120889C61308390714087D24140880
:1003500081681408058B14085DBB14087DC8140857
:1003600019021508350C15080000000000000000F7
:10037000EFF30383EFF30982EFF30881DFF814D082
:100380002DE9FE4F684600F0FDFFBDE8FE4F8D46AB
:1003900070470000542E0024F1EE101AA0EC200A41
:1003A00001607047A0EC108A704700BF81F00041E7
:1003B00002E000BF83F0004330B54FEA41044FEA4A
:1003C000430594EA050F08BF90EA020F1FBF54EAE5
:1003D000000C55EA020C7FEA645C7FEA655C00F081
:1003E000E2804FEA5454D4EB5555B8BF6D420CDD52
:1003F0002C4480EA020281EA030382EA000083EAD5
:10040000010180EA020281EA0303362D88BF30BD74
:1004100011F0004F4FEA01314FF4801C4CEA1131CA
:1004200002D0404261EB410113F0004F4FEA033329
:100430004CEA133302D0524263EB430394EA050FB4
:1004400000F0A780A4F10104D5F1200E0DDB02FA23
:100450000EFC22FA05F2801841F1000103FA0EF2B7
:10046000801843FA05F359410EE0A5F120050EF17D
:10047000200E012A03FA0EFC28BF4CF0020C43FAAE
:1004800005F3C01851EBE37101F0004507D54FF0BB
:10049000000EDCF1000C7EEB00006EEB0101B1F50B
:1004A000801F1BD3B1F5001F0CD349085FEA300051
:1004B0004FEA3C0C04F101044FEA445212F5800F5C
:1004C00080F09A80BCF1004F08BF5FEA500C50F1F9
:1004D000000041EB045141EA050130BD5FEA4C0CDC
:1004E000404141EB0101013C28BFB1F5801FE9D239
:1004F00091F0000F04BF01460020B1FA81F308BF5C
:100500002033A3F10B03B3F120020CDA0C3208DD27
:1005100002F1140CC2F10C0201FA0CF021FA02F102
:100520000CE002F11402D8BFC2F1200C01FA02F172
:1005300020FA0CFCDCBF41EA0C019040E41AA2BF97
:1005400001EB0451294330BD6FEA04041F3C1CDA5F
:100550000C340EDC04F11404C4F1200220FA04F07F
:1005600001FA02F340EA030021FA04F345EA030129
:1005700030BDC4F10C04C4F1200220FA02F001FAEB
:1005800004F340EA0300294630BD21FA04F029466D
:1005900030BD94F0000F83F4801306BF81F4801106
:1005A0000134013D4EE77FEA645C18BF7FEA655C79
:1005B00029D094EA050F08BF90EA020F05D054EA4B
:1005C000000C04BF1946104630BD91EA030F1EBF50
:1005D0000021002030BD5FEA545C05D14000494154
:1005E00028BF41F0004130BD14F580043CBF01F547
:1005F000801130BD01F0004545F0FE4141F470012D
:100600004FF0000030BD7FEA645C1ABF1946104607
:100610007FEA655C1CBF0B46024650EA013406BF08
:1006200052EA033591EA030F41F4002130BD00BFC7
:1006300090F0000F04BF0021704730B54FF4806484
:1006400004F132044FF000054FF0000150E700BF05
:1006500090F0000F04BF0021704730B54FF4806464
:1006600004F1320410F0004548BF40424FF0000151
:100670003EE700BF42004FEAE2014FEA31014FEA94
:1006800002701FBF12F07F4393F07F4F81F06051E3
:10069000704732F07F4208BF704793F07F4F04BF2E
:1006A00041F40021704730B54FF4607401F000450B
:1006B00021F000411CE700BF50EA010208BF70476B
:1006C00030B54FF000050AE050EA010208BF70475C
:1006D00030B511F0004502D5404261EB41014FF4C5
:1006E000806404F132045FEA915C3FF4D8AE4FF0CD
:1006F00003025FEADC0C18BF03325FEADC0C18BFB0
:10070000033202EBDC02C2F1200300FA03FC20FA00
:1007100002F001FA03FE40EA0E0021FA02F114444D
:10072000BDE600BF80F0004002E000BF81F0004164
:1007300042001FBF5FEA410392EA030F7FEA226C87
:100740007FEA236C6AD04FEA1262D2EB1363C1BF17
:10075000D218414048404140B8BF5B42192B88BF86
:10076000704710F0004F40F4000020F07F4018BFA9
:10077000404211F0004F41F4000121F07F4118BFC9
:10078000494292EA030F3FD0A2F1010241FA03FC71
:1007900010EB0C00C3F1200301FA03F100F0004359
:1007A00002D5494260EB4000B0F5000F13D3B0F121
:1007B000807F06D340084FEA310102F10102FE2A90
:1007C00051D2B1F1004F40EBC25008BF20F0010000
:1007D00040EA03007047490040EB0000013A28BF9F
:1007E000B0F5000FEDD2B0FA80FCACF1080CB2EB22
:1007F0000C0200FA0CF0AABF00EBC25052421843A0
:10080000BCBFD0401843704792F0000F81F4000144
:1008100006BF80F400000132013BB5E74FEA410317
:100820007FEA226C18BF7FEA236C21D092EA030F83
:1008300004D092F0000F08BF0846704790EA010FFD
:100840001CBF0020704712F07F4F04D1400028BF2A
:1008500040F00040704712F100723CBF00F500000C
:10086000704700F0004343F0FE4040F40000704742
:100870007FEA226216BF08467FEA236301464202EE
:1008800006BF5FEA412390EA010F40F48000704701
:100890004FF0000304E000BF10F0004348BF4042A7
:1008A0005FEA000C08BF704743F0964301464FF0E3
:1008B00000001CE050EA010208BF70474FF000033F
:1008C0000AE000BF50EA010208BF704711F0004380
:1008D00002D5404261EB41015FEA010C02BF844650
:1008E0000146002043F0B64308BFA3F18053A3F5AF
:1008F0000003BCFA8CF2083AA3EBC25310DB01FAF6
:1009000002FC634400FA02FCC2F12002BCF1004F79
:1009100020FA02F243EB020008BF20F0010070470A
:1009200002F1200201FA02FCC2F1200250EA4C005E
:1009300021FA02F243EB020008BF20EADC707047A4
:100940007BB972B90029BEBF00204FF0004106E01C
:1009500008BF00281CBF6FF000414FF0FF3000F0CF
:1009600039BAADF1080C6DE904CE002909DB002B82
:100970001ADB00F0C7F8DDF804E0DDE9022304B07B
:100980007047404261EB4101002B1BDB00F0BAF8DD
:10099000DDF804E0DDE9022304B0404261EB4101EF
:1009A000524263EB43037047524263EB430300F050
:1009B000A9F8DDF804E0DDE9022304B0404261EB70
:1009C00041017047524263EB430300F09BF8DDF8AE
:1009D00004E0DDE9022304B0524263EB43037047B5
:1009E00053B94AB9002908BF00281CBF4FF0FF3196
:1009F0004FF0FF3000F0EEB9ADF1080C6DE904CE18
:100A000000F080F8DDF804E0DDE9022304B070476F
:100A100030B1012390FAA0F0B0FA80F0184470478A
:100A200008460029FBD02123F4E700BF430803F068
:100A30005533C01A830803F0333300F033301844C1
:100A400000EB101000F00F3000EB002000EB004036
:100A5000000E704708B502460B4643EC172BB5EE67
:100A6000C07BF1EE10FA03D4BDE8084000F02AB8CC
:100A7000B1EE477B51EC170B00F024F8404261EBDC
:100A8000410108BD9FED0B6B07EE900A9FED0B5BDC
:100A9000B7EEE77A27EE066BBCEEC66BB8EE464BB8
:100AA000A4EE457BFCEEC77B16EE101A17EE900AFB
:100AB000704700BF000000000000F03D0000000093
:100AC0000000F0419FED0B6B41EC170B9FED0B5BB2
:100AD00027EE066BBCEEC66BB8EE464BA4EE457B2C
:100AE000FCEEC77B16EE101A17EE900A704700BF97
:100AF000AFF30080000000000000F03D00000000A7
:100B00000000F0412DE9F047089D04468E46002B79
:100B10004DD18A42944669D9B2FA82F252B101FAB1
:100B200002F3C2F1200120FA01F10CFA02FC41EAC1
:100B3000030E94404FEA1C48210CBEFBF8F61FFA46
:100B40008CF708FB16E341EA034306FB07F19942E1
:100B50000AD91CEB030306F1FF3080F01F81994294
:100B600040F21C81023E63445B1AA4B2B3FBF8F06E
:100B700008FB103344EA034400FB07F7A7420AD9F5
:100B80001CEB040400F1FF3380F00A81A74240F21D
:100B900007816444023840EA0640E41B00261DB188
:100BA000D4400023C5E900433146BDE8F0878B42BD
:100BB00009D9002D00F0EF800026C5E9000130467C
:100BC0003146BDE8F087B3FA83F6002E4AD18B4256
:100BD00002D3824200F2F980841A61EB0303012000
:100BE0009E46002DE0D0C5E9004EDDE702B9FFDEEC
:100BF000B2FA82F2002A40F09280A1EB0C014FEA97
:100C00001C471FFA8CFE0126200CB1FBF7F307FBF3
:100C1000131140EA01410EFB03F0884208D91CEB96
:100C2000010103F1FF3802D2884200F2CB80434633
:100C3000091AA4B2B1FBF7F007FB101144EA014412
:100C40000EFB00FEA64508D91CEB040400F1FF31A1
:100C500002D2A64500F2BB800846A4EB0E0440EA8F
:100C600003409CE7C6F12007B34022FA07FC4CEA98
:100C7000030C20FA07F401FA06F31C43F9404FEA8B
:100C80001C4900FA06F3B1FBF9F8200C1FFA8CFEA0
:100C900009FB181140EA014108FB0EF0884202FAF4
:100CA00006F20BD91CEB010108F1FF3A80F08880B5
:100CB000884240F28580A8F102086144091AA4B272
:100CC000B1FBF9F009FB101144EA014100FB0EFEF3
:100CD0008E4508D91CEB010100F1FF346CD28E4522
:100CE0006AD90238614440EA0840A0FB0294A1EBB3
:100CF0000E01A142C846A64656D353D05DB1B3EB10
:100D0000080261EB0E0101FA07F722FA06F3F1403F
:100D10001F43C5E9007100263146BDE8F087C2F1E6
:100D20002003D8400CFA02FC21FA03F3914001435E
:100D30004FEA1C471FFA8CFEB3FBF7F007FB103697
:100D40000B0C43EA064300FB0EF69E4204FA02F443
:100D500008D91CEB030300F1FF382FD29E422DD996
:100D6000023863449B1B89B2B3FBF7F607FB1633CB
:100D700041EA034106FB0EF38B4208D91CEB01014B
:100D800006F1FF3816D28B4214D9023E6144C91ACB
:100D900046EA004638E72E46284605E70646E3E6DB
:100DA0001846F8E64B45A9D2B9EB020864EB0C0EE5
:100DB0000138A3E74646EAE7204694E74046D1E7F4
:100DC000D0467BE7023B614432E7304609E76444A2
:100DD000023842E7704700BF02E000F000F8FEE78B
:100DE00072B6374880F30888364880F30988364859
:100DF0003649086040F20000CCF200004EF6347133
:100E0000CEF200010860BFF34F8FBFF36F8F40F247
:100E10000000C0F2F0004EF68851CEF200010860EA
:100E2000BFF34F8FBFF36F8F4FF00000E1EE100A5A
:100E30004EF63C71CEF200010860062080F3148863
:100E4000BFF36F8F43F156FA41F17AFF4FF05530FF
:100E50001F491B4A91423CBF41F8040BFAE71D4968
:100E6000184A91423CBF41F8040BFAE71A491B4A61
:100E70001B4B9A423EBF51F8040B42F8040BF8E7B3
:100E800000201849184A91423CBF41F8040BFAE788
:100E900043F172FA42F194F8144C154DAC4203DA66
:100EA00054F8041B8847F9E704F0A8FD114C124DD3
:100EB000AC4203DA54F8041B8847F9E743F15ABA05
:100EC00000060024002200240000020808ED00E0D3
:100ED000000000240006002470531B080022002498
:100EE000602C0024602C0024DC460224E00202086E
:100EF0006803020868030208680302082DE9F04F3E
:100F00002DED108AC1F80CD0D0F80CD0BDEC108AB1
:100F1000BDE8F08F002383F311882846A047002006
:100F200041F13CFCFEE741F13BFA00DFFEE7000047
:100F300070B54FF0FF0C4CF4E06C1CEA11541DBF6F
:100F40001CEA135594EA0C0F95EA0C0F00F0DEF83A
:100F50002C4481EA030621EA4C5123EA4C5350EA1F
:100F6000013518BF52EA033541F4801143F4801370
:100F700038D0A0FB02CE4FF00005E1FB02E506F001
:100F80000042E0FB03E54FF00006E1FB03569CF056
:100F9000000F18BF4EF0010EA4F1FF04B6F5007F5C
:100FA00064F5407404D25FEA4E0E6D4146EB0606CE
:100FB00042EAC62141EA55514FEAC52040EA5E5057
:100FC0004FEACE2EB4F1FD0C88BFBCF5E06F1ED801
:100FD000BEF1004F08BF5FEA500E50F1000041EB38
:100FE000045170BD06F0004646EA010140EA0200E5
:100FF00081EA0301B4EB5C04C2BFD4EB0C0541EA07
:10100000045170BD41F480114FF0000E013C00F31B
:10101000AB8014F1360FDEBF002001F0004170BD3F
:10102000C4F10004203C35DA0C341BDC04F1140458
:10103000C4F1200500FA05F320FA04F001FA05F2E4
:1010400040EA020001F0004221F0004110EBD370B1
:1010500021FA04F642EB06015EEA430E08BF20EADD
:10106000D37070BDC4F10C04C4F1200500FA04F380
:1010700020FA05F001FA04F240EA020001F0004112
:1010800010EBD37041F100015EEA430E08BF20EA85
:10109000D37070BDC4F1200500FA05F24EEA020ECD
:1010A00020FA04F301FA05F243EA020321FA04F0FC
:1010B00001F0004121FA04F220EA020000EBD370B3
:1010C0005EEA430E08BF20EAD37070BD94F0000FB3
:1010D0000FD101F00046400041EB010111F4801FE7
:1010E00008BF013CF7D041EA060195F0000F18BF98
:1010F000704703F00046520043EB030313F4801FD4
:1011000008BF013DF7D043EA0603704794EA0C0F8D
:101110000CEA135518BF95EA0C0F0CD050EA4106A3
:1011200018BF52EA4306D1D181EA030101F0004120
:101130004FF0000070BD50EA410606BF1046194648
:1011400052EA430619D094EA0C0F02D150EA013654
:1011500013D195EA0C0F05D152EA03361CBF104695
:1011600019460AD181EA030101F0004141F0FE4134
:1011700041F470014FF0000070BD41F0FE4141F4B8
:10118000780170BD4FEA410212F5001215D211D557
:101190006FF47873B3EB625212D94FEAC12343F074
:1011A000004343EA505311F0004F23FA02F018BFF6
:1011B000404270474FF00000704750EA013005D1BF
:1011C00011F0004008BF6FF0004070474FF0000082
:1011D000704700BF4FEA4102B2F1E04324BFB3F5CC
:1011E000001CDCF1FE5C0DD901F0004C4FEAC0029E
:1011F0004CEA5070B2F1004F40EB830008BF20F082
:101200000100704711F0804F21D113F13872BCBF3B
:1012100001F00040704741F480114FEA5252C2F190
:101220001802C2F1200C10FA0CF320FA02F018BFD9
:1012300040F001004FEAC1234FEAD32303FA0CFC2C
:1012400040EA0C0023FA02F34FEA4303CCE77FEABB
:10125000625307D150EA01331EBF4FF0FE4040F405
:101260004000704701F0004040F0FE4040F40000B4
:10127000704700BF01F0FF01102A2BDB10F0070FB1
:1012800008D010F8013B013A8B422DD010F0070F27
:1012900042B3F6D1F0B441EA012141EA014122F022
:1012A00007047FF000070023F0E80256083C85EAB7
:1012B000010586EA010685FA47F5A3FA87F586FA5D
:1012C00047F6A5FA87F68EB9EED1F0BC01F0FF0122
:1012D00002F0070232B110F8013B013A83EA010340
:1012E00013B1F8D10020704701387047002D06BFB8
:1012F00035460338073815F0010F07D1013015F4D2
:10130000807F02BF013015F4C03F0130F0BC0138CE
:10131000704700BFEC46A0E8F05F4FF00000704758
:10132000B0E8F05FE546080008BF0120704700BF45
:1013300010F8012B11F8013B012A28BF9A42F7D07F
:10134000D01A7047034613F8012B002AFBD1181A54
:1013500001387047A8B110B504460AE000F096FACB
:1013600014F8041C54E903031B1AB3FBF1F200F058
:101370008DFA204654F80C3B082201210133EDD1AF
:1013800010BD70472DE9F04F0023A7B00293C36A48
:10139000009013F0040FD0E9002118BF0A46D906C7
:1013A0004FF0E021D3694CBF02F1200002F1680048
:1013B0000192DB0903F0040303430393D1F8883D52
:1013C00003F4A003B3F5A00F01D1012302939369A5
:1013D0004FF004094F4D4FF001081B884E4C03F4A9
:1013E0007F43A3F53E43B3FA83F35B09049329E0FB
:1013F00000F040F9FFF7AEFF4FF0E023D3F8003DD7
:1014000003F47023B3F5402F0ED0444A4FF0FF335E
:1014100005A88DF81C90059214328DF8288006924C
:10142000CDE90833FFF796FF2B68A34206D03C4B6B
:101430000422012105A8059300F028FA00F070FBB2
:1014400000285ED103A82C6000F00CFC04220121CE
:10145000344800F01BFA0422012102A800F016FA19
:1014600010220121019800F011FA00982022012198
:101470000C3000F00BFA019804220121103000F02A
:1014800005FA0422012103A800F000FA01980C22B9
:101490000121143000F0FAF90C220121009800F02B
:1014A000F5F9029BDA07A3D5009BDB6ADB0622D4A1
:1014B00015A80DF1140AFEF775FFDDF804E0D44617
:1014C0000EF120060EF1600B3068103656F80C1C39
:1014D000674656F8082C0CF1100C56F8043C5E4593
:1014E0000FC7F1D1DEF860302593842250460121E8
:1014F00000F0CCF97CE70DF1140A5046FEF74CFFE2
:10150000F3E7049B1BB1019A93690233936127B0FF
:10151000BDE8F08F602C0024ED55CEAC28ED00E046
:10152000ACCE55ED44E6160838B535206D253EF1B4
:10153000B7FF144B144A4FF0FF34D3F890100D202E
:1015400041F48011C3F89010D3F8901021F4801169
:10155000C3F89010D3F89010D3F8E81041F480113C
:10156000C3F8E810D3F8101141F48011C3F810113A
:101570000121D3F81031054BD56014621060197049
:1015800038BD00BF00440258005000408C2E00249B
:10159000002953D02DE9F84F074689460026284DEB
:1015A000DFF8A480274C17F801AB2B784FEA1A120A
:1015B00018F802B0002B3CD0C4F828B0E3695806F4
:1015C00004D442F15DFEE3695906FAD50AF00F0A28
:1015D0002B7818F80AA04BB3C4F828A0E3695A0680
:1015E00004D442F14DFEE3695B06FAD50136B145FC
:1015F00022D03107D7D12B784FF00D0BDFF84CA05C
:101600008BB1C4F828B0E3695A0604D442F138FE1D
:10161000E3695B06FAD51AF801BFBBF1000FC2D02F
:101620002B78002BEDD1FFF77FFFEAE7FFF77CFF78
:10163000D2E7FFF779FFBFE7BDE8F88F704700BF3B
:101640008C2E002400500040CCE6160820FF17081E
:10165000014B1868704700BFFCFF1F08014B024890
:10166000C01A7047E05D1B08000020080048704762
:10167000E05D1B08774943F69822774B09682DE90E
:10168000F04F0A441B7883B0744F02EB030940F11A
:1016900085FD734B0446002800F0C8800225FF1A20
:1016A000DFF8E0810126DFF8CCB130E01846019187
:1016B00042F1D6F90199002836D1206AAA460AF1EA
:1016C00001030AEB4A0E04F13C058944DBB20144F4
:1016D0000BEB8E0CB94503EB43034BF82E40CCF8D3
:1016E00004500AF102058CF808600BEB830CEDB294
:1016F0004BF823008CF80860CCF8041023D2204665
:1017000040F15CFD0446002835D04E2D33D8206AC8
:10171000404505D0211AE369002BC7D1AA46CEE780
:10172000504BA3EB0801F6E705EB450C01350BEB3D
:101730008C005FFA85FA0672E3694BF82C300D33A2
:101740004360206ABBE74F2D63D94FF0FF3301227E
:10175000CBF8B4338BF8BC23CBF8B833424B1B78AF
:101760002BB1424A424B12681B68CBE90023414827
:1017700003B0BDE8F08FB7EB0900E4D44E2DE2D8FA
:101780000AF1030A3C4EDFF800C15FFA8AFAA6EBC1
:101790000C03BAF14E0F514694BF0024012483423A
:1017A0002BDC05EB450503EB090201200BEB850360
:1017B0004BF825C05E601872BA1A12D48CB92F4843
:1017C00001EB41052E4BC41A944224DD1A440AF160
:1017D00001014BF825300BEB8503C9B25A60012299
:1017E0001A7201EB41054FF0FF3201210BEB85032B
:1017F0004BF8252019725A60B0E705EB4505012228
:1018000060440BEB85034BF825C01A723A465860CA
:10181000D2E72946E5E70AF1010101224BF825301C
:101820000BEB8503C9B258601A72DAE7FF1AB7EBFF
:1018300009000BD4104E4FF0030ADFF84CC002250C
:10184000DFF830B05146A6EB0C03A8E70221DFF821
:1018500024B0C6E77C2E0024542E0024000020086B
:10186000E05D1B080022002400220024802E0024BA
:10187000782E002404220024DC46022400000824E0
:10188000E046022400060024602C00249A4B1B78BA
:101890002DE9F04F824685B00E4693462BB9974B03
:1018A0001B782BBB05B0BDE8F08F022900F0EE805D
:1018B000042900F0B580012900F0AE80904D2B780E
:1018C0000D27DFF858828F4C7BB1A762E3695A0677
:1018D00004D442F1D5FCE3695B06FAD518F8017F20
:1018E000002FDCD02B78002BEFD1FFF71DFEECE7AB
:1018F000854B4FF00009854A9B1A0093CB45D1D008
:10190000834F844C38682578031D009A2B449342FA
:1019100079D2202D51D0022E24D0042E0DD0012EAC
:10192000ECD12378DFF8F0815A1C22701AF80920D4
:1019300009F1010908F80320E0E7DFF8DC81002560
:10194000434620789AF80010421CE9400835D2B28C
:1019500008F80010202A227018D0202DF1D109F1AA
:101960000109CBE725789AF80030DFF8AC8108F858
:1019700005300135EDB2202D257030D06B1C09F1FA
:1019800001092370002308F80530B7E738685F497C
:1019900001920844194641F103FE39684FF00003F3
:1019A000019A203123705C4B39600021184648F1C0
:1019B00053F942F165FC584BCFE7544B2A46564940
:1019C000184441F1EDFD3B6800212A46203352487E
:1019D00021703B6048F140F942F152FC9BE74B4BD0
:1019E0002A4638684146184441F1DAFD3B68002137
:1019F0002A462033404621703B6048F12DF942F1E0
:101A00003FFC2578BAE7444A4FF0FF312023D161EB
:101A1000237005B0BDE8F08F1146FFF7B9FD4DE723
:101A2000002A3FF44BAF02460027354D0DF10C085C
:101A300052F8043B334C0092039301910137042187
:101A40004046FFF7A5FDBB451ED0009ABE0752F8E1
:101A5000043B00920393F1D12A780D26DFF8BC9065
:101A60007AB1A662E369580604D442F109FCE3693D
:101A70005906FAD519F8016F002EDFD02A78002A0E
:101A8000EFD1FFF751FDECE7019E18E7002A3FF484
:101A900015AF024600271A4D0DF10C0832F8023B33
:101AA000184C0092ADF80C300191013702214046EC
:101AB000FFF76EFDBB45E7D0009A790732F8023B8D
:101AC0000092ADF80C30F0D12A780D26DFF84C905A
:101AD0007AB1A662E3695A0604D442F1D1FBE36904
:101AE0005B06FAD519F8016F002EDED02A78002A9D
:101AF000EFD1FFF719FDECE7552E0024002200245A
:101B00008C2E00240050004000002008E05D1B08DF
:101B10007C2E0024542E0024582E002420FF170869
:101B2000F8B5324B1A782AB9314A1078F0B9012247
:101B30001A70F8BD2F4E0D252F4F304C3B7893B1C6
:101B4000A562E3695A0604D442F19AFBE3695B0695
:101B5000FAD516F8015F002DF0D1294B58680038EE
:101B600018BF0120F8BDFFF7DFFCE9E7254D264E41
:101B70002B68264C26481A1D3178241A0A44A242A2
:101B800006D239BB9C421CD8002041F1BFFDE4E7DE
:101B9000204A4FF0FF31D1612022327018442022B8
:101BA0001C4941F1FDFC2A6833780021194813448F
:101BB000202231702B6048F14FF842F161FB2B6815
:101BC000E0E7144920221448CB6141F1E9FC42F1DD
:101BD00057FBD9E703F120029442DFD81F29DDD853
:101BE0000C4AD36120223270D8E700BF552E002462
:101BF0000022002448E616088C2E002400500040E5
:101C0000842E00247C2E0024542E00240000200862
:101C1000E05D1B08582E0024E0FF1F080E4B1B78C8
:101C200010B5B3B1642100200C4A0D4CD3699B065A
:101C3000FCD5536ADBB28B424FF0640101D0002027
:101C4000F4E70130C0B20E2801D0015DEEE70020BC
:101C500010BDFFF769FCE5E78C2E00240050004022
:101C600058E616082DE9F04102680646EFF30581B3
:101C7000D9205369C9B2D6F0ABFF674B1B782BB99B
:101C8000664C2378002B37D1BDE8F081644B0D27DB
:101C9000DFF8B081634D644C96E8030083E80300ED
:101CA0002B7833B3A762E3695F0604D442F1E8FA04
:101CB000E3695806FAD518F8017F002FF0D1736850
:101CC0000BB32B784227DFF88081574C73B1A762A2
:101CD000E369590604D442F1D3FAE3695A06FAD506
:101CE00018F8017F1FB32B78002BF0D1FFF71CFCF5
:101CF000EDE7FFF719FCD5E73568002D47D1002344
:101D00002370BDE8F081DFF844814327464C2B78EF
:101D1000002B6AD0A762E3695B0604D442F1B0FAF3
:101D2000E3695F06FAD518F8017F002FEFD1DFF8DD
:101D3000208120273C4C2B78002B53D0A762E369ED
:101D4000580604D442F19CFAE3695906FAD518F80A
:101D5000017F002FEFD1FFF761FF2B78DFF8F480D0
:101D60000D27314C83B1A762E3695A0604D442F1CE
:101D700087FAE3695B06FAD518F8017F002F3FF474
:101D80007FAF2B78002BEED1FFF7CEFBEBE7284699
:101D900041F166FE0028B2D0284641F189FE00F2EA
:101DA0001450854231D3214BA5F214521A602846B3
:101DB00041F194FE05F5E053834220D81C4A13609C
:101DC00000231C481C4A03601C481D49801A0B70E4
:101DD00002D10DE083420BD252F8041B04330131CF
:101DE000F8D08CE7FFF7A0FBA8E7FFF79DFB91E792
:101DF00042F146FA0120BDE8F04141F187BC284696
:101E000041F16CFE0A4B1860DAE7284641F150FEBA
:101E1000064B1860CBE700BF552E0024002200249B
:101E2000842E00248C2E002400500040802E00249C
:101E3000782E00247C2E0024E05D1B080000200882
:101E4000542E002468E6160870E61608C4E6160844
:101E50007CE6160820FF1708002070470368002260
:101E60001B6818470F4B70B51C68E56A2B681E6825
:101E7000C6F0E4FE014628B1E06A0B4A0368DB695C
:101E800093420AD12846B04770F0D4FDE36ABDE81A
:101E9000704093F89C106FF089BC9847411E18BFA2
:101EA0000121EFE7982E0024591E020870B505465F
:101EB0008EB010480E46D2F0EDFA00212E220446D4
:101EC00002A8019147F1C8FEC2F096FC20B132226F
:101ED00001A9C2F033FC10B120460EB070BD04461B
:101EE00001AB2846044A3146C7F0F8FA20460EB046
:101EF00070BD00BFB88300241CE7160870B50C46FF
:101F000082B040210546C6F0A5FEE8B1184BD3E9E2
:101F1000D02140F21453B2F90A00984217DCB2F90A
:101F20000E0040F2A36290421BDDB1F90A00984214
:101F30001ADCB1F90E30934218DD2146284602B072
:101F4000BDE87040C7F03EB8012002B070BD094E38
:101F5000094B2846224640210096C6F083FE002009
:101F6000F3E7044E054BF4E7054EF1E7044EF9E7BD
:101F7000A09E0024E0E616082CE7160844E71608A1
:101F8000E8E616082DE9F041294F8EB005460E46C9
:101F9000D7F8F43D1A681846536A984728B9D7F815
:101FA000F40D03689B6A984728B331462846C7F06A
:101FB00033F9044618B920460EB0BDE8F0814FF061
:101FC00000080DF091FE04462E22414602A8CDF8ED
:101FD000048047F141FE2046322301AA01210DF081
:101FE00069F80446B0B197F80C3E4BB9114804F0BB
:101FF00045F80446A8B1012420460EB0BDE8F081A2
:10200000444628460C4A3146C7F068FA20460EB0CE
:10201000BDE8F08101AB094A31462846C7F05EFAB7
:10202000C9E7074A31462846C7F058FAC3E700BF58
:10203000A0AE0024A02E002468E716085CE716086E
:1020400078E716082DE9F043C57F8FB0002D4FD1FA
:102050003C4B04460E461B68986A03685B6B9847C6
:10206000002850D0A3683BB92368314620469B6BBB
:102070000FB0BDE8F0431847334F97F97C3E002B73
:1020800005DD07F27C50D1F04DF800284BD03146E9
:102090002046C8F083FB314680462046FFF706FF06
:1020A00000212E22814602A8019147F1D5FD32225E
:1020B00001A92648A0F0C2F80546E8B108EA0905DA
:1020C000EDB220212046C6F0C5FD50B107F254679D
:1020D000DFED1F7A97ED007AB4EEE77AF1EE10FAB1
:1020E00027DB1C4BD3F8F40D03689B69984798B124
:1020F00028460FB0BDE8F08301AB174A31462046B1
:10210000C7F0ECF9DDE72046144A3146C7F0E6F99E
:1021100028460FB0BDE8F0830546114A31462046F7
:10212000C7F0DCF9E4E70F4A31462046C7F0D6F99C
:10213000DEE70D4B3246202120460025C6F092FDF9
:10214000CFE700BF982E0024A08E0024609D0024BD
:1021500000000034A0AE0024CC201A0890E7160836
:1021600008E71608A8E71608F4E6160883680BB90E
:1021700001207047C6F0DCBE38B50546C8F03EFC0D
:10218000044630B90C4A2046137843F0010313701B
:1021900038BD01210948CFF09DFF094808F094FAA5
:1021A0000848D1F05FF82846FFF75CFE284606494C
:1021B000C8F088F9204638BD10CB0024B088002430
:1021C00068C800241C940024CCE7160838B50546DE
:1021D000C8F09CFC044680B1094A0A4BD2F8F42DA1
:1021E0009A4203D003F1380039F0FAFA2846FFF793
:1021F00039FE05492846C8F065F9204638BD00BFBC
:10220000A0AE0024F8C30024DCE7160830B51C4D4E
:102210000C462DED028BD5F8F40D85B0B0EE408A5A
:1022200003681B69984728B90025284605B0BDEC0E
:10223000028B30BDA5F63C40C6F000FD05460028E7
:10224000F2D00DF051FD21460BF06AFFB4EE488A42
:10225000F0EE400AF1EE10FA0FD6DFED0A7A9FEDAC
:102260000A0A28EE278A28EE000A084807F0A4FC8C
:10227000284605B0BDEC028B30BD9FED050AF4E7A2
:10228000A0AE0024E02E65420000C84280C30024B6
:1022900000000000014802F0FFBD00BFA02E002496
:1022A00001489DF08DBD00BF3C6D0024704700BF0C
:1022B000704700BF704700BF002070470020704784
:1022C0000120704700207047704700BF0020704712
:1022D000C8207047012070470120704708207047D0
:1022E00090F8D0308B4204D900EB8100D0F8D400B4
:1022F00070470020704700BF90F8D0308B4204D95F
:1023000000EB8100D0F8D40070470020704700BF78
:102310000020704708B5034BD3F8F40D03681B6821
:10232000984708BDA0AE0024044BD3ED007AFDEE23
:10233000E77A17EE903A18B2704700BFE0830024A6
:10234000014B93F834037047A06E0024034B93F9BC
:102350006803003818BF0120704700BFA06E00243A
:10236000014B93F936037047A06E0024054800F531
:10237000004300F51440D3F8F43D181A18BF0120AB
:10238000704700BFA02E0024104B10B5D3F8F44DB9
:1023900023682046DB68984798B123682046DB6BAA
:1023A0009847F2EE046A9FED0A7AC0EE267AF4EEC0
:1023B000C77AF1EE10FA05D5FCEEE77A17EE903AFF
:1023C00098B210BD4FF6FF7010BD00BFA0AE002444
:1023D00000FF7F47704700BF08B504480AF082F845
:1023E00000280CBF0A200B2008BD00BFA02E00242F
:1023F00038B5174DD5F8F40D0368DB699847D5F863
:10240000F43D00281A6818460CBF01244124D36803
:10241000984708B144F008040E4B93F94C2603F595
:102420005053002AD5F8F42D0CDD9A4207D044F021
:1024300040040948C6F002FC08B144F0800444F0AE
:10244000010038BD9A42F4D144F0010038BD00BF0C
:10245000A0AE0024A08E002464A200242DE9F04147
:10246000204E96F8683A2DED028B84B0A3B39FED11
:102470001E8A0024804606F5FD67F0EE488A254650
:102480002146384665F06AF980B1436835B1D3ED2D
:10249000007AF4EEE87AF1EE10FA07D5DA88012531
:1024A000D3ED008A07EE902AB8EE678A013496F8D9
:1024B000683AE1B28B42E4D875B10823532498F806
:1024C0001000AD210DEB0302CDED028A8DED038AE4
:1024D000CDE9003475F0DAFA04B0BDEC028BBDE84A
:1024E000F08100BFA03E00240000000030B504468B
:1024F00083B00D46064811460192D0F095FB019A33
:102500002946204603B0BDE830407CF087BF00BFBD
:10251000509300242DE9F0419FED130A84B0134F2E
:102520004FF000080D4606468DED030A1446009252
:102530004FF47A73CDF80480B1F90220D7F8401334
:102540007DF030FACDF804809DED030A4FF47A73E4
:10255000B5F904203046D7F8441300947DF022FAF0
:1025600004B0BDE8F08100BF0000FA44A09E002442
:102570000148D3F03DBC00BF20B8002408B576F078
:10258000C1FE034640F2CD10184308BD0D4B10B5F7
:10259000D3F8F44D82B023682046DB68984778B1C1
:1025A00023682046DB6A984732F060FBF6EE007A3B
:1025B00020EE270AFCEEC07ACDED017A9DF80400EA
:1025C00002B010BDA0AE002470B54FF444700D46AB
:1025D000164616F0E7FA044628B13246294677F047
:1025E000F9FC024B2360204670BD00BF30EA16089C
:1025F00010B5044616F0E2FA204610BD0B4B93F8D6
:10260000042E72B993F80C2E5AB9D3F8F40D03F5D1
:10261000A053984207D03833984214BF04200320B7
:102620007047052070470220704700BFA0AE00240D
:1026300008B54B69012B0BD0022B03D0BDE8084035
:1026400076F0C6BE0648D0F025FE30B1002008BDA9
:102650000348D0F011FE0028F8D1042008BD00BFC7
:102660001C940024124B10B5D3F8F43D82B00446FC
:102670001A681846D3689847A8B123682046D3F84B
:10268000B8309847B1EE047ADFED0A7A20EE070AF7
:10269000B4EEE70AF1EE10FA07D5FCEEC07ACDED04
:1026A000017A9DF8040002B010BDFF2002B010BDF9
:1026B000A0AE002400007F4300B50F4883B0D0F0E7
:1026C00031FD10B903B05DF804FB0C4BDFED0C7A63
:1026D00093ED000A20EE270A32F0C8FAF6EE007AEF
:1026E00020EE270AFCEEC07ACDED017A9DF80400B9
:1026F00003B05DF804FB00BF1C9400246494002424
:10270000E02E654200B5104883B0D0F00BFD98B1C3
:102710000E4BF1EE046A9FED0E7AD3ED007A67EE70
:10272000A67AF4EEC77AF1EE10FA08D5FCEEE77A55
:10273000CDED017A9DF8040003B05DF804FBFF20A5
:1027400003B05DF804FB00BF1C940024C094002477
:1027500000007F4330B595B0044603A815F074FA25
:102760001A4B03A9D3F8F40D03681B6C984750B3B8
:10277000257CD6F0A3FADDED047A9621059C002293
:10278000F8EEE77A9FED127A089400243323019142
:1027900067EE877A4FF6F8518DF84E40069C079009
:1027A00028460B920C920D920E920F92109211925B
:1027B000129207AAADF84C1057210093CDED0A7A7A
:1027C000099475F063F915B030BD00BFA0AE0024C8
:1027D0000AD7233C2DE9F041304C05462DED028B04
:1027E000D4F8F43D8AB01A681846D368984720B9DF
:1027F0000AB0BDEC028BBDE8F081D4F8F44D284856
:1028000095F81080CCF0CCFB236820469FED258AFC
:102810001B6B20EE088A9847BDEEC00A236820464D
:10282000DB6A10EE102A17B29847BDEEC00A236883
:10283000204610EE102ADB6B16B29847DFED1A7AAD
:10284000B4EEE70AF1EE10FA24D5FCEEC07A17EEEA
:10285000903A9DB2236820465B6B984700211A236B
:10286000B72203914046059106913E21ADF82070B4
:102870008DED070A8DED048AADF82260ADF8245085
:10288000CDE9003203AA75F001F90AB0BDEC028B64
:10289000BDE8F0814FF6FF75DCE700BFA0AE002475
:1028A00044840024E02E654200FF7F472DE9F04379
:1028B0005F4D8DB00446B5F84433D90700F1BE80B2
:1028C0009A0700F1FC805F0700F12C811E0700F1E0
:1028D0006681D80600F1A281990606D45A0636D43C
:1028E0001B066BD40DB0BDE8F083524A622013463C
:1028F00053F8141B0491196809230591116A8DF886
:10290000243021230190CDF82510D169009319239B
:10291000CDF829109168207C0691D1680791116942
:1029200052F8042C0891C221039203AA75F0AEF864
:10293000207C75F02BF80646207C76F057F800F1E5
:1029400021039E426ED3B5F844335A06C8D53A4A9D
:102950006220D2F81831D2F82C110493212305916A
:102960000A210093192301908DF82410D2F8381110
:10297000207CCDF82510D2F83411CDF82910D2F8EA
:1029800020110691D2F824110791D2F82811D2F81B
:1029900014210891C221039203AA75F077F8207CD4
:1029A00074F0F4FF0646207C76F020F800F1210355
:1029B0009E4237D3B5F844331B0693D51E49622295
:1029C0002125D1F844310493D1F858310192D1F83E
:1029D0006001D1F86421CDF829000095D1F84C01AF
:1029E00005930B230690D1F85001CDF8252003AABA
:1029F0000790D1F85401D1F840118DF824301923F3
:102A000008900391C221207C75F040F8207C74F07E
:102A1000BDFF0546207C75F0E9FF00F121039D42D2
:102A2000BFF460AF207C0DB0BDE8F04374F07EB819
:102A3000A06E002454880024A09E0024964ADFED56
:102A4000976A516902F1080392ED007A0591D16805
:102A500027EE267A1B68052207912121069362231F
:102A600000918F4901931923D1ED007A05F5B351F7
:102A7000007C096867EEA67A8DF8242003AA0891E5
:102A800088498DED047A0968CDED037ACDF82510DB
:102A900085490968CDF82910C22174F0F7FF207C20
:102AA00074F074FF0646207C75F0A0FF00F121034E
:102AB0009E42B7D3B5F844339A077FF504AF7B4AFB
:102AC0006220134653F8141B0491196804230591DE
:102AD000116A8DF8243021230190CDF82510D16999
:102AE00000931923CDF829109168207C0691D168B4
:102AF0000791116952F8042C0891C221039203AA8C
:102B000074F0C4FF207C74F041FF0646207C75F011
:102B10006DFF00F121039E4284D3B5F844335F0773
:102B20007FF5D4AE624902226220DFED5C6A0B467B
:102B300011ED017AD1ED007A14338DF824208A68E2
:102B400027EE267A1B6867EEA67A0190059321236B
:102B5000069203AA00931923C8688DED037A0790A3
:102B60000869CDED047A0890086AC969CDF8250096
:102B7000CDF82910C221207C74F088FF207C74F0ED
:102B800005FF0646207C75F031FF00F121039E42CF
:102B9000FFF448AFB5F844331E077FF59AAE002125
:102BA0004448BAF05FFCD0F8B410D0ED297A212760
:102BB000D0F8B8E04FF06208D0F8ACC0D0F8C4301C
:102BC000D0F8C020D0F8B060D0F8A000089107215C
:102BD0000390CDF8253019238DF82410C221CDF8AB
:102BE000292003AACDED047ACDF814E0CDF818C061
:102BF0000796CDE90078207C74F048FF207C74F0C3
:102C0000C5FE0646207C75F0F1FEC3199E42FFF416
:102C100009AFB5F84433D8067FF55EAE01212548EB
:102C2000BAF020FCD0F8B410D0F8A4E04FF021089E
:102C3000D0F8B8C04FF06209D0F8C430D0F8C02046
:102C4000D0F8B060D0F8AC70D0F8A000089108219E
:102C50000390CDF8253019238DF82410C221CDF82A
:102C6000292003AACDF810E0CDF814C007960697E6
:102C7000CDE90089207C74F009FF207C74F086FE89
:102C80000646207C75F0B2FE00EB08039E42FFF47E
:102C9000C9AEB5F844331FE6F0840024E02E654247
:102CA000EC840024108500240C85002478870024FF
:102CB000D88600249081002430B504462D482DED9F
:102CC000048B89B0D1F036FB00283ED09FED2A9AC4
:102CD000492080F0ABFE9FED298A20EE090A4A20A8
:102CE00060EE088A80F0A2FE20EE090A20EE088A33
:102CF000257CD5F0E3FF034620461C467DF086FA8E
:102D0000BDEEC88A0021FDEEE88A8DF81D00ADF801
:102D10000E10284618EE103AADF8121018EE902A50
:102D20008DF81C10ADF81030ED23ADF80C2002AA80
:102D3000CDE901341623CDE905112221009374F069
:102D4000A5FE09B0BDEC048B30BD1A209FED0B8AA7
:102D500080F06CFEDFED0A7A4620C0EE278A80F014
:102D600065FEDFED087A20EE270A68EE888A20EEFD
:102D7000088ABDE7B88300246F12833A00401C46DE
:102D800000A08C450AD7233C2DE9F047044692B0B9
:102D9000007C74F0FBFD0546207C75F027FE00F1F9
:102DA00026039D4211D34D4809F09CFB50B14C4B7A
:102DB000D3F800A0BAF1000F04D01921504664F0F6
:102DC00075FD40B912B0BDE8F087207C12B0BDE8B7
:102DD000F04773F0ABBE0CF087FF074604A814F071
:102DE00033FF04A938460CF015FF9AF88062002ED4
:102DF000E8D094F80F134FF000090131C846C9B26A
:102E0000B14217D284F80F13504609F1010964F05A
:102E1000A5FC054620B1836893F92130192B0DD00C
:102E20005FFA89F3B342CDD294F80F130131C9B2DE
:102E3000B142E7D3002184F80F83E5E765F030F96C
:102E40000028EDD02B68274A9B6A93423FD100238C
:102E50000393284665F01AF994F810800646D5F0D9
:102E60002DFF69680246DDED057AA6F104060968C2
:102E70004046F8EEE77A94F80F330F91B6FA86F6EB
:102E8000D7F804129FED187A76090C91D7F808123A
:102E900067EE877A08922F220D91D7F80C128DF8E1
:102EA000443026230E910699039C099107990192BB
:102EB00008AA0A9142F61E3100938DF84560CDEDC7
:102EC0000B7A109474F0E2FD12B0BDE8F08703A90C
:102ED000284698470028BCD1B9E700BFA02E00249F
:102EE000E4CB0024112302080AD7233CF0B500F5F7
:102EF000A0452DED048B95F8E062C7B096B304466B
:102F00000F467022002104F5104406A846F1A4FEE5
:102F1000012E94EDF88AB7EEC88A27D094EDF99A7D
:102F2000B7EEC99AD5F0CAFE4FF47A7395F8E0125D
:102F3000002203FB00F071248DF8101102A92392E6
:102F40008022229024A88DED028B8DED049B46F10A
:102F500039FE892322AA42F228313846CDE90034CD
:102F600074F094FD47B0BDEC048BF0BD9FED019B68
:102F7000D8E700BF00000000000000003C29F0B5C9
:102F8000064683B03FD00C460CD940291DD04D29B0
:102F900044D1262173F0DCFD054690B90025284672
:102FA00003B0F0BD1B2940D0242937D10C2173F088
:102FB000CFFD05460028F1D0317C2248D0F078F9C9
:102FC000EDE73046FFF7E0FEE9E7A3F03FF80746FC
:102FD000002834D02621304673F0BAFD054600287B
:102FE000DDD0002321460DF106023046ADF8063053
:102FF0007AF030F80028D2D0BDF806203846317C6F
:10300000A2F0E2FECBE7892173F0A2FD054600287D
:10301000C4D0317C0C48FFF769FFC0E72146304639
:1030200003B0BDE8F0407DF0C1BA162173F090FD09
:1030300005460028B2D03046FFF73EFEAFE7012537
:10304000ADE700BF1C940024A02E002470B50C46F0
:10305000272200212DED028BE57890B0954206A83D
:1030600028BF154646F1F8FD04F10C0106A82A46D2
:103070002D4D46F1A7FDD5F8F40D03681B6998475F
:1030800020B19DF83E4014F0400603D010B0BDECD6
:10309000028B70BDFFEE000A40F28F30B7EE001ACF
:1030A0009DED0E0A31F072FE3146B0EE408AD5F841
:1030B000F40D8DED0E0A03F009FF630768EE000AB8
:1030C0001FD5079B02A80899099A02930A9BCDED88
:1030D000010A03910492059335F06AFD9FED137A7E
:1030E00005F5A750DFED127A20EE070ADDED010AA3
:1030F00020EE270A10B0BDEC028BBDE8704006F050
:103100002BBDDDED0D7A05F5A7509FED087A9FEDFB
:10311000080A67EE877A27EE800A10B0BDEC028BB2
:10312000BDE8704006F048BDA0AE0024E02E654228
:103130000000C84270B50E4D86B00C46D5F8F40DAF
:1031400003681B69984780B102AE304614F07CFDDD
:1031500006AB13E903008DE8030004F1080105F54F
:10316000A75096E80C0006F02FFF06B070BD00BF18
:10317000A0AE0024F0B52E4F8BB0D1ED017A0646FB
:10318000D7F8F43D0C46FDEEE77A1A68184617EEBC
:10319000905A13699847EB0701D400283AD0D4E934
:1031A000040132F0DBFE002834D023690BB96369D7
:1031B00083B302A814F048FD02AA214630467AF0F3
:1031C000D5FD38B3D7F8F40D03681B69984720B3D1
:1031D00094ED000ADFED177AB4EEE70AF1EE10FA8B
:1031E00005DBD7F8F40D0368DB6C9847E0B106AC5B
:1031F000204614F029FD0AAB13E9030094E80C0003
:103200008DE8030002A90C4806F0DEFE60B1002044
:103210000BB0F0BD02200BB0F0BD02220F21074819
:1032200008F0F8FF0028D3D104200BB0F0BD00BF98
:10323000A0AE00240000003480C30024A02E00248F
:1032400010B58B8B84B0D12B16D8B12B34D9B23BAF
:103250001F2B3DD8DFE803F0413C3C3C3C3C3C3C70
:103260003C3C3C3C3C3C4C3C513C3C3C3C3C3C3C79
:103270003C3C3C3C3C3C3C61B3F5967F28D1D1EDD5
:10328000007A9FED377AF0EEE77AF4EEC77AF1EE46
:1032900010FA62D5D1ED017AF0EEE77AF4EEC77A52
:1032A000F1EE10FA59D502222E492F4808F028FFD6
:1032B00058B9042004B010BD142B09D102222B49A7
:1032C000294808F01DFF0028F3D0002004B010BDED
:1032D00004B0BDE810407DF045BD254B91ED010ADD
:1032E000D3F8F40D0368DB6C98470028EDD1E0E7D4
:1032F00004B0BDE81040FFF73DBF1D4BF7EE000ADC
:1033000091ED000AD3F8F44D31F05AFB0146204606
:1033100003F0F2FD002004B010BDD1ED027AD1ED32
:10332000016AFDEEE77A91ED007AFCEEE66A91ED36
:10333000030ABCEEC77A014617EE903A0A48CDED73
:10334000026A1CB28DED037A9DF808309DF80C20BE
:10335000009407F0FFFC04B010BD0220B6E700BFE8
:1033600000000034F8C30024A02E0024B4C70024B9
:10337000A0AE00242DE9F04F0D46352200212DEDA1
:10338000048BEC78A1B0944212A828BF144646F1F1
:1033900063FC05F10C0112A82246C84C46F112FC50
:1033A000D4F8F40D03681B69984720B921B0BDEC2F
:1033B000048BBDE8F08F06AE304614F045FC314674
:1033C000A4F5B7400CF054FC0028EFD09DF87C70B9
:1033D000012F6DD0FB1F022BE8D8BDF8785004F602
:1033E000DC430DF1280815F0C00F05F0180905F4AD
:1033F000806A05F4006B14BF012200220492C5F319
:1034000080220392C5F3C02215F0030505920FCB6D
:1034100088E80F000CD1072F68D19DED141A4046A3
:103420009DED130AB7EEC11AB7EEC00A15F042F9C6
:10343000B9F1000F00F09A809FEDA60AB0EE408A25
:10344000BAF1000F0DD1DDED1C7A083F9FED9C7A9B
:103450009FED9C0A012F67EE877A27EE800A40F2E3
:103460001481BBF1000F6CD1DDED1D7ADFED946AA4
:103470009FED947A67EEA67A67EE877AB9F1000F2E
:1034800000F0F280002D62D0B9F1000F8ED0049BC5
:10349000002B8BD0BAF1000F40F03381059B002B3D
:1034A00000F02F81DFED8B0A874806F055FB7DE7A2
:1034B000BDF8785004F6DC430DF1280815F0C00F74
:1034C00005F0180905F4806A05F4006B14BF0122A9
:1034D00000220492C5F380220392C5F3C02215F0A6
:1034E000030505920FCB88E80F00A1D1A7F10803CF
:1034F000012B00F2F180754E40469DED140A06F551
:10350000DA639DED137AD3ED007A06F2DC63D3ED36
:10351000006A20EE271A26EEC00AA7EE261AA7EEAA
:10352000270AB7EEC11AB7EEC00A15F0C3F8B9F111
:10353000000F00F0F6809FED670A0025B0EE408A8C
:103540007EE7B9F1000F6BD0DFED627A9AE70EAC3F
:10355000204614F079FB10A903C994E80C008DE80B
:1035600003004146584806F02FFD1FE74946D4F8AE
:10357000F40D03F0ABFCDDED178AB0EE408A9DED53
:10358000169A28EEA80AA9EE090A31F087FAF1EE98
:10359000480AB0EE481A40F2E33031F0F7FBF0EEA3
:1035A000490AB0EE408AB0EE680A43F177FCDFEDDD
:1035B000447AA7F1080360EE277A9FED420A012BB7
:1035C00027EE800A3FF63CAFA946404ED6F880363B
:1035D00007EE903AF8EEE77A37EE800A31F024FBF6
:1035E000BAF1000F18D1DDED1C7A4D469FED347A0B
:1035F000D1469FED340A67EE877A27EE800A06F5FA
:10360000D0634FF0000AD3ED007AF8EEE77A37EE98
:10361000800A31F009FB24E7BBF1000F18D04D46BA
:10362000BAF1000F00F0A780F7EE000ADFED297A6B
:10363000002D8CD0049B002B3FF4B8AE039B33B31A
:10364000059B23B360EE880A1F4806F085FAADE6B5
:10365000DDED1D7A4D46DFED1A6AD9469FED197AE8
:1036600067EEA67A67EE877ADFED196AFFEE000A49
:103670009DED166AB7EE007ACB46B4EEE66AF1EE3F
:1036800010FA88BFF0EE470AD2E7104EB7E7BBF159
:10369000000F09D1039B3BB160EE880A0A48B0EEE7
:1036A000670A06F089FA81E6BAF1000F7FF47EAE70
:1036B000059B002B3FF47AAEC4E700BFA0AE002408
:1036C000E02E65420000C84280C30024A04E0024C2
:1036D000000000B40000000096E80F009DED141AF1
:1036E00000259DED130AB7EEC11AB7EEC00A88E8AF
:1036F0000F00404614F0DEFFB9F1000F7FF49CAEDE
:1037000034E7BBF1000F7FF451AE039B002B3FF475
:103710004DAEB0EE670A5FED110A194806F04CFA9B
:1037200044E64946D4F8F40D03F0D0FBDDED178AEA
:10373000B0EE408A9DED169A28EEA80AA9EE090A75
:1037400031F0ACF9F1EE480AB0EE481A40F2E3303D
:1037500031F01CFBF0EE490AB0EE408AB0EE680A88
:1037600043F19CFBDFED077A60EE277A9FED060AB6
:1037700027EE800A2AE7D946DFED047A74E700BF16
:1037800080C30024E02E65420000C8420000000013
:103790002DE9F04F0C46352200212DED048BE57804
:1037A0009DB095420EA828BF154646F155FA04F182
:1037B0000C010EA82A46844D46F104FAD5F8F40D02
:1037C00003681B69984708B39DF86C300B2B1DD814
:1037D000DFE803F0211C1C211C21211C1C1C2121C1
:1037E000002E00F0D3809FED790A002B40F0BB80C3
:1037F0000AAD284614F028FA0CA903C995E80C0074
:103800008DE803002146724806F0DEFB1DB0BDECDA
:10381000048BBDE8F08FBDF868C005F6DC4306AC4C
:103820001CF0C00F0CF018060CF48067CCF3802954
:1038300014BF4FF0010A4FF0000A0CF40068CCF3FB
:10384000C02B0FCB84E80F001CF003034ED0002EDA
:103850005DD0DFED5E7AB0EE678A4FB9DDED187AA4
:103860009FED5C7A9FED5C0A67EE877A67EE807A5F
:10387000B8F1000FB4D19DED197ADFED566A9FEDD6
:10388000560A27EE267A27EE000A002EADD19FEDCC
:10389000536AFFEE000ADDED125AF7EE006AF4EE0D
:1038A000C65AF1EE10FA88BFF0EE660A002B9FD0E0
:1038B000002E5BD1BAF1000F55D0B9F1000F02D044
:1038C000BBF1000F0AD1B8F1000F02D1B9F1000F1E
:1038D00062D1002F9AD1BBF1000F97D068EE200A79
:1038E0003B48B0EE670A06F037F98FE7DDE90F21B4
:1038F00005931046CDE9031232F030FB002885D045
:10390000049A0399059B08920991002EA1D1314692
:10391000D5F8F40D039303F0D9FADDED138AB0EE78
:10392000408A9DED129A28EEA80AA9EE090A31F004
:10393000B5F8F1EE480AB0EE481A4FF48A6031F05B
:1039400025FAF0EE490AB0EE408AB0EE680A43F17B
:10395000A5FADFED207A039B60EE277A9FED1E0A21
:1039600067EE807A79E7002E3FF450AFBAF1000F8E
:103970003FF44CAFB7B9BBF1000F13D0B0EE670AFC
:10398000DFED120A124806F0E7F83FE7C7B1F7EE9D
:10399000000A9FED0E0A89E768EE200A0C4806F03F
:1039A0000BF933E7B8F1000F7FF430AFB9F1000F36
:1039B0003FF42CAFDFED050A054806F0FDF825E7DA
:1039C0009FED020A63E700BFA0AE002400000000E4
:1039D00080C30024E02E65420000C842000000B40D
:1039E0004B7A91F80AC0CA7A43EA0C2343EA0243AD
:1039F000542B05D0562B07D0522B03D07CF044B863
:103A0000FFF7B8BCFFF722BBFFF7C2BE014B93F82C
:103A100032037047A06E0024074B084AD3F8F41D08
:103A2000914201D000207047A3F5005393F9780527
:103A3000B0FA80F040097047A0AE002468C80024A6
:103A4000084B094AD3F8F41D914201D00020704779
:103A5000A3F5005393F97805A0F10100B0FA80F0C6
:103A600040097047A0AE002468C8002438B5436AF6
:103A700004462B4D43F4B8434362D5F8F40D036874
:103A80001B6A984738B1D4E90A3242F4406243F4E1
:103A90004063C4E90A32D5F8F40D0368DB6898473F
:103AA00038B1D4E90A3242F4A04243F4A043C4E955
:103AB0000A321C4B1D68ADB1284697F025F8002846
:103AC00007DDD4E9092342F4807243F48073C4E92A
:103AD0000923284697F018F8012803D0E36A43F435
:103AE0008073E362104B186810B190F8803203B90C
:103AF00038BDD4E90923002142F4807243F4807375
:103B0000C4E9092363F02AFE0028F1D064F0C8FA62
:103B10000028EDD0E36A43F48073E36238BD00BF50
:103B2000A0AE002494D70024E4CB002470B545F265
:103B3000A45684B0044641F69825064425443046F0
:103B4000CBF02EFADFED1C7A002301A920EE270A24
:103B500004F51250019303938DED020A09F0A2FEC1
:103B60000CF0C2F80CF036F845F24C626D21284694
:103B700022446DF08BFC284606F54C726C216DF0EA
:103B800085FC204601F0CEFF70B904F5C04393F9DF
:103B90007C3E002B06DD45F6B01269212846224402
:103BA0006DF074FC04B070BD45F634026A212846FD
:103BB00022446DF06BFCE8E7E02E65422DE9F04F02
:103BC00006463F482DED028B93B008F08BFC20B9E0
:103BD00013B0BDEC028BBDE8F08F41F2E8771921FC
:103BE0003744384663F062FE0028F1D00EA806F58F
:103BF000805814F029F80EA906F512500CF00AF8B6
:103C000098F8683A002BE3D00025DFF8CCA0DFF865
:103C1000CC90AB469FED2B8A06E0013598F8683AC8
:103C20005FFA85FB5B45D3D95946384663F096FD6C
:103C300004460028F1D0836893F92130192BECD188
:103C400064F02EFA06EB8B030028E6D0626803F5D9
:103C500000431169D3F8142E8A42DED0C3F8141E33
:103C600023689B6A534525D18DED0D8AD5F02EF83A
:103C70009DED0D7A144AB7EEC77A8DED0A7B636825
:103C800093ED007A119BB7EEC77ACDF810B006938A
:103C9000109BCDF8049005930C4BCDE9020141F641
:103CA000982000930A4930440A4B8DED087B6EF052
:103CB00027FAB2E70DA9204698470028D6D1D3E7C6
:103CC000A02E00240000000068EB160898EB1608F0
:103CD00088EB160860EB16081123020890EB160813
:103CE000F0B58BB0154606460F462422002101A8E8
:103CF0001C4645F1B1FFA3238DF8043095238DF8C0
:103D0000053003238DF80630D4F0E0FF2B68242221
:103D1000CDF8070041F6982004936B683044CDF845
:103D20000B1001A90593AB686568069323688DF8AD
:103D30000F700793A368089509936DF057FD0BB0BA
:103D4000F0BD00BF30B589B01D2204460021684691
:103D500045F182FF952304F50045A3218DF801303C
:103D600001238DF800108DF80230D4F0AFFFCDF8AC
:103D70000300D5F8F40DCDF807100368DB6B984706
:103D8000D5F8F40D10EE103ACDF80B300368DB6A6D
:103D90009847D5F8F40D10EE103ACDF80F300368BF
:103DA0001B6B984710EE103AD5F8F40DCDF8133090
:103DB00004F50053D3F88036ADF8173003685B6B19
:103DC000984741F6982010EE103A1D22694620448B
:103DD000CDF819306DF00AFD09B030BD2DE9F04184
:103DE00000F5C0452DED088B95F97C3E90B0002B79
:103DF00040DD044646F27C5041F698282044A04419
:103E0000CFF090F900283AD105469FED228AD4F0F0
:103E10005DFF45F21853074646F67C6023440E4684
:103E200020441D4C93ED119A93ED12AA93ED13BA11
:103E3000B7EEC99A07F024FCB7EECAAAB7EECBBA20
:103E40001649B7EEC88A4046B7EEC00A144B154A69
:103E50000495CDE900148DED0CBB13498DED0AAB33
:103E60008DED089B8DED068B8DED0E0BCDE9027669
:103E70006EF046F910B0BDEC088BBDE8F08105F29C
:103E80007C539FED0A8A95F83C5693ED137A27EE02
:103E9000088ABCE75241C07FE4EB1608ECEB160839
:103EA000A0EB1608A8EB1608DCEB1608E02E65421E
:103EB00030B545F2A4552F4B044605442DED028B39
:103EC0008BB028469FED2C8A69460093CBF064F9AD
:103ED0002122002101A845F1BFFEA3238DF8043063
:103EE00095238DF8053002238DF80630D4F0EEFED0
:103EF00004F5E043CDF80B10CDF80700D3F84033BC
:103F0000B3F90830ADF80F3045F2185323445B6A1B
:103F1000CDF8113004F50043D3F8F40D03689B6B22
:103F2000984710EE103A2846CDF81530009BCDF892
:103F30001930CAF0F3FE20EE080A42F2B87142F2DC
:103F40009470214410EE103A2044CDF81D3036F024
:103F50001BFB20EE080A41F69820212201A92044EB
:103F600010EE103ACDF821306DF040FC0BB0BDECF6
:103F7000028B30BD5241C07FE02E654200F5805378
:103F8000244970B58AB093F8953445F2A455044697
:103F9000019103EB430300F68841054401EB8303E1
:103FA000284601A9D3F87862CBF08EF81D220021B3
:103FB00002A845F151FEA3238DF8083095238DF812
:103FC0000930D4F083FE04F5E043CDF80B00CDF8C2
:103FD0000F102846D3F84433B3F90830ADF8133046
:103FE00045F2185323449B6ACDF81530CBF094FA70
:103FF00041F6982010EE103A1D2202A9CDF8193092
:104000002044019BCDF82160CDF81D306DF0EEFB12
:104010000AB070BD5241C07F38B541F698250446BC
:10402000054404F5805428466CF022FD28466CF0C7
:10403000CBFD94F9C83B03B938BD2846BDE83840EC
:104040006CF0FABE00F5004310B50446D3F8F40D49
:1040500003681B68984704F58043014641F69820A1
:1040600093F8382120446DF09DFD04F512500CF0BA
:1040700047F804F55670BDE810401FF093BD00BF2F
:10408000A92070472DE9F041054604307DF0B6FACD
:104090004D4F4E4B05F1BC0405F56F766B60204625
:1040A0007DF022FD44F8307BB442F8D105F6047669
:1040B00020467FF055FE05F6887405F6486005F544
:1040C0000058C3F03FFB3046B8F00AFF31462046A7
:1040D00041F23C26B9F0DAF841F2B0102E44214604
:1040E000284442F65057CFF0EBFF3046CAF016FD99
:1040F00041F2A860002142F2E82428442F44CDF088
:1041000033FB05F5BB5096F05BFA314B05F50450D7
:104110002C44C8F8FC309EF00FFD42F248102844B1
:10412000CEF0ACFB42F2E01028449BF021FA42F2C0
:10413000FC10284462F0B2F9264B42F21420C8F871
:10414000FC312844CEF0A4FF3A4631462046CCF05C
:104150009DF8214B04F2C470C8F8E83213F074FDE6
:1041600004F2D47013F070FD04F2E47013F06CFDEF
:1041700004F2F47013F068FD04F6040013F064FD1B
:1041800004F6140013F060FD42F61430284406F0E3
:10419000F1FF42F6583028449DF0FEFF42F61C50D5
:1041A0002844C0F05FFA31463846CBF0AFFB42F608
:1041B0003070284404F02CFC284608495FF0A2FF28
:1041C0002846BDE8F08100BF203C1708343C1708A2
:1041D000A8C800244CE81608C8351A0890321708F9
:1041E00044F228311022F0B50144B5B004466BF01A
:1041F000DBF900222B215E4814AF60F04BFD61F02B
:1042000085FC5C4A1A210020138843F002031380C6
:104210007FF058FC462102207FF054FC204601F03C
:1042200081FC002840F08D80534D7FF083FD0DF11F
:10423000100C95E80F008CE80F0002A9604660F0B2
:104240001DFC50B110359DF808C03E46BCF10C0F66
:1042500095E80F0007C633707DD9484B08AD0CAE0A
:1042600003F1100C0FCB85E80F009CE80F0086E8E7
:104270000F0003A9284660F001FCB7EE000A0028F1
:1042800053D00021284660F049FC44F26835802272
:104290003B49384645F196FC254408210022384622
:1042A00060F0F8FCB1EE0C0A364861F037FC10A95A
:1042B00028465FF087FC002835D0334A1368D907B9
:1042C0001AD443F62831314B43F66410214420447C
:1042D000D96043F69C6118602144996143F6D0216E
:1042E0002144596243F6B4712144196341F6AC315B
:1042F0002144D9630123136028460622234901255E
:1043000060F044FD41F698210023214A2144FD201C
:10431000009560F0D9FC1F4B1A68D2070AD501211D
:104320001D4860F051FD35B0F0BD0146304660F0EB
:10433000F5FBAAE742F26C3217491D6022440A607D
:10434000EDE746F2A8401E23394620448DF8503050
:1043500061F074FF68E734AB07989C441CF8803C1C
:1043600000EE103AB8EE400A61F0D8FB75E700BFE6
:10437000E02F1708ACCB002438DE160858DE1608EC
:1043800078DE1608CC2F1708902E0024C4250024B0
:104390008C271808942E00240C2600240069C0F3F2
:1043A000401070470F2904D8302303FB0100B830B8
:1043B00070470020704700BF014B93F95C037047C2
:1043C000A06E0024024B93F8FC0D00F00100704732
:1043D000A0AE0024014BD3F840037047A09E0024F8
:1043E000002905DB0748CBB290F85C239A4200D243
:1043F0007047D0F858330122A0F5E040595C07F02F
:1044000009BF00BFA09E002408B50368084A9B6846
:10441000934208D1074B93F8FC0D00F0010080F0A7
:104420000100C0B208BD984780F00100C0B208BDCD
:10443000C5430208A0AE002430B589B00023124C59
:1044400003AD07932846CDE90133CDE90333CDE928
:10445000053313F0F9FB1023ADF8063094E80F0094
:1044600085E80F0001A904F6B40037F0DDFC40B187
:10447000064BB4F8E8281B680549986903681B686F
:10448000984709B030BD00BF7CBB0024982E0024A3
:10449000183A170801290A4604D0022901D001B1AF
:1044A00070470122014807F04FBC00BF1C9D00244B
:1044B0004A292ADC032930DD0B1F462B2DD8DFE8E3
:1044C00003F0392C2C392C2C2C2C2C2C2C2C392C6A
:1044D0002C2C2C2C2C2C2C2C2C2C2C2C2C2C2C2C1C
:1044E0002C2C2C2C2C2C2C2C392C2C2C2C2C2C2CFF
:1044F00039393939393939392C392C2C2C392C2C7A
:104500002C2C2C2C2C2C392C3A00D32905DCC82936
:1045100005DC61290ED09B2910D07EF085BBA1F16E
:10452000C90C012303FA0CF340F2434C13EA0C0FBD
:10453000F3D0704770471146FFF7ACBF704700BF1C
:104540009B29F0B5054683B000F3AC8029297FDDB7
:10455000A1F12A03712B00F2B080DFE813F04B01C8
:10456000AE00AE00AE00AE00AE00AE00AE00720017
:104570005801650172017E018A0196011D01AE009C
:104580002A01AE00AE00AE003701AE00AE00AE00B4
:10459000AE00AE00AE00AE00AE003F01AE00EB00DC
:1045A000AE00AE00AE00AE00AE00AE00AE00AE009B
:1045B000AE00AE00AE00AE00AE00AE00AE00AE008B
:1045C000AE00AE00AE00AE00AE00AE007500AE00B4
:1045D000AE00AE00AE00AE00AE00AE00AE00AE006B
:1045E000AE00AE00AE00AE00AE00AE00AE00AE005B
:1045F000AE00AE00AE00AE00AE00AE00AE00AE004B
:10460000AE00AE00AE00AE00AE00AE00AE00AE003A
:10461000AE00AE00AE00AE00AE00AE00AE00AE002A
:10462000AE00AE00AE00AE00AE00AE00AE00AE001A
:10463000AE00AE00AE00AE00AE00AE00AE00AE000A
:10464000F100022A00F094810124204603B0F0BD5D
:10465000102932D8102930D801A353F821F000BF17
:1046600049460208BB460208BB460208BB46020890
:10467000DF460208BB460208BB460208F7460208AE
:10468000BB460208BB460208BB460208BB460208FE
:10469000BB460208BB460208BB460208BB460208EE
:1046A000C7460208A1F1C9030A2B06D8012440F22B
:1046B000434004FA03F30342C7D1284603B0BDE8E0
:1046C000F0407DF0F7BD002A00F0F880022ABBD14F
:1046D0003522B249B248012407F012FDB5E7002A9D
:1046E00000F0DF80022AAFD13522AE49AC48012468
:1046F00007F006FDA9E7022AA6D1AB4EA74FD6F8D0
:10470000F43DBB42A0D0A6F63C40C4F097FA044664
:10471000002800F03281D6F8F43DBB4294D006F573
:104720008056B6F9C435002B00F05C812846FFF7AF
:1047300083FE8AE7114628460124FFF7ABFE84E793
:104740009A480192CFF0F6FD00287FF47DAF98489B
:10475000C4F074FA00283FF477AF96499248A1F26A
:104760005443019AD0F8F44D8C4218BF9C4214BFB8
:1047700001240024022A14BF002404F00104002CA8
:104780003FF462AF1A207EF093FF7BF05DFD8A4A12
:10479000022171F0F3FE58E7002A00F09780022A08
:1047A0007FF452AF352285497D48012407F0A8FCEB
:1047B0004BE7002A00F09B80022A7FF445AF3522A8
:1047C0007F497748012407F09BFC3EE7764B0124A4
:1047D000D3F8F40D03685B6D984736E7002A7DD067
:1047E000022A7FF431AF352276496D48012407F063
:1047F00087FC2AE7002A00F0AB80022A7FF424AF6E
:10480000352271496648012407F07AFC1DE7002A29
:1048100000F0A680022A7FF417AF35226B4960486A
:10482000012407F06DFC10E7002A00F08980022ABD
:104830007FF40AAF352266495948012407F060FC2D
:1048400003E7002A74D0022A7FF4FEAE35226149C4
:104850005348012407F054FCF7E6002A60D0022AEE
:104860007FF4F2AE35225C494D48012407F048FC44
:10487000EBE6002A4BD0022A7FF4E6AE35225749F8
:104880004748012407F03CFCDFE6002A37D0022A23
:104890007FF4DAAE352247494148012407F030FC65
:1048A000D3E6414A3F4BD2F8F42D9A427FF4CCAE86
:1048B0007DF012F901247DF009F8C6E63A4A374B3B
:1048C000D2F8F42D9A427FF4BFAEF1E7364A3B4B63
:1048D000D2F8F42D9A427FF4B7AEE9E7324BA3F653
:1048E0006852D3F8F43D93427FF4AEAEE0E72E4A2F
:1048F000334BD2F8F42D9A427FF4A6AED8E72A4A79
:104900002C4BD2F8F42D9A427FF49EAED0E7264B82
:1049100003F5A752D3F8F43D93427FF495AEC7E771
:10492000214A2D4BD2F8F42D9A427FF48DAEBFE789
:104930001D4A284BD2F8F42D9A427FF485AEB7E792
:10494000194A234BD2F8F42D9A427FF47DAEAFE79B
:10495000154A1D4BD2F8F42D9A427FF475AEA7E7A5
:10496000114A1A4BD2F8F42D9A427FF46DAE9FE7AC
:104970000B48012401F080FA67E607F1380036F0B1
:1049800059FF7BF061FC164A052171F0F7FD2146C5
:10499000A6F50040012401F0CFF856E6F8C3002444
:1049A000A02E0024B4C70024A0AE0024B8830024A5
:1049B00064A200242CC70024483A17082CC80024FD
:1049C00068C8002438A10024F0C7002410C30024C4
:1049D00048C3002478C70024D8C2002480C3002420
:1049E0002C3A17082846FFF727FD9FE6002070475E
:1049F000002070470020704700207047002070475B
:104A00000020704700207047704700BF704700BF0C
:104A1000002070470020704700207047002070473A
:104A2000002070470020704700207047002070472A
:104A3000002070470020704700207047002070471A
:104A400000207047002070470020704708B50368B9
:104A5000DB68984780F00100C0B208BD01207047B4
:104A6000012070479FED010A704700BF0000000061
:104A7000002070470120704700207047704700BF3A
:104A80001020704700487047503C1708704700BF1F
:104A900000207047012070470020704700207047B9
:104AA000034644F22C301844704700BF004870475A
:104AB000A019170800F50040D0F8F40D03681B6832
:104AC000184700BF00F5004249F258530344D2F89A
:104AD000F40DC01AB0FA80F04009704710B4044CCD
:104AE00026200C60082110705DF8044B1960704797
:104AF000FC40170845F21853DFED096A9FED097A6B
:104B00000344012093ED096AC6EE267AC1ED007ACE
:104B1000D3ED0A7A67EE877AC2ED007A704700BF5C
:104B200000A08C450AD7233C00F50040D0F8F40DD6
:104B30000368DB6C184700BFA1F10A00B0FA80F0EF
:104B40004009704703685B68184700BF01F04ABA24
:104B500001F096B88AF05ABC69F078BC2DF006BA1C
:104B60006CF0E0BF07F01AB99AF05CBD05F02EBEFC
:104B700001F042BB01F01ABD0FF016BF80F06CBE11
:104B800080F0AEB806F070B98CF064BF0FF0FAB8E0
:104B90007CF024BE79F072BF7AF0DCBD07F0FAB881
:104BA00007F018B9CEF07EBC95F076BFC2F0BEBF5C
:104BB0000EF02AB81FF07CBD00F04ABF5BF042BF88
:104BC00007F0C0B906F06EBA01F0C0BC10B50368BA
:104BD0000446DB68984700B910BD20460021BDE8B7
:104BE000104002F089B900BF03F04CBD03F006BCD1
:104BF00002F0E2BE38B500F5004305462DED028B0C
:104C0000D3F8F40DB0EE408AF0EE608A03681B69B9
:104C10009847044640B149F2E040F0EE680AB0EE31
:104C2000480A284404F0FAFF2046BDEC028B38BD48
:104C300038B500F5004305462DED028BD3F8F40D91
:104C4000B0EE408AF0EE608A03681B69984704461C
:104C500050B19FED070A49F2E040F0EE680A28EEF5
:104C6000000A284404F0A8FF2046BDEC028B38BDA2
:104C70000000C8420139034610B51446072900F266
:104C80009D80DFE801F014778724384D620445F2F7
:104C90001852B7EE001AFFEE000AF8201A4492EDFF
:104CA000100A30F073F8012084ED000A10BD45F2BF
:104CB0001852B7EE001AFFEE000AF2201A4492EDE5
:104CC0000E0A30F063F8012084ED000A10BD45F2B1
:104CD0001852DFED3B7AB7EE001A0244FFEE000AED
:104CE000FE2092ED090A80EE270A30F04FF80120ED
:104CF00084ED000A10BD45F21852DFED327AB7EEAE
:104D0000001A0244FFEE000A40F2011092ED0D0A73
:104D100020EE270A30F03AF8012084ED000A10BD99
:104D200045F21852DFED277AB7EE001A0244FFEE83
:104D3000000A4FF4827092ED110A20EE270A30F03B
:104D400025F8012084ED000A10BD45F21852DFED70
:104D50001D7AB7EE001A0244FFEE000A40F2071077
:104D600092ED120A20EE270A30F010F8012084EDAF
:104D7000000A10BD45F21852B7EE001AFFEE000A05
:104D8000F5201A4492ED0F0A30F000F8012084ED6E
:104D9000000A10BD45F21852DFED0A7AB7EE001A8C
:104DA0000244FFEE000AFB2092ED0A0A20EE270AD9
:104DB0002FF0ECFF012084ED000A10BD002010BD93
:104DC00000A08C450AD7233C49F2585C844400F586
:104DD0000040D0F8F40D604501D00020704702F08B
:104DE0000DBD00BF49F2585300F500420344D2F80C
:104DF000F40D984200D0704702F01EBD0B4B70B509
:104E0000D3F8F43D05460E461A681846D36898470D
:104E1000044640B105F50040D0F8F40D0368DB6BA3
:104E2000984786ED000A204670BD00BFA0AE002462
:104E30000B4B70B5D3F8F43D05460E461A6818467C
:104E4000D3689847044640B105F50040D0F8F40D0A
:104E50000368DB6A984786ED000A204670BD00BFF4
:104E6000A0AE00240B4B70B5D3F8F43D05460E46BA
:104E70001A681846D3689847044640B105F50040C3
:104E8000D0F8F40D03685B6B984786ED000A204666
:104E900070BD00BFA0AE002400F5004370B504460D
:104EA000D3F8F40D86B00D4603681B69984780B1AE
:104EB00002AE304612F0C8FE06AB13E903008DE8DF
:104EC000030049F2E040294696E80C00204405F032
:104ED0007BF806B070BD00BF00F5004370B5064614
:104EE0000D462DED028BD3F8F40D03681B6998472E
:104EF000044600B395ED010AD5ED007A20EE000AD4
:104F0000A7EEA70A2FF0CAFDD5ED000AB0EE408A41
:104F100095ED010A41F1C2FFDFED097A9FED097AB3
:104F200049F2E04020EE270AF0EE480A304420EE35
:104F3000070A04F011FE2046BDEC028B70BD00BFD5
:104F4000E02E65420000C842F8B5464900F500432E
:104F5000454A05460160D3F8700CC3F8742A08B1BD
:104F600013F030FE414B43F61C602B60284412F0D6
:104F7000E7FD05F5405393F8582842B9D3F8544853
:104F80002CB120462BF032F9204613F017FE42F2E6
:104F9000503041F6DC6441F6C46628442C442E446B
:104FA000BEF07CF914F8043C083C3BB9276838464D
:104FB00027B12BF01BF9384613F000FEA642F1D1C1
:104FC00041F6C83041F2847441F2247628442C44DE
:104FD0002E4480F0FBFA2046183C2AF09DFBA642A6
:104FE000F9D141F2B01441F26817214B2C442F44FF
:104FF000C5F8883C14F8043C083C3BB926683046A8
:1050000026B12BF0F3F8304613F0D8FDBC42F1D1B5
:1050100005F64C6070F076FA05F5626070F072FA91
:1050200005F6F45070F06EFA05F6485070F06AFA22
:1050300005F61C5070F066FA05F54F6070F062FAE4
:105040000C4A95F81032C5F8FC2043B9D5F80C424B
:105050002CB120462BF0CAF8204613F0AFFD2846AD
:10506000F8BD00BF044417085C441808581F18080E
:1050700060C017081C2F1A08094B10B51B7804468E
:1050800043B904F50044D4F8F40D0368BDE81040BA
:105090009B68184745F2A4502044CAF027FCF0E76B
:1050A000CCD0002400F5804393F9543353B300F57A
:1050B000004370B5D3F86C5C044605B970BDD3F0FD
:1050C000FDFD04F5E042DFED107A034692EDA50AFE
:1050D00040F269109FED0D1A5D1B20EE270ADFEDEF
:1050E0000C0A2FF053FEFCEEC07A2046094A02213A
:1050F00017EE903A9D42BDE8704034BF0023012373
:1051000001F052B9704700BF00007A440000804FA0
:1051100000000000E42D1708F8B56F4B0546002786
:1051200044F2481440F8043B44F2C8268AF0C2FA1C
:1051300005F110000EF086FF05F1B000C5F042FD4C
:1051400005F5287068F064FF05F556701DF0B6FB94
:1051500005F5F4600DF04CF905F63C1013F08CFDEC
:1051600005F688402CF0FAFB41F218702C442E44CE
:1051700028448AF021F841F2E870284461F05EFD8D
:1051800041F6982028446CF027FA41F6AC302844C8
:1051900099F008FC41F6C830284480F0FFF941F648
:1051A0000440284411F084FD05F5E650ADF09CFC68
:1051B00042F250302844BEF05DF842F26C30284490
:1051C00069F034FB42F2DC3028448BF0D9FE05F55F
:1051D000005342F23040414A83F8207442F22043A7
:1051E00028442B44136058F09DFC394605F51250B5
:1051F00008F096FC42F67830284491F043F942F6E4
:10520000A8302844ACF092FB43F234602844B5F057
:1052100017FA43F24C702844B3F0D0FE43F2747096
:105220002844B8F085FA05F56050BCF0A3FF43F6BA
:1052300064002844BDF026FD43F6BC002844AAF0D3
:1052400035FC43F66410284407F0D2FA43F6D02028
:105250002844ADF095F943F628302844C0F062FDAB
:1052600043F67C601E4928445EF04CFF43F6946090
:105270002844C7F013FE43F69C6028449AF0F8FADD
:1052800043F65C702844BFF0DBF943F6B470284461
:10529000D3F034FD05F5804383F8387120460C3493
:1052A00070F07AFBB442F9D144F2D4200D4C28447A
:1052B000C0F0F8FB44F2F82028446FF01DFF23688B
:1052C00033B9284608495EF01DFF28462560F8BD21
:1052D0000648D3F0C1FC00BF581F180804D70024AB
:1052E00080CC19081CCC0024C01D1808583C170895
:1052F0002DE9F04186B00446FFF70EFFC449C54BC7
:1053000044F22435C44A1960254422600B7C4BB119
:10531000002301339BB203EB830201EB8202127C78
:10532000002AF6D1BD49BE4A0B80BE490B801368E6
:10533000002B40F06A8144F26830156004F5E045C6
:1053400048F67428204448F64436FEF79BFE47F2A0
:10535000383004F50047A04420442644C5F018FC2A
:1053600044F25D3347F2603023442044C5F858339B
:10537000062385F85C337FF067FA47F2C430204497
:10538000C3F038FCA84B47F22440C5F8C43320448E
:10539000C2F052F9A54B47F22840C5F8243448F62C
:1053A000A42520445BF0D8FA47F268402544204405
:1053B000A1F02AFB48F680102044D0F011FB9C4B52
:1053C00008F10C00C7F8743AD2F0D0FC2846143526
:1053D00077F078FBB542F9D11E22002340F2CC6071
:1053E000C7F8742CA7F8783C13F0E2FB034648F6A4
:1053F0007C40C7F8703C2044D2F0B8FC48F6C0406E
:105400002044D2F0B3FC8B4B1A68002A00F0FA80DB
:10541000894B48F6DC4004F5144549F25856C7F864
:10542000743A204412F010FC48F6EC404FF48051DE
:10543000264420444FF0FF380EF052FF48F66C50DF
:10544000204480F0F1F97D4BC7F8F45D48F64060E8
:10545000009306AB7A4A4FF4007120444FF6FF7771
:10546000CDE9044213E90C000DF0F0FF284601F0ED
:10547000ABFA04F51045734B49F23840C5F80034D7
:10548000204401F0A1FA704B49F27040C5F838345D
:10549000204401F099FA6D4B49F2A840C5F87034E8
:1054A000204401F091FA6A4B49F2E040C5F8A83473
:1054B000204401F089FA674B49F24850C5F8E034BE
:1054C000204412F0C1FB304601F07EFA624A634B81
:1054D00049F2D450C5F85825C5F8B0352044604A83
:1054E000604BC5F8B825C5F8C035C5F8AC65C5F83A
:1054F000B465C5F8BC65383612F0A6FB49F2F05029
:10550000204412F0A1FB49F20C60204412F09CFBF5
:10551000554B49F22860A5F82476C5F8203620447A
:1055200012F092FB514B52493046C5F8D8871E60A5
:105530005EF0E8FD49F2F070A5F8CC85A5F8E875B5
:1055400049F68C07204449F6702612F07DFB49F697
:1055500040002744264420444FF0804812F074FB5A
:1055600049F65C00204412F06FFB49F678002044B5
:1055700012F06AFB384601F027FA3E4B07F138007B
:10558000C5F88C3812F060FB49F6D800204401F0D1
:105590001BFA394B49F61410C5F8D838204401F0ED
:1055A00013FA364B49F65010C5F81439204401F06F
:1055B0000BFA334B49F68C10C5F85039204401F0F2
:1055C00003FA304B49F6C810C5F88C39204401F075
:1055D000FBF92D4B49F60820C5F8C839204403F0E3
:1055E0000FFF03A93046CDF80C8070F05BFA02A9DA
:1055F00006F10C00CDF8088070F054FA204606B091
:10560000BDE8F081C3F8008002E72048D3F024FB16
:1056100040351708D4CB002404441708D0CB00240D
:105620006CCB0024A0CB0024F8E716083CE8160851
:105630005C44180898D0002428EB1608F443170897
:10564000C94B0208903C1708EC4C1708D44D1708BA
:10565000A0461708804C170880481708E94B020835
:10566000ED4B0208F14B02080000FFFFBCCA00240A
:10567000D8D21708604D1708C84F1708584E17089A
:105680005C4F1708CC4B1708CC4E17086C3C17081A
:1056900070B5044647F2C43084B004F51255204476
:1056A000FCF7E0FB204606F061FC0021284604F5EB
:1056B00000460AF0F9F948F6DC41284621440AF090
:1056C000A9FA04F5005386F8100E93F8FC1611F0B1
:1056D000010104D123682046D3F8AC309847002359
:1056E00001A928460193029303930AF0CDFA0028FA
:1056F00045D194F8F92694F864368AB10121204600
:1057000006F0EAFEF8B98021204606F0E5FE30BB3F
:105710004FF48011204606F0DFFE58BB04B070BD88
:10572000B02202FB034393F84134022BE6D905F281
:10573000044306F63C66012120461B68336006F0F0
:10574000CBFE0028DFD02046FEF7F0F92046FEF71A
:1057500045FB8021204606F0BFFE0028D8D02EF061
:1057600073FD2BF043FD4FF48011204606F0B4FE8C
:105770000028D3D0284608F073F904B070BD06F6AF
:105780003C6601A834F04EFA86ED000AB6E700BF89
:10579000FFF77EBFF8B50221044606F09DFE88B9EA
:1057A0001021204606F098FEF0B92021204606F090
:1057B00093FE38BB4FF48061204606F08DFE002832
:1057C00047D1F8BD0121204606F086FE0028E7D12A
:1057D0002046FEF7ABF92046FEF700FB10212046DD
:1057E00006F07AFE0028E0D02046FEF7C7FB45F21F
:1057F000B0102044C2F0BEF92021204606F06CFE15
:105800000028D7D047F2B8052046FEF79BFA25447A
:105810002846CAF0C1F80028CCD041F6982647F2B5
:10582000D407284626442744CAF028FA6E2107F1F7
:10583000400230466BF02AFE6F21304607F16C02C1
:105840006BF024FE4FF48061204606F045FE0028F0
:10585000B7D045F6C8202044BDE8F84095F0A6BA78
:10586000FFF798BF10B54FF40051044606F034FE20
:1058700088B94FF48041204606F02EFEA8B9802159
:10588000204606F029FEF0B94FF48051204606F07C
:1058900023FE38BB10BD2046FEF70AFB4FF48041C3
:1058A000204606F019FE0028E9D02046FEF7B4FB9A
:1058B00045F26C202044B7F087FB8021204606F09B
:1058C0000BFE0028E0D02EF0BFFC2BF0B5FC04F559
:1058D000E650AEF013FA4FF48051204606F0FCFD7E
:1058E0000028D7D048F66C502044BDE8104080F026
:1058F00077BB00BFFFF7B6BFF0B547F2C436036809
:1059000083B00446D3F8BC3006449847374D7EF048
:105910002BFC374F7DF074FD00213046FCF792FBE5
:1059200003463046AB710123EB71C3F087F93B6846
:105930002871DB6A2F4A93F89C306B7104F580451F
:10594000B5F832131170002B3FD095F83A31002B87
:1059500045D045F6082685F83A3145F218552644D3
:10596000254496ED000A28468DED010ACEF0E2FCB2
:10597000014646F250609DED010A2044CAF086FEC1
:1059800096ED000A28468DED010ACEF0D3FC0146C3
:1059900047F2B8009DED010A2044CAF03DF868F0D6
:1059A00013FE68F097FA45F2F0202044B7F060FD4E
:1059B000ACF064FF04462846CFF016FF01462046AF
:1059C00003B0BDE8F040ACF0B5BE204600F028F9C9
:1059D0003B68DB6A93F89C30002BBAD0B5E7D3F074
:1059E0006DF90123C5F83C01B3E700BFF0CA0024FC
:1059F000982E0024F4270024FFF77EBF38B5054C0D
:105A00000A46054B01462468256820462C68A047B5
:105A1000002038BD982E0024A02E002410B5084C7C
:105A2000D2F0FEFC074B024620461A60FFF760FCEE
:105A30002046054A0549BDE8104040F191B900BF34
:105A4000A02E0024982E0024807B0124494F0208B8
:105A500000F5104393F8FD330BB105F07BB810B59A
:105A6000044682B045F2A450002301A920440193CA
:105A7000C9F02AFB47F2C4302044C3F0DFF80146E6
:105A800045F21850D4EDD40A9DED010A2044CFF020
:105A90002FFE02B010BD00BF0346DFED1F7ADFED21
:105AA0001F0A45F2A45003F5C042184410B50C4635
:105AB00091ED006A02F5C96102F2A44226EE676A1E
:105AC00093EDD41A91ED007A03F5A043D2ED006A6C
:105AD000B7EEC77A93F8183526EE266A66EEA00A66
:105AE00013F00C0F9FED0A5BB7EEC66A14BF0121DD
:105AF000002127EE057BA6EE057BB7EEC70BC9F0AC
:105B000041F9DFED077A20EE270A84ED000A10BD87
:105B1000000000A046DF913F0AD7233C35FA8E3CB7
:105B20000000C84200F5A04090F9C40AA0F10300AB
:105B3000B0FA80F04009704770B5044684B00D4655
:105B400004F51256684612F07FF8304608F058FD0A
:105B500018B90025284604B070BD694630460AF0E1
:105B600059F80028F5D023682A4669462046D3F81C
:105B7000B030984705460028EBD045F610200121AB
:105B80002044CCF0A7FAE5E7F0B5044687B000F56D
:105B900012500F46164609F073FC054670B386BBDB
:105BA00049F29050204436F063F997ED015A97ED91
:105BB000036A48F6742097ED027AB8EEC55AB8EE3B
:105BC000C66ADFED147AB8EEC77ADFED136A134ABE
:105BD000062125EE265A204426EE276A27EE277A4C
:105BE000B7EEC55AB7EEC66AB7EEC77A8DED045B5D
:105BF0008DED026B8DED007B70F0C0FC284607B088
:105C0000F0BD04F5005292F8FC3643F0020382F82E
:105C1000FC36C5E795BFD6330AD7233CD4441708D2
:105C200070B500F5005584B095F8FC369A0701D59B
:105C300004B070BD00F512560446684612F004F830
:105C40006946304609F0E6FF0028F1D004F5F4601B
:105C50000CF070FC95F8FC36DB070BD506F51B71D4
:105C6000684612F0DDF9B6EE007BB4EEC70BF1EE3C
:105C700010FADDD46946304609F002FC04B070BD6C
:105C800070B547F2C435044605442846C2F0D6FF35
:105C900000285AD004F5804696F95533002B54D08D
:105CA00004F50043D3F8F40D0368DB689847002837
:105CB00046D004F5C04393F9A834002B49D007EE31
:105CC000903A04F51252B8EEE77B92ED826A9FEDAE
:105CD000445BB0EEC66A27EE057BB7EEC66AB4EE4B
:105CE000C76BF1EE10FA0ADC92ED816AB0EEC66A7B
:105CF000B7EEC66AB4EEC76BF1EE10FA29DD2046A6
:105D0000FFF710FF18B9384A1388013313806CF07D
:105D100091FE01220C216CF0AFFB2046FFF702FF41
:105D200000284AD048F67420304A0021204470F000
:105D300025FC284601220C21BDE87040FCF746BA3C
:105D40002046FFF7EFFE0028B3D1274B00221A8030
:105D500070BD2046FFF7E6FE0028F9D142F6840325
:105D6000DFED237A04F50052234493ED007AB4EE7C
:105D7000E77AF1EE10FAE8DA02F2947292ED027A22
:105D8000B0EEC77AB4EEE77AF1EE10FADDDA45F25A
:105D90001853B1EE047A2344D3ED0A7AF0EEE77A91
:105DA000F4EEC77AF1EE10FACFD40F4A138801331C
:105DB0009BB2132B1380AAD870BD014648F67420FD
:105DC0000C4A204470F0DAFB49F238411322204695
:105DD000214406F095F996F95533022BA9D070BDF0
:105DE000000000A046DF913F38C90024F4441708A2
:105DF0000AD7A33D084517082DE9F04104462DEDCB
:105E0000028B88B06CF016FE8046D2F05FFF04F57E
:105E10001043064649F67020D3F8887A0D46204490
:105E2000003F18BF01276FF0BBFD90ED008A49F6D7
:105E30007C202044B7EEC88A6FF0B2FD03460B4ABF
:105E4000404693ED007A0A49B7EEC77A094B0297AC
:105E50008DED048BCDE900658DED067B6CF060F96E
:105E600008B0BDEC028BBDE8F08100BF28451708E3
:105E7000444517082045170810B5044647F2C430BA
:105E800082B02044C2F0DAFE30B145F2A450694637
:105E90002044C9F019F968B904F51043002148F607
:105EA0007420184AC3F8881A0221204470F066FB57
:105EB00002B010BD49F67020694620446FF072FDB3
:105EC00045F2185349F67C2001A9234420449B6ADB
:105ED00001936FF067FDD2F0F1FE04F51043014627
:105EE00000222046C3F8881AC3F88C2AFFF784FFE3
:105EF00048F67420044A0221204470F03FFB02B0AF
:105F000010BD00BF4C4517086845170810B504467A
:105F100049F67C202DED028B204484B06FF040FDCB
:105F2000034649F6702093ED008A20446FF038FD57
:105F3000B2EE047AD0ED007AB4EEC78ACDED037AE2
:105F4000F1EE10FA06DB9FED237AB4EEC78AF1EE8C
:105F500010FA12D948F674201F4A0221204470F02A
:105F60000DFB04F5104300222046C3F8882AFFF7F2
:105F700043FF04B0BDEC028B10BD9FED187AF4EE28
:105F8000C77AF1EE10FAE5DBFDEEC87A44F246304E
:105F90000DF10B01204417EE903A8DF80B3060F0B4
:105FA0007BF944F2383003A9204460F00BF904F582
:105FB000804348F674200A4A93EDCE7A022193F981
:105FC00046332044B7EEC77A8DED007B70F0D6FAE9
:105FD000C7E700BF0000C842A4451708000000340E
:105FE0008045170870B500F5104584B0D5F8883A9B
:105FF0000BB904B070BD044645F2A45001A9204479
:10600000C9F062F80028F4D049F67020194E01A9B1
:1060100003AA204403966FF057FD45F2185349F642
:106020007C2003AA234402A9204403969B6A02937E
:106030006FF04AFDD5F88C3A0F4A03FB02F2B2F139
:10604000333F10D90133C5F88C3AD2F037FED5F87A
:10605000883AC01AB0F5FA6FCBD3002BC9D02046CE
:10606000FFF754FFC5E72046FFF7C6FED5F88C3A88
:10607000E8E700BF0AD7A33CCDCCCCCC10B5044692
:1060800082B000F5125008F0BBFA08B902B010BD9A
:1060900001A9144808F0E8FB47F2C4302044C2F0DC
:1060A000CDFD9DF8043080B9DC06C3F30010EDD4BB
:1060B0009DF805209107C2F34000E7D41C07C3F305
:1060C000C000E3D402F00100E0E7D90604D583F074
:1060D0008000C00902B010BD1A07C3F3C000D5D5B7
:1060E000F5E700BF2053002430B58BB000220446F2
:1060F00000F5125007AD06A905AB07920892099268
:1061000003AACDE9005104A909F04CFA284634F05D
:1061100063FE04F580439DED047AD3EDD67ADDED80
:10612000036AB4EEE70AF1EE10FAF4EEC77AACBFF8
:1061300001230023F1EE10FAF4EEE67A98BF013362
:10614000F1EE10FA01D80133DBB204F5E042D2F8E7
:106150002814A1B192F82C24D20710D5F4EEC77AF6
:10616000F1EE10FA01D80133DBB2012B0ED8204634
:10617000FFF784FF80F00100C0B20BB030BD77EEB6
:10618000A76AB4EEE67AF1EE10FAE7DB01200BB075
:1061900030BD00BF70B500F5004595F80C3E03B169
:1061A00070BD0126044685F80C6E6CF043FC324647
:1061B00011216CF061F9D5F8F40D03685B6A98471A
:1061C0000028EDD004F5804393F95633002BE7D037
:1061D000022B06D049F2384106222046214405F020
:1061E0008FFF48F67420034A02212044BDE8704026
:1061F00070F0C4B968E7160870B584B00446684604
:1062000011F022FD694604F5125009F031FD08B97C
:1062100004B070BD47F2C4302044C2F00FFDE8B1B5
:1062200004F58043D3EDD67AF5EEC07AF1EE10FA9C
:1062300014D92046FFF758FF054680B3424D6B78CE
:1062400003F00102DB0705D42B780133DBB2092B05
:1062500052D82B703D4BDA7304B070BD3A4904F547
:1062600000423A4800250B88C57323F4FF7323F0DE
:1062700001030B8092F80C3E002BC9D082F80C5E13
:106280006CF0D8FB2A4611216CF0F6F848F6742021
:106290002F4A0221204470F071F904B070BD2A4EDB
:1062A00033782BB3013B33703388C3F30803B3F562
:1062B000807F73781DD160F3000373706CF0BAFBBC
:1062C0002A4610216CF0D8F804F5004393F80C2E00
:1062D00072B183F80C5E6CF0ADFB2A4611216CF0B4
:1062E000CBF848F674201A4A0221204470F046F98F
:1062F000737803F00102ADE72B8823F4FF7323F0DA
:10630000010343F485732B806CF094FB022210216F
:106310006CF0B2F8D2F0D2FC6A6847F23053801ABF
:10632000984206D82046FFF735FF6B7803F001024C
:1063300090E748F67420074A0221204470F01EF9C5
:10634000D2F0BCFC6860EDE73CC90024F0CA002430
:10635000BC451708D445170838B50446D2F0A4FC4C
:106360000E4BB4F8F6221988914203D00C491A80DA
:10637000086038BD0A4B0B4A1B68C31A9342F8D910
:1063800047F2C4352819C2F059FC0028F1D0281969
:1063900001220621BDE83840FBF718BF44C900249C
:1063A00048C90024400D03002DE9F04700F50044E2
:1063B0000F460646904694F8FC1D002B61D041EA3A
:1063C000070584F8FC5D71B93DB994F8043E002BD3
:1063D0005AD184F8045EBDE8F087D2F06FFC94F8DF
:1063E000FC5DC4F8000E94F8040E08B1002D4BD0EB
:1063F000284084F8040E002DEDD00028EBD1D2F017
:106400005DFCD4F8003E06F58045DFED4C6AC01A0D
:1064100095EDD37A07EE900A27EE267AF8EE677AA2
:10642000F4EEC77AF1EE10FAD5DD49F61419D4F876
:10643000F43DB1444B45CED049F2384AB2445345BD
:1064400034D0434648F6742894F8FC2D0421B04417
:1064500084F8042E40463A4A70F090F87BF06CF9CC
:1064600049F25853D4F8F42D33449A4251D095F957
:106470004833013B042BAED8DFE803F028301F403F
:10648000370021EA07059CE748F6742043462D4A69
:106490000621304470F072F894F8040E94F8FC5D14
:1064A000284084F8040E002DA7D194E706F5E043B8
:1064B000D3F88030DB078ED5C3E749F65011192297
:1064C0003046314405F01CFE002884D1192249468B
:1064D000304605F015FE00287FF47DAF514630466A
:1064E0001922BDE8F04705F00BBE47F2C430012287
:1064F00014213044BDE8F047FBF768BE49F650115F
:1065000019223046314405F0FBFD00287FF463AFCB
:10651000E4E7012F0CD0022FA9D195F95433022BB7
:10652000A5D14046084A0421BDE8F04770F026B8DE
:1065300095F95033022B9AD1F3E700BF00007A445B
:10654000F8451708E445170804461708013A10B53E
:106550000446042A1CD8DFE802F00A1203251C00B6
:1065600049F650110422014405F0CAFD80B949F6EC
:10657000141104222046214405F0C2FD40B949F21D
:106580003841204604222144BDE8104005F0B8BD42
:1065900010BD47F2C430012207212044BDE810405D
:1065A000FBF714BE49F65011E3E700BF2DE9F843AD
:1065B00043F69C6647F2C43800F540570021064474
:1065C0008044044697F8D89E304699F041FE05462F
:1065D0004046C2F033FB70B155B197F9A23E63B9A2
:1065E0006CF028FA2A460921BDE8F8436BF044BF55
:1065F000B9F1000FF4D1BDE8F8833046294699F08F
:10660000B1FEDFED1A7AB4EEE70AF1EE10FA1BD80C
:1066100097F9A23E013B042BE2D8DFE803F00C150A
:1066200003231D0049F650110A222046214405F09B
:1066300067FD0028D4D149F614110A2220462144CE
:1066400005F05EFD0028CBD149F238410A222046F0
:10665000214405F055FDC3E701220F214046FBF719
:10666000B5FDBDE749F65011E7E700BF0000C8429D
:1066700001207047002070470120704701207047BB
:1066800010B503680446DB68984750B1E26842F6EB
:106690009C23DFED057A134493ED000A20EE270AD0
:1066A00010BD9FED020A10BD0AD7233C0000000078
:1066B00010B503680446DB68984750B1E26842F6BB
:1066C0009823DFED057A134493ED000A20EE270AA4
:1066D00010BD9FED020A10BD0AD7233C0000000048
:1066E00010B503680446DB68984730B1E26842F6AB
:1066F000A023134493ED000A10BD9FED010A10BDC5
:106700000000000010B503680446DB68984730B10C
:10671000E26842F69423134493ED000A10BD9FED06
:10672000010A10BD0000000010B503680446DB68D4
:10673000984700B910BDE36842F61430BDE8104038
:10674000184405F073B800BF70B5624E84B00D46B2
:106750000446D6EDD40A806A8DED010AC8F0F4FE35
:106760008DED010A002D4FD1E368002103F50052A1
:10677000039192F9142B002A3FDCF0EEC07A9FEDD2
:10678000567AF4EEC77AF1EE10FA5CD403F5805332
:10679000A06A93F8B0315A072DD490F868131B07FC
:1067A000A3689FED4E1AD3ED040A48BF012293F966
:1067B0001E3058BF90F8682307EE903AD6EDD41AF1
:1067C000F8EEE77A27EE811AC8F032FFDFED447A5F
:1067D00020EE270A8DED030A3E48FFF7A3F90028B3
:1067E00039D1E36841F2B0109DED030A1844CDF0B1
:1067F000FFFC04B070BD0121D1E742F6143003A9BB
:10680000184404F0B9FEECE7E368A06A03F5045508
:10681000C8F064FEF6EE000A63682846D6EDD41A86
:1068200093ED831A01A960EE200A9FED2E0A9EF0D7
:1068300053F9E36842F61430184404F0A5FC78B923
:106840009DED010A90E72348FFF76CF9F0B1E3688A
:106850009DED010A9AE703A91E48FFF71DF9C0E75D
:10686000E568D2F02BFA05F50055D5F82831C01AA5
:10687000B0F5FA7FE4D206F500421B4BD2F8F40DD6
:106880009842DDD003685B6D9847D9E7D4E90212DE
:10689000DFED120A0DF10B0391F91E0002F5805293
:1068A00091ED040A07EE900A92F8B01196EDD41A11
:1068B000F8EEE77AC1F3C002A06AC1F3800167EE87
:1068C000A00AC8F075FFDFED067A20EE270A8DEDED
:1068D000030A81E7A02E0024000000340AD7233CDD
:1068E0000000C8420000000048C3002470B52DED30
:1068F000028B90F91F300D461446012B22D0032B3A
:106900002E4B43D0D3F84423FFEE007AB7EE007A43
:10691000B2F9082006EE902A002AF8EEE66A27FE71
:10692000277AC4ED006AD3F84033B3F9083007EE94
:10693000903AF8EEE77ABDEC028B67EE877AC1ED0C
:10694000007A70BD1D4ED6F840037BF0A9F9B0EE79
:10695000408AD6F844037BF0A3F9B6EE007A78EECD
:10696000007A9FED176A38EE408ADFED166A67EE0F
:10697000877A28EE078A67EE867A28EE268AC4EDA3
:10698000007A85ED008ABDEC028B70BDD3F84423FC
:10699000B2F9082007EE902AF8EEE77AC4ED007A03
:1069A000D3F84033B3F9083007EE903AF8EEE77ABF
:1069B000BDEC028BC1ED007A70BD00BFA09E00242B
:1069C0000000C84200A08C450C4A0D4910B40D4C83
:1069D000C0E900420C4A0D4CC0E902120C4A0D49B4
:1069E000C0E9044208321034C0E906120C310A4AE8
:1069F000C0E9084182625DF8044B704720530024CF
:106A0000C87100242C46170808720024E0A1002455
:106A1000E4A10024E8A10024448400240368DB6D81
:106A2000184700BF204B1B6830B5DB6A83B00446B3
:106A300093F89C3093B9236820469B6D9847054690
:106A400048B1236820461B6D9847E36842F614302E
:106A5000184404F01DFF284603B030BD01A91348B7
:106A600007F002FF1248FFF709FB60B1114B93F8E2
:106A70000C3E43B9236820465B6A9847236820464A
:106A80009B6A9847D7E7236820465B6A984748B9CE
:106A9000236820469B6A98470028CCD09DF8043094
:106AA0009B07C8D40025D6E7982E00242053002445
:106AB000A02E0024A0AE0024434B70B52DED028B18
:106AC00093F8FC3D05460E461446DB073AD4806831
:106AD000FFF70CFFEB6841F2B0101844CDF02AFC30
:106AE00000283AD194ED000AEB6841F2B010374A21
:106AF0001844D2EDD40ACDF005FCDFED357A94EDE3
:106B0000007AB4EEE77AF1EE10FAB4EEE70A94BF39
:106B100001220022F1EE10FA94BF012300239A42D1
:106B20000BD0AB6893F91F3033F0020305D1D6EDDB
:106B3000007AF1EE677AC6ED007A84ED000ABDECCA
:106B4000028B70BD002341F2B0100B601360EB6844
:106B50001844CDF0EFFB0028C4D0DFED1E7AB7EE6D
:106B6000001A96ED000AFFEE000A722080EE270A56
:106B70002EF00CF9DFED187A7320B0EE408A94ED18
:106B8000000AB7EE001A20EE270AFFEE000A2EF0E8
:106B9000FDF8B0EEC88AB0EEC00AB7EE007A78EE23
:106BA000007AF4EEC77AF1EE10FA9BDDD6ED006ABA
:106BB00086EEA77A86ED007A94ED007A87EE270AB2
:106BC00084ED000A90E700BFA0AE0024A02E0024B0
:106BD000000000B400A08C450AD7233C444B70B59C
:106BE0002DED028B93F8FC3D82B004460E46DB0788
:106BF00015466FD401AA8068FFF778FE9FED3D8AA5
:106C00009DED010A20EE088AA368B7EE007ADFED59
:106C1000396A93F91E2093ED040A07EE902AF8EEE4
:106C2000E77A67EEA67AF4EEC77AF1EE10FA3ADD6B
:106C3000B3EE0E1A40F27D10DFED2F0A2EF0A6F80B
:106C400020EE080A2D4B41F23C2085ED000AD3EDE1
:106C5000D40AE3681844C8F077FCDFED297A95ED93
:106C6000007AB4EEE77AF1EE10FAB4EEE70A94BFD8
:106C700001220022F1EE10FA94BF012300239A4270
:106C80000BD0A36893F91F3033F0020305D1D6ED82
:106C9000007AF1EE677AC6ED007A85ED000A02B05F
:106CA000BDEC028B70BDDFED176AF4EEE67AF1EE13
:106CB00010FABDD4E26842F610539FED136A1344F4
:106CC000D3ED006AF4EEC66AF1EE10FA0BDBB0EE1B
:106CD000660AADE7DFED087AB0EE678AC1ED007AAB
:106CE000CDED017A90E7C7EE276A20EE260A9FE7EE
:106CF000A0AE00240AD7233C00000000A02E0024F0
:106D0000000000B4CDCC4C3D000000340B4B93F898
:106D1000FC2DD2070DD4A3F58053D3F8483343B1EB
:106D2000B3F9083007EE903AF8EEE77AC1ED007A51
:106D30007047DFED037AC1ED007A7047A0AE002402
:106D400000000000F8B5464F04460E461546D7F839
:106D500040032DED028B7AF0A3FFB7EE001AFFEE91
:106D6000000AA6202EF012F8D7F84403B0EE408AAD
:106D70007AF096FFB7EE001AA720FFEE000A2EF079
:106D800005F8A368F0EE408A93F91F30012B09D172
:106D9000F6EE007A78EE008A38EE407A68EEA78A3E
:106DA00027EE278AF0EE680AB0EE480A40F176F83E
:106DB000DFED2C7A20EE270A2DF080FF28EE088ADE
:106DC00086ED000AB0EE480AA8EEA80A2DF066FE8D
:106DD000A368B7EE007ADFED246A93F91E20B0EEC7
:106DE000408A93ED040A07EE902AB4EEC78AF8EEC3
:106DF000E77AF1EE10FA67EEA67A58BFB0EE478A4E
:106E0000F4EEC77AF1EE10FA0EDDB3EE0E1A40F290
:106E10007D10DFED160A2DF0B9FF28EE000A85ED92
:106E2000000ABDEC028BF8BDDFED116AF4EEE67AE4
:106E3000F1EE10FAE9D4E26842F610539FED0D6AC4
:106E40001344D3ED006AF4EEC66AF1EE10FA02DBE9
:106E5000B0EE660AD9E7C7EE276A20EE260AD4E725
:106E6000A09E0024A00CB3450AD7233C00000000DC
:106E7000CDCC4C3D0000003470B5C36904460D46CE
:106E80001646186858B17AF0BDFE85ED000A236AEF
:106E9000186850B17AF0B6FE86ED000A70BD002386
:106EA0000B60236A18680028F4D10023336070BD9A
:106EB00010B5436A0C46186820B17AF0A3FE84ED41
:106EC000000A10BD00230B6010BD00BFC36861B194
:106ED00041F25872DFED077A1A4492ED000AB4EEDF
:106EE000E70AF1EE10FA00DB704703F5005393ED6B
:106EF000BB0A704700000034C36803F5005383F8F1
:106F0000791A704730B5444D83B0002304462846B3
:106F10008DF80330FEF706FE002844D09FED3F1A9F
:106F2000A06AD5EDD41A9FED3E0AD4E9022392F966
:106F30001E1003F58053D2ED040A07EE901A93F861
:106F4000B021F8EEE77AC2F38001C2F3C00227EE67
:106F5000811AC8F06DFBDFED337A01A9284620EED7
:106F6000270A8DED010AFEF797FDE36842F614301B
:106F7000184404F0E3FAE36841F2B0109DED010A11
:106F80001844CDF035F99DF8033083B39FED240A02
:106F9000E36841F2B01001211844CDF023F99DF8C7
:106FA000030003B030BDD4E90212DFED1C0A0DF17D
:106FB000030391F91E0002F5805291ED040A07EED9
:106FC000900A92F8B01195EDD41AF8EEE77AC1F371
:106FD000C002A06AC1F3800167EEA00AC8F0E8FB16
:106FE000DFED107A20EE270A8DED010ABDE7E36898
:106FF000D5EDD40A03F580539FED090AA06A93F8F2
:10700000B011C1F3400201F00101C8F0DFF8DFED7B
:10701000067A20EE270ABBE7A02E00240AD7233CDD
:10702000000000000000C84200A08C4530B50446B6
:107030002DED028B8068B0EE408A83B090F91E205F
:10704000531FDBB25F2B05D9B0EE480A03B0BDEC8D
:10705000028B30BD3D4B0D4693F8FC3DDB0763D4FE
:1070600001AA6946FFF742FCDFED398A9DED010A6E
:10707000A06860EE288A90F91E2007EE902ADFEDC6
:10708000346AB7EE007A90ED040AF8EEE77A67EE1C
:10709000A67AF4EEC77AF1EE10FA2EDDB3EE0E1AF0
:1070A00040F27D10DFED2B0A2DF070FE20EE280A55
:1070B000DFED297AB4EEE70AF1EE10FA0EDB002DCF
:1070C000C2D1DFED267AB4EEE70AF1EE10FABBD9B1
:1070D000B4EEC80AF1EE10FAB6D4B7E7DFED1F7AC6
:1070E000B4EEE70AF1EE10FA27D8002DACD0B4EEDA
:1070F000C80AF1EE10FAA7DCA8E7DFED196AF4EE92
:10710000E67AF1EE10FAC9D4E26842F610539FED28
:10711000126A1344D3ED006AF4EEC66AF1EE10FA77
:107120000EDBB0EE660AB9E7DFED0A7AF0EE678AA9
:10713000CDED007ACDED017A9FE7002DC8D0D6E7DE
:10714000C7EE276A20EE260AA8E700BFA0AE0024FB
:107150000AD7233C0000000000000034000000B407
:10716000CDCC4C3D10B52DED028B03680446B0EE3E
:10717000408ADB689847E36828B103F5005292F92A
:10718000E422002A0BDCB0EE480A41F2B0100121E3
:107190001844BDEC028BBDE81040CDF023B8BDEE25
:1071A000C80A2369186810EE103A1BB200EE103AB4
:1071B000B8EEC00A7AF0C0FEE368B0EE408AE2E7BB
:1071C0000C4B10B5D3EDD40A0446C368806A03F5AE
:1071D000805393F8B011C1F3400201F00101C7F0F0
:1071E000F5FFDFED057A204620EE270ABDE81040C6
:1071F000FFF7B8BFA02E002400A08C4510B5C368CF
:1072000004469FED107A03F58053DFED0F7A20EEF0
:10721000070A0E4A93F8B01160EEA70A806A20EEC2
:10722000270A92EDD41AC1F3400201F00101C8F01F
:10723000F9F8DFED077A204620EE270ABDE8104076
:10724000FFF790BF0AD7233C35FA8E3CA02E0024CE
:1072500000A08C4510B5836A0446DFED187A93EDE3
:10726000C21AB4EEE71AF1EE10FA21DDDFED147A5E
:1072700021EE271AF1EE410A4FF4F2702DF086FD4F
:10728000E368104A03F58053A06AD2EDD40A93F85C
:10729000B011C1F3400201F00101C8F0DBF8DFEDED
:1072A0000A7A204620EE270ABDE81040FFF75ABFB1
:1072B0009FED061ADFED060ADEE700BFCDCCCC3D20
:1072C0000AE81C41A02E002400A08C45DD0C7B3F69
:1072D000DD0C7BBF034610290AD8DFE801F00B0F55
:1072E0000913171B1F23272C30343809093C400091
:1072F0000020704749F270401844704749F2A84096
:107300001844704749F6D8001844704749F238408D
:107310001844704749F68C001844704749F68C10A1
:107320001844704749F6C8101844704700F5C0402B
:10733000D0F86404704747F298201844704749F227
:1073400058501844704749F614101844704749F6CD
:1073500050101844704749F2E0401844704700F557
:107360001440704782B030B583B08E46C56804467D
:1073700006A90DF1200C81E80C009CE8030006AB87
:107380008DE8030042F2E82071460CCB2844C9F096
:1073900017FF40B1E16842F6A42300220B441B68AA
:1073A00084F83020E36203B0BDE8304002B070479B
:1073B00070B52DED028BC36882B0044603F5005210
:1073C00003F52A5392F8791A93ED000A09B1B1EE48
:1073D000400A204642F2E825FFF728FEE068B0EEBA
:1073E000C00A554E2844C8F091FFE06896EDD40AD3
:1073F0002844C9F001FFE26842F6A42342F61430A3
:10740000134410441B68E36203F0BEFE002867D1FA
:10741000E16842F68C23226820460B44002142F6A4
:10742000143593ED000A136E9847E36842F2E820A2
:107430001844C9F073FEE068B0EE408A284404F0B6
:1074400063FAC0B1E068B0EE480A284404F0C8FA14
:10745000E0688DED010A284404F026FA9DED010A4A
:10746000A0BBDFED360A204602B0BDEC028BBDE8C2
:107470007040FFF7C3BEE56805F5005505F52963C3
:1074800093ED008AD1F01AFCD5F82831C01AB0F576
:10749000FA7FA06A37D3E368B0EE480AD6EDD40A83
:1074A00003F5805393F8B011C1F3400201F00101DC
:1074B000C7F08CFEDFED227A204620EE270A02B0CC
:1074C000BDEC028BBDE87040FFF74CBEE36803F5EE
:1074D0000053B3F9F63200EE903AF8EEE00AC2E754
:1074E000E568D1F0EBFB05F50055D5F82831C01A59
:1074F000B0F5FA7F8CD206F50043D3F8F40D03689B
:107500005B6D984784E7C8F007F8A06AB0EEC00A40
:10751000D0EDBF7AF5EEC07AF1EE10FAD8BFDFED0C
:10752000077AB4EE670ADFED057AF1EE10FA98BF3C
:10753000B0EE678AAFE700BFA02E00240000000075
:1075400000A08C45012070470048704790461708FE
:107550000120704700207047F0B585B00446806A6E
:1075600001A9C7F0B1FD002848D1474D204602A926
:1075700003AAFFF7A1FA2846FEF7D4FA002877D12C
:10758000E36841F2B0109DED030A1844CCF030FEE0
:10759000DDED027A9FED3D7AF0EEE77AF4EEC77A00
:1075A000F1EE10FA5DD5E06842F61436304404F08E
:1075B0007BF988B3E068A76A304404F001F9E36816
:1075C00095EDD41A384603F5805203F50053B3F90C
:1075D000F63292F8B01100EE903AC1F3400201F099
:1075E0000101F8EEE00AC7F01DFFDFED297A204621
:1075F00020EE270AFFF7B6FD05B0F0BD02A9204630
:1076000003AA214DFFF7EAFA236801219DED030A41
:107610001B6E20469847BBE7DDED026ADFED1C7A62
:10762000E36886EEA77AD5EDD40A03F58053A06A05
:1076300003F2A46293F8B01192ED006AC1F3400224
:1076400001F00101B7EEC66A9FED0D5B26EE056BFA
:10765000B7EEC77A27EE067BB7EEC70BC7F0B6FDCD
:10766000C3E7E36842F61430184404F011F99AE7CE
:1076700003A92846FEF710FA82E700BFAFF30080A7
:10768000000000A046DF913FA02E0024000000343F
:1076900000A08C4508B5034641F2B010DB681844E1
:1076A000CCF048FE80F00100C0B208BD034642F6AF
:1076B0001430DB68184404F02BB800BF0A20704770
:1076C00000487047044717080120704790F884026B
:1076D00000F0FD00A0F10400B0FA80F0400970470E
:1076E00090F83C30012B00D07047383034F074B83B
:1076F00010B5B0F86C30012B23D9C368044642F2B0
:10770000E8209FED140A1844C9F08AFB00231248B0
:1077100084F8863202F0B8FA104804F0E3FE38B973
:10772000052384F884320123184684F8853210BD7D
:107730000B48FFF777F90028F2D0032384F884324E
:10774000F1E778F081FD074A05216EF017FF002070
:1077500010BD00BF0000000080C30024A02E002444
:107760002CC700240C47170890F9702012B190F82C
:10777000711001B17047FFF7BFBB00BF30B50446C1
:1077800085B0D1F09BFAD4F8AC321BB1C31AB3F573
:107790007A7F0DD90DF10F01C4F8AC020DF10E0383
:1077A0000DF10D0200911221124871F0A9F908B9EA
:1077B00005B030BD78F048FD02680F4D12699DF8A4
:1077C0000F10AA4211D190F8D0208A420FD900EBB5
:1077D0008103D3F8D40004F526739DF80E209DF89C
:1077E0000D1076F0E1FD05B030BD9047F3E70020C5
:1077F000F1E700BF40CF0024E1220208844690F860
:107800008402062801D000207047BCF8C20208801C
:1078100001209CF8C8121170DCF8CC221A60009A82
:10782000DCF8D0321360019ABCF9D4321380029A8A
:10783000BCF9D6321380704790F88432062B00D002
:107840007047B0F8C2328B42FAD1012380F8C032BF
:10785000704700BF30B52DED028B90F8865283B093
:1078600004469DB1836893F915104B1C04D128463A
:1078700003B0BDEC028B30BDC9B2354804F014FE34
:10788000012859D094F88632002BF0D1A36893F9DF
:1078900015104A1C26D0C9B22D4804F005FEA8B325
:1078A000A36893ED067AF0EEC77ADFED2A6AF4EE6C
:1078B000E67AF1EE10FA0FD4274B93F89524A3F54E
:1078C0005E7302EB420203EB820393ED9E8AB4EEF9
:1078D000C78AF1EE10FA20DA0025284603B0BDEC85
:1078E000028B30BD93ED067ADFED1A6AF0EEC77AAF
:1078F000F4EEE67AF1EE10FAD7D501231D4684F8AE
:107900008632284603B0BDEC028B30BD78F09CFC7B
:10791000124A04216EF032FEEFE778F095FCB7EEE4
:10792000C88A0F4A04218DED008B6EF027FE0123DB
:107930001D4684F886329AE778F086FC094A0421CD
:107940006EF01CFE00231D4684F886328FE700BFD0
:10795000A02E002400000034A03E00243C4717085D
:10796000544717082847170838B5054610480C46ED
:10797000FFF758F800B938BD04230D4885F8843264
:1079800002F088F9A3680BB9E3686BB105F5267CB2
:1079900094E80F008CE80F000649604610F0A2FF43
:1079A000012385F8A83238BD85F8A83238BD00BF5C
:1079B00080C300247CBB00241A4A10B51378044607
:1079C00043F08003137078F03FFC174A05216EF0F6
:1079D000D5FDE36803F5005393F9DC32022B07D0A1
:1079E000032B16D0012B0BD0052384F8843210BD55
:1079F00008220E490E4804F083FB0028F4D010BD85
:107A00000C48FFF70FF80028EED0032384F88432E7
:107A100010BD08220849064804F072FB0028E3D094
:107A200010BD00BF10CB00247047170848C30024C6
:107A3000A02E00242CC7002410C3002430B583B02E
:107A400004460D46D1F03AF903462248C4F8BC3248
:107A500004F048FD00BB052384F88432D5ED027A9A
:107A6000F5EEC07AF1EE10FA25DD9FED1B7A67EE98
:107A7000877AFCEEE77AC4EDAE7A78F0E5FBD4F8CD
:107A8000B832164C0621164AA4FB0343CB4003B080
:107A9000BDE830406EF072BD1248FEF7C3FF00280B
:107AA000D9D0032384F88432D5ED027AF5EEC07A7A
:107AB000F1EE10FAD9DC97F0A5FC002295F90E3012
:107AC000009295F90D2095F90C1097F08DFBC4F8F4
:107AD000B802D2E7A02E002400007A44D34D6210F1
:107AE000844717082CC7002438B50B7C0D46044684
:107AF0002DED028BFBB991ED028A9FED170A28EE5E
:107B0000008AE36840F22F3095ED030A03F5005335
:107B100093EDBB1AF1EE410A2DF038F90022012352
:107B200084EDA20A84ED0D8A84F88C2284F88432D4
:107B3000BDEC028B38BD436891ED027A93ED800A6B
:107B4000DFED057AB8EEC00AA7EE270A2DF06CF833
:107B5000B0EE408AD5E700BF0000C84270B50368A8
:107B600082B004460E469B6C98470546C8B194F80F
:107B700094329BB90122B4F88E3284F894222BB34C
:107B800078F062FBB4F88E22338806210092154A01
:107B90006EF0F4FCD1F092F8C4F89002B4F88E3292
:107BA00013B9284602B070BDD1F088F8D4F890120D
:107BB0000D4A401AB4F88E32A2FB0020B3EB901F9E
:107BC00094BF01250025284602B070BD78F03CFB2B
:107BD0003388064A06216EF0D1FCB4F88E32002BB1
:107BE000DFD0E1E794471708D34D6210C04717086C
:107BF00090F88432042B01D0012070478B88002B31
:107C0000FAD010B590F8A832044693B100F5267169
:107C10000A4810F005FAE36803F5005393EDBC7AC7
:107C2000B7EEC77AB4EEC70BF1EE10FA01D8012017
:107C300010BD0348BDE8104002F03AB87CBB0024F8
:107C400080C3002470B501F1080384B00C460646D9
:107C50006D460FCB85E80F001249284610F042FE12
:107C60006288A388122A4FEA132313D0227A07EEE0
:107C7000903AF46842F63070B8EE670AC2F34002F8
:107C80002946204401F056FA10B1072386F88432C1
:107C900004B070BD227ED207E8D503EB83035B00FE
:107CA000E4E700BF7CBB002410B5036882B0D1F8C4
:107CB00009200C46DB6C00EE102A984708B902B088
:107CC00010BD78F0C1FAD4F80930064A062107EE53
:107CD000103AB7EEC77A8DED007B6EF04FFC02B024
:107CE00010BD00BFF047170838B5044619480D46C7
:107CF000FEF798FE18B9012384F8C03238BDB4F8F5
:107D0000C23206210022013384F8841284F8C02292
:107D1000A4F8C232D0F0D2FF034605F10A00C4F83D
:107D2000C4322B7A84F8C8326B7A84F8C93210F0E6
:107D30004DFF05F10C0084EDB30A10F047FF84ED10
:107D4000B40AB5F90E30A4F8D432B5F91030A4F85D
:107D5000D63238BD80C3002438B52DED028B0446E1
:107D6000B0EE408A0D46FFF775FD48B1B0EE480A07
:107D700029462046BDEC028BBDE83840FEF7E4BC46
:107D8000BDEC028B2046BDE83840FFF7BBB800BF12
:107D9000874B1B6830B52DED028BDB6A85B004463E
:107DA00093F89C301BB9B0F86C30012B14D994F8BF
:107DB0008532C3B168460FF047FF6946606807F037
:107DC00057FF70BB94F88432072B73D8DFE803F0B9
:107DD0005676B84E1B3B2143052380F8843294F835
:107DE0008532002BE6D104F5367033F0FFFB20B16D
:107DF00094F83C30012B00F0AB8004F138052846A4
:107E000036F014FADEE794F8A83213B12046FFF7F3
:107E1000B5FC684805B0BDEC028BBDE8304001F010
:107E200081BF04F1380036F0C7FC002304F536703A
:107E300084F8853233F0DAFBC4E75F4804F052FB84
:107E4000002840F09F80204605B0BDEC028BBDE8C5
:107E50003040FFF757B8E36842F63070184405B079
:107E6000BDEC028BBDE8304000F040BF534805B088
:107E7000BDEC028BBDE8304002F05CB94E4804F026
:107E800031FB002876D0E36842F2E8201844C9F0BC
:107E900029F900286ED0E36803F5005393F8383AC7
:107EA000002B67D14548FEF7BDFD002862D00323B3
:107EB00084F8843205B0BDEC028B30BD94F88C326E
:107EC000002BBAD1DFED3E0A204694ED0D0AFFF7F4
:107ED00095F994EDA20ADFED3B7A20462368B4EED3
:107EE000E70A1D6EF1EE10FA94BF01210021FFF7A1
:107EF0009DF8354BB0EE408A9D424AD12046FFF7AF
:107F0000A9FC002849D0B0EE480A01212046FEF71E
:107F10001BFC636894ED0D7AD3ED807ADFED2B6A5C
:107F2000F8EEE77A77EE677AF0EEE77AF4EEE67A43
:107F3000F1EE10FA4CBF0123002384F88C32B9E72C
:107F4000234805B0BDEC028BBDE8304002F01CBBFD
:107F500094F88432002B7FF450AF04F138052846A2
:107F600036F00CF9E8B178F06FF91A4A02216EF098
:107F700005FB44E7204605B0BDEC028BBDE8304070
:107F8000FFF716BA0D48FEF74DFD00283FF45BAF32
:107F90008DE701212046A847BBE72046FEF7B2FF48
:107FA000B7E778F051F90C4A02216EF0E7FA26E7BC
:107FB000982E002480C30024A02E00242CC7002467
:107FC00000000000000000B4597D02080000FA43E0
:107FD000B4C70024004817082848170890F88432CE
:107FE000072B24D8DFE803F00D23181B0423040714
:107FF000104801F017BDC36842F63070184400F015
:10800000C3BCC26842F69C23DFED0B7A134493EDA8
:10801000000A20EE270A70470848FEF731BB084BDC
:10802000DFED057A93ED000A20EE270A70479FEDF9
:10803000050A704780C300240AD7233CB4C7002434
:1080400060C700240000000090F88432072B24D879
:10805000DFE803F00D23181B04230407104801F088
:1080600003BDC36842F63070184400F055BCC268C6
:1080700042F69823DFED0B7A134493ED000A20EECD
:10808000270A70470848FEF713BB084BDFED057A57
:1080900093ED000A20EE270A70479FED050A70470E
:1080A00080C300240AD7233CB4C7002460C700243F
:1080B0000000000090F88432072B08D8DFE803F0B6
:1080C000140711070407040A0B4801F0EFBC9FEDE9
:1080D0000B0A7047C26842F63073134493ED260AC8
:1080E00070470748FEF7FCBAC26842F6A023134463
:1080F00093ED000A704700BF80C300240000000019
:10810000B4C7002490F88432072B1BD8DFE803F0B3
:108110000D1A1417041A04070C4801F01DBFC36898
:1081200042F63070184400F0D3BBC26842F6942384
:10813000134493ED000A70470548FEF7E3BA05487B
:10814000FEF7E0BA9FED040A704700BF80C3002429
:10815000B4C700242CC700240000000090F884322B
:10816000072B1AD8DFE803F00E19111504190407BC
:108170000B4801F0ABBCC26842F63073134493ED78
:108180000B0A704790ED0B0A7047064B93ED000AFF
:108190007047054B93ED000A70479FED040A704746
:1081A00080C30024E0C7002458C70024000000005A
:1081B00010B5036804461C4ADB6B934209D190F862
:1081C0008432072B2CD8DFE803F0202B2327152B34
:1081D00015199847D4EDAC7AF8EEE77AB4EEE70AD1
:1081E000F1EE10FA01D4002010BD00230120C4F8E4
:1081F000B03210BD0D4801F069FCEBE7C26842F6F1
:108200003073134493ED0B0AE4E790ED0B0AE1E7BA
:10821000074B93ED000ADDE7064B93ED000AD9E723
:108220009FED050AD6E700BF5D81020880C30024E8
:10823000E0C7002458C700240000000030B54B8878
:1082400083B00446722B0CD85B2B2AD8103B9AB211
:10825000042A5CD8042B5AD8DFE803F064696D8DDA
:108260009500DE2B2ED8B12B51D9B23B2C2B4ED8FA
:10827000DFE803F049494D4D4D4D4D4D4D4D4D4DB0
:108280004D4D4D4D49494D494D4D4D494D4D4D4D2E
:1082900049494D4D4D4D4D454D4D4D4D4D4D4D4D1E
:1082A00049005C3B162B32D8DFE803F07F73313195
:1082B00031313131313131313131313131313131AE
:1082C000843190004AF2CE62934220D190F8C0529D
:1082D00095B990F8C932002B51D0D0F0EFFC4FF493
:1082E0007A75D4F8C42294F8C932801A03FB05F5D4
:1082F000A84294BF00250125284603B030BD94F85C
:108300008432012B67D00125284603B030BD01918E
:1083100077F09AFF01990125344A4B8804216EF0C9
:108320002DF9E9E703B0BDE83040FFF717BC0025A1
:10833000FFF714FCE0E70B7907EE903A0B7E9B0702
:10834000F8EE677A03D59FED2A7A67EE877AE268BE
:1083500042F630739FED276A134493ED247AB0EE12
:10836000C77AC7EE066AF4EEE76AF1EE10FAACBF20
:1083700001250025C0E7FFF7F1FB054670BB00258E
:10838000284603B030BD03689B6C03B0BDE83040A5
:108390001847D0F093FCD4E9AE32801A9842EED957
:1083A00000230125C4F8B832A6E703B0BDE8304089
:1083B000FFF71EBCD0F082FCD4E9AC32801A9842A0
:1083C000DDD900230125C4F8B03295E703B0BDE83C
:1083D0003040FFF7EDBE94F88C528DE777F034FF14
:1083E000054A04216EF0CAF886E700BF5C4817080A
:1083F0000000803BDB0FC940D847170838B50D4651
:10840000FFF71CFF044608B9204638BD77F01CFF73
:10841000298874F035FB204638BD00BF38B590F888
:1084200084320C46072B24D8DFE803F01123191EF1
:10843000042304091548BDE8384001F0A3BDC36812
:1084400042F630701844BDE8384000F049BAC368BD
:1084500003F5005292F8785A75B9284638BD0C4891
:10846000BDE8384002F0DAB80A48BDE8384001F00B
:1084700059BE0025284638BD42F2E8201844C8F00D
:1084800043FE0FC884E80F00E7E700BF80C3002465
:10849000B4C700242CC7002482B08C4610B582B02B
:1084A000044604A906A881E80C0003C804AB8DE8C3
:1084B0000300614620460CCBFEF754FF10B10023A9
:1084C00084F8843202B0BDE8104002B0704700BFAB
:1084D0002DE9F04101F1080396B004460E4603ADC4
:1084E00017460FCB85E80F004249284610F0FAF9ED
:1084F000B6F904300022002BC4F8902223EAE3727C
:10850000A4F88E2227DD11A80FF09EFB07AE23688A
:1085100030465F6C0FF098FB374B9F4251D10DF105
:108520002C0C0DAF96E80F008CE80F0097E80300C5
:108530008DE80300294620469CE80C00FEF712FF58
:1085400030B1002384F884320023012084F894326F
:1085500016B0BDE8F0810DF1440840460FF074FB01
:10856000002FD3D131880FAA04F13800013189B22C
:1085700035F068F80028C9D007AE98E80F0086E803
:108580000F002946304610F0ADF92368D3F8448037
:10859000194B984521D10DF12C0C0DF1340E96E8B4
:1085A0000F008CE80F009EE803008DE803002946C9
:1085B00020469CE80C00FEF7D5FEC8B184F8847212
:1085C000C2E709A903C996E80C008DE80300294613
:1085D0002046B8470028B7D1BAE709A903C996E8E9
:1085E0000C008DE8030029462046C0470028ABD187
:1085F0000020ADE77CBB00249984020890F8843207
:10860000062B08D8DFE803F00C070907040704006D
:10861000064801F07BBB01207047054801F0ACBF64
:10862000C36842F2E8201844C8F05CBD80C300244F
:10863000B4C7002490F884220346072A1BD8DFE839
:1086400002F007160D1A040704100C4801F078BA5E
:10865000C36842F2E8201844C7F046BE084801F05B
:108660003DBFC36842F63070184400F04BBC012097
:1086700083EDA20A70470020704700BF80C300242A
:10868000B4C7002470B54B880C460646722B0CD834
:108690005B2B2DD8103B9AB2042A26D8042B24D861
:1086A000DFE803F0746267626B00DE2B54D8B12BF5
:1086B0001BD9B23B2C2B18D8DFE803F0BAC0171730
:1086C000171717171717171717171717CD6D176DD8
:1086D0001717176D1717171717171717171717A843
:1086E0001717171717171717AE000025284670BD64
:1086F0005C3B162BF9D801A252F823F0CB87020875
:10870000F5870208EB860208EB860208EB86020872
:10871000EB860208EB860208EB860208EB8602086D
:10872000EB860208EB860208EB860208EB8602085D
:10873000EB860208EB860208EB860208EB8602084D
:10874000EB860208EB860208EB860208D587020852
:10875000EB860208FD8702084AF2CE629342C4D13A
:108760000125FFF7C1FAC1E70122BDE87040FFF71C
:10877000AFBEBDE87040FFF765BA4848FEF752F952
:10878000054628B3022386F88432AFE70022BDE80D
:108790007040FFF79DBEE368002B6ED12369002B6C
:1087A0006BD16369002B68D13D4C94F8E51D04F64C
:1087B0006C507DF06BF804280AD194F8E51D04F69E
:1087C0006C5001257DF06CF890E78B88002B5FD111
:1087D00001258BE7D0F072FA9FED327AC6F8B40229
:1087E0000125D4ED027A67EE877AFDEEE77AC6EDD1
:1087F000AC7A7BE70125FFF721F977E7D1ED027A23
:108800000125FDEEE77AC0EDAC7A6FE721463046F0
:108810000125FFF769F969E7A3884FF47A7194EDB0
:10882000040A0125204803FB01F101F029FA5DE764
:10883000214630460125FFF737FA57E7A388012B79
:1088400013D1174890F8105E7DB10021A0F50040CB
:10885000FDF772F94AE7A18801253046491BB1FAB4
:1088600081F14909FEF748FB40E7002204F10801C5
:108870000E480125FDF788F938E7094804F1080298
:10888000012590F8E51D00F66C507DF0C5FB2DE745
:1088900008310125FFF768F828E700BFB4C70024B6
:1088A000A0AE002400007A4480C30024A02E00243F
:1088B0000920704700487047882D1708012070472D
:1088C00090ED260A704700BF90ED0B0A704700BF7D
:1088D000C26842F65053134493ED710A704700BFCB
:1088E00008B500F1440386468C46DFED0A7A0FCBCB
:1088F0008CE80F009EED1B0A60469EED171A20EED5
:10890000270AB7EEC11AB7EEC00A0FF077FF0120B1
:1089100008BD00BFE02E6542034642F6505000B548
:10892000DB6885B01844C7F069F9B0EEC06B9FED05
:10893000127B8DED000B8DED021BB4EEC76BF1EEDB
:1089400010FA06D5B0EEC11BB4EEC71BF1EE10FA5B
:108950000BD4684631F0B6FCB7EEC00BDFED087AF9
:1089600020EE270A05B05DF804FB9FED060A05B06E
:108970005DF804FBAFF30080000000000000803EC3
:10898000E02E65420000000010B5002386B00446CA
:108990000093019307F0A8F9694605F0B1FE18B9F4
:1089A0009FED180A06B010BD94ED1C7B94ED1E6B74
:1089B000694604A8B7EEC77BB7EEC66B8DED047AA7
:1089C0008DED056A31F072F8B0EEC07ADFED0E7A07
:1089D0008DED020ACDED030AB4EEE77AF1EE10FA5E
:1089E00006D5F0EEE00AF4EEE70AF1EE10FAD7D47D
:1089F00002A831F0CDF8DFED057A20EE270A06B0A7
:108A000010BD00BF0000000000000034E02E6542F1
:108A100010B50446FDF7D8FF114B204640F8443B03
:108A20000FF012F9002320460E496365A365C4F8D0
:108A30008030C4F88430C4F88830C4F88C309FED9E
:108A4000067B84ED1C7B84ED1E7B5BF05BFB20468C
:108A500010BD00BFAFF30080000000000000000068
:108A6000B44917086C49170810B5002384B00446B0
:108A70000093019307F038F9694605F041FEA0B173
:108A800004F15401684631F011F802A88DED020A94
:108A9000CDED030A31F0C6F8B0EEC00ADFED0A7A78
:108AA000B4EEE70AF1EE10FA06D507F01DF9D0F89A
:108AB0000C32E36604B010BD02A831F069F884ED11
:108AC0001B0A04B010BD00BF00000034B6EE007AEF
:108AD0009FED274ADFED277A00F17001DFED263A9E
:108AE00010B590ED171A0446C36882B0B4EEC71AE9
:108AF000D0ED264A03F5B55390ED166A90ED155A60
:108B0000B7EEC11AF1EE10FA93ED007A90ED1B0A60
:108B1000B7EEC66A90F89430B7EEC55A67FE847A0D
:108B2000B4EE677A20EE230A08460191F1EE10FABE
:108B3000B7EEC00A77FE277AF4EEE74A84ED1C5BB5
:108B4000F1EE10FA84ED1E6B98BF43F0010384F838
:108B5000943031F0E9FB094AE36842F6505092ED57
:108B6000D40A0199184402B0BDE81040C6F0F8BF1D
:108B7000CDCCCC3DCDCC4C3EE02E6542A02E002489
:108B800070B5044642F65053B6EE007A544DD320E9
:108B9000D5EDD47A2DED048BE26882B094ED180AFD
:108BA0001344D4ED1A6A93ED5B1A30EE660A21EE97
:108BB000071A21EE271AF1EE410A2CF0E7F8D4ED5E
:108BC0001A7A94F89C30B0EE408A70EE277AC4EDA1
:108BD0001A7A002B7AD1DFED436A94ED177A636E2F
:108BE00027EE267AC7EE878A68EEA68A002B6AD11E
:108BF00095EDD49A94ED1B0AA9EE280AB7EEC00AA7
:108C00002CF084F894ED247AF7EEC07BA9EE287A54
:108C1000C4ED1B7A84ED247A94ED166A04F1700198
:108C200094ED155A04F180069FED2F0AB7EEC66A3F
:108C3000B7EEC55A94ED171A27EE800A0846B7EE2C
:108C4000C11A019184ED1C5B84ED1E6BB7EEC00A66
:108C500031F06AFB94ED1B7AA36E3046B7EEC77A0B
:108C6000C4F8803000239FED1C0BC4F8843037EE2D
:108C7000000BB7EEC00B31F083F8D4ED1A7A95ED06
:108C8000D47A04F1880367EEE77A94ED176AC8EEA8
:108C9000076A94ED1B0A1846009387EE867AC4EDA6
:108CA000236A84ED227A31F06BF8E46842F6505082
:108CB000009B32460199204402B0BDEC048BBDE814
:108CC0007040C6F061BFF1EE688A91E72046FFF779
:108CD000CBFED4ED1B7A9FE700000051FB21F93F4A
:108CE000A02E0024DB0FC940E02E654210B5002302
:108CF00004462DED028B8AB00293039306F0F4FF35
:108D000002A905F0FDFC00287CD004F1540102A862
:108D100030F0CCFE02A906A8CDED050A8DED040ABF
:108D200094ED1E6B94ED1C7BB7EEC66BB7EEC77B64
:108D30008DED076A8DED067A30F0B8FE08A8CDED0E
:108D4000090A8DED080A30F06DFF04A884ED0B0AC6
:108D500030F068FF94ED177A94F8943030EE470ABB
:108D6000B0EEC00A84ED260A53B3B6EE006AE3689B
:108D7000DFED3B7A03F5B552DFED3A6AB4EEC67A21
:108D800092ED007AF1EE10FA67FEA67AB4EE677AF9
:108D9000F1EE10FA77FE277A37EEA77AB4EEC70A1B
:108DA000F1EE10FA35DD94F89C20002A3FD0B4EEA5
:108DB000E70AF1EE10FA35D5002284F89C2003E092
:108DC0002046FFF783FEE368274A42F6505092EDB3
:108DD000D40A1844C7F02CF8E26842F650532046F3
:108DE000134493ED6F8A93ED700AFEF7E9F9236857
:108DF000B0EE480A01211B6E204698470AB0BDEC30
:108E0000028B10BD2046FEF77DF80AB0BDEC028B48
:108E100010BDB4EEE70AF1EE10FA03D594F89C20E9
:108E2000002AC9D12046FFF7ABFEE368CCE7D4EDBA
:108E3000187A9FED0E7A67EE877AC4ED187A77F08C
:108E400003FA94ED187A0A4A0421B7EEC77A8DED39
:108E5000007B6DF093FB0122E36884F89C20B3E76C
:108E6000CDCC4C3ECDCCCC3DA02E0024CDCC4C3F27
:108E7000E448170810B541F24453C268DFED1C7A8C
:108E800082B01344044693ED000AB4EEE70AF1EE13
:108E900010FA19DDDFED177A20EE270AD4ED177AE4
:108EA00020EE270A2BF0FAFDB5EEC00AD4ED187AB1
:108EB000F1EE10FAD8BF9FED100AF4EEC07AF1EE91
:108EC00010FA04DC02B010BD9FED0C0AE6E784ED59
:108ED000180A77F0B9F994ED187A094A0421B7EE27
:108EE000C77A8DED007B6DF049FB02B010BD00BF6D
:108EF000CDCCCC3D0AE81C4100000000DD0C7B3FDE
:108F000010491708DFED147AB4EEE70AF1EE10FA13
:108F100001DA0020704710B5044680ED180AFFF70B
:108F2000A9FF42F65053E26894ED180A1344D3EDBA
:108F30005A7AB4EEE70AF1EE10FA01DC012010BD16
:108F40001846D3ED5D1A93ED5C1AD3ED5B0AC6F0BB
:108F50002FFD012010BD00BF0000003410B52DED25
:108F6000028BD0ED0E7A82B09FED647A0446F0EE6B
:108F7000E77AC36803F5B553F4EEC77AF1EE10FA59
:108F800077FE877AC0ED177A93ED007AF4EEC77A10
:108F9000F1EE10FA00F1A08094F94030D4ED0F7A90
:108FA0009FED577AA3F10103F4EEC77AB3FA83F386
:108FB0005B09F1EE10FA636604DAE36803F5005327
:108FC000D3EDBB7AC4ED187A06F08EFE0021D0F8FE
:108FD0000C2204F1440C4B4BA166E2660FCB8CE8EB
:108FE0000F002046FFF746FFE26841F22C530021B4
:108FF00041F23C20134484F89C10104493ED008A05
:10900000B5EEC08AF1EE10FA57DDC6F067FAB4EE9D
:10901000408AF0EE400AF1EE10FA48BFF0EE480A3E
:10902000DFED377AF4EEE70AF1EE10FA4EDBE26894
:109030009FED337A02F50053D3EDC27AF4EEC77A8E
:10904000F1EE10FA05DBF4EE670AF1EE10FA77FEA6
:10905000A00AD3EDC31A41F24453DFED297A42F658
:109060005050134494ED180AF4EEE71ADFED237A1A
:1090700093ED001A1044F1EE10FAB4EEE71A61FE17
:10908000A01AF1EE10FA24DDDFED1F7A21EE271A87
:10909000C6F08EFCE36842F650501844C6F0C6FC99
:1090A000002300220120C4F89030C4F8983084F8DE
:1090B000942002B0BDEC028B10BDC6F00FFAB5EEE5
:1090C000C00AF0EE400AF1EE10FAA9DDF7EE000A50
:1090D000ADE79FED0E1ADBE780ED177A77F0B4F875
:1090E000E3680B4A042103F5B55393ED007AB7EE1C
:1090F000C77A8DED007B6DF041FA4DE7CDCCCC3DCC
:10910000000000347CBB00240AE81C41DD0C7B3FDE
:109110002C49170810B5044606F0E6FD04F1540189
:1091200005F0EEFA20B12046BDE81040FFF716BF6B
:1091300010BD00BFF0B50D46002304461746284673
:109140002DED028B85B0B0EE408A02A90293039305
:109150000EF0C4FE00283DD023682C4A9B6D93423C
:109160003ED106F0C1FD04F1540105F0C9FA88B3FF
:109170002046FFF7F3FE064666B39FED250A02A8D8
:1091800030F0A4FCDFED237A84ED150AB0EEC80AB6
:10919000E368C4ED160AB4EEE70A03F5B553F1EE41
:1091A00010FA30FE270A84ED170AD3ED007AB4EEE8
:1091B000E70AF1EE10FA17D467662046FFF754FC71
:1091C000443495E80F0084E80F00304605B0BDEC4C
:1091D000028BF0BD0026304605B0BDEC028BF0BD21
:1091E000204698470646C7E7C4ED177A77F02CF873
:1091F000E368094A042103F5B55393ED007AB7EE0D
:10920000C77A8DED007B6DF0B9F9D5E715910208AD
:109210000AD7233CCDCCCC3D2C49170808207047F9
:1092200000487047602D17080120704790ED0B0A29
:10923000704700BF70B5694D95F980392DED028BEF
:10924000002B00F09C80044605F51860CCF068FD0A
:109250000646002800F0938094F940304BB1DFEDD2
:10926000607A94ED0F7AB4EEE77AF1EE10FA40F2FC
:10927000AD8094ED0E8ADFED5B7AE268B4EEE78AAA
:10928000F1EE10FAC0F29A8041F22C5341F23C20E8
:1092900013441044D3ED008AF5EEC08AF1EE10FAC3
:1092A00078DCC6F01BF9B5EEC00AF0EE400AF1EE2C
:1092B00010FA7ADDF3EE040AE2689FED4A7A02F5CD
:1092C0000053D3EDC27AF4EEC77AF1EE10FA06DB62
:1092D000F4EE607AF1EE10FA48BFF0EE670AD3EDD3
:1092E000C31A41F244539FED3F7A42F65050134463
:1092F000DFED3D7AF4EEC71A104493ED001AF1EE5B
:1093000010FAB4EEE71A61FEA01AF1EE10FA5ADD77
:10931000DFED367A21EE271AB0EE480AC6F048FB98
:10932000E36842F650501844C6F080FB95F9BE2918
:10933000E368A2F10402DFED2E7A03F50053B2FADE
:1093400082F2520983F8082F94ED0F8A28EE278ABB
:10935000B0EE480A3CF10AFDF0EE407AB0EE480A61
:10936000B0EE678A3DF19EFB002384ED180A30467B
:1093700084ED178A84F86430BDEC028B70BD76F002
:1093800063FF1C4A052100266DF0F8F83046BDEC5D
:10939000028B70BDC6F0A2F8F4EE408AF0EE400AEF
:1093A000F1EE10FA48BFF0EE680ADFED0E7AF4EE47
:1093B000E70AF1EE10FABFF67FAF7BE702F5005344
:1093C00093EDBB8A60E79FED0C1AA5E776F03CFFB2
:1093D0000A4A052100266DF0D1F8D7E7A0AE002497
:1093E000000000B400000034CDCCCC3D0AE81C41A4
:1093F00035FA8E3C184A1708DD0C7B3F344A1708B3
:1094000010B50446FDF7E0FA094A00230948E26472
:109410000022094920652046216063650749A3654C
:10942000E3652366A4F864205AF06CFE204610BD64
:10943000000096430000A041604B1708F84A170847
:1094400070B5002384B00D4606460093019306F0E4
:109450004BFC694605F054F9044688B19FED0A0AB1
:10946000684630F033FB06F1540002A98DED020A84
:10947000CDED030A30F01AFB85ED000AC5ED010AB7
:10948000204604B070BD00BF0000C84210B52DEDED
:10949000048BB6EE009A86B0F0EEC08AB0EE408A39
:1094A000F4EEC98AF1EE10FA05D5B0EE480A06B01E
:1094B000BDEC048B10BDDFED3C9A69460446CDED52
:1094C000009ACDED019ACDED029AFFF7B9FF002881
:1094D000EBD006F009FC694600F54870B7EE008A4B
:1094E0002CF090FDF0EE607A8DED030AF0EE416A0B
:1094F00094ED147AB0EE481AB0EEE70ADD20F0EEF3
:10950000690ACDED047ACDED056A80EE070A2BF0ED
:109510003DFC9DED036ADFED256AE520F9EE047A56
:10952000B2EE047AF0EE690AE6EE267AF0EE409AA0
:10953000B0EE481A87EE870A38EE400A2BF026FC78
:10954000A9EEC08AD4ED0B7A42F6505394ED127A0C
:10955000E26877EEC77A134468EE888AF0EEE77A1D
:1095600093ED5B0AF4EE498A77EEA77AF1EE10FAF2
:1095700027EE800A48BFF0EE498A2BF08FFAE368A5
:10958000F4EE408A03F5005393F8083FF1EE10FA29
:1095900048BFB0EE680A002B89D0B1EE400A06B091
:1095A000BDEC048B10BD00BF000000000AD7233CB7
:1095B000F0B52DED068B90F864309FB004468BB16A
:1095C00090F865303BB18C481FB0BDEC068BBDE810
:1095D000F04000F0AFBD1FB0BDEC068BBDE8F04021
:1095E000FDF790BC00F154069FED848A8448314613
:1095F000CCF0B8FB12A9054620468DED128A8DED00
:10960000138AFFF71DFF002800F0B08012A830F089
:1096100009FB9FED7C7AD4ED137A20EE070AD4ED96
:10962000126A67EE877A84ED0B0AB4EEE70AF1EE70
:1096300010FAB4EEE60A4CBF01230023F1EE10FA53
:1096400004D985F00100C0B298B193B1012384F828
:10965000643076F0F9FD6C4A06216CF08FFF6B48A0
:1096600002F040FF002840F094801FB0BDEC068B54
:10967000F0BDB4EEE70A94ED159A94ED16AAF1EE5A
:1096800010FA04D494F94030002B40F088801AADD1
:10969000B7EEC99A2846B7EECAAA42F650555B4EB5
:1096A0009FED530B8DED1A9B8DED1CAB30F0ECFD57
:1096B000E06816A928448DED160B96EDD40A8DEDC1
:1096C000181BC6F04DFAE06896EDD40A2844C6F09F
:1096D000AFFBE2682B4620461344D3ED708A93ED2E
:1096E0006F0AFFF7D3FE2046B0EE408AB0EE680A5C
:1096F000FDF766FD2368B0EE480A01211B6E204687
:10970000984769F097F90546CFF0E0FA94ED0B4AD7
:1097100094ED165AB7EEE87A94ED156AB7EEC44A9E
:10972000B7EEC55A0246B7EEC66A0B46B7EEC88A10
:10973000374C38492846CDE90223CDE90014364B91
:10974000364A37498DED107B8DED0E8B8DED0CABD0
:109750008DED0A9B8DED084B8DED065B8DED046B59
:1097600068F0F4FC1FB0BDEC068BF0BD41F2B01503
:10977000E068B0EE480A2844CAF03AFDE068B0EE6E
:10978000480A01212844CAF02DFD1FB0BDEC068B0C
:10979000F0BD1948FDF746F984F8650065E704F166
:1097A0005C071AAD12A894ED118A394630F0D2FA4E
:1097B0002846CDED1B0A8DED1A0A30F033FA28EE5B
:1097C000000A384630F082F930462946CDED1B0AB2
:1097D0008DED1A0A30F06AF9B0EE409A8DED140A58
:1097E000B0EE60AACDED150A52E700BFAFF30080DE
:1097F00000000040E17A843F2CC7002400000000F4
:1098000020B800240AD7233C684A1708A02E002459
:109810006C151708C04A1708804A17088C4A1708A1
:10982000602D170806207047004870477C2C1708E9
:10983000012070479FED010A704700BF0000000043
:1098400000207047C268034602F5005292F94801B1
:1098500018B1D2F8EC2201209A637047C36803F56F
:10986000005393ED6B0A7047C36803F5005393ED03
:109870006A0A7047DFED067A0346B4EEE70AF1EEB6
:1098800010FA03D9012083ED0E0A704700207047BB
:10989000000000B4034642F24810DB681844C9F0E7
:1098A0001BB800BF30B52DED028B8DB00446806A29
:1098B0006946C5F009FC002870D0002142F248102A
:1098C00009AB06AA039104910591069107910891AD
:1098D00009910A910B91E168084403A9C9F0C8FAFB
:1098E00000286ED0E368DDED065A03F50053DDED88
:1098F000097A9DED076A93ED597A9DED0A0AE5EE26
:10990000877ADFED396AA6EE070AB0EEE77ACDED89
:10991000017A8DED020AB4EEE67AF1EE10FA06D580
:10992000B0EEC07AB4EEE67AF1EE10FA49D420EE49
:10993000000A002384F83030A7EEA70A2BF0AEF817
:10994000B0EEC07ADFED287AB0EE408AB4EEE77A66
:10995000F1EE10FA06D494ED0E0AB4EEC80AF1EE58
:1099600010FA38D4DDED010A9DED020A3DF196FAB8
:10997000DFED1E7A20EE270A2BF056F92046DFEDA8
:109980001C0AFDF73BFC2368B0EE480A01211B6E60
:10999000204698470DB0BDEC028B30BD41F2B015AA
:1099A000E0689FED130A2844CAF022FCE068012118
:1099B0009FED0F0A2844CAF015FC0DB0BDEC028BD8
:1099C00030BD0123204684F83030FDF79BFA0DB0FE
:1099D000BDEC028B30BD80EE080A01A830F0A0F883
:1099E00094ED0E8ABEE700BF00000034A00CB34522
:1099F0000000000002680549D26A8A4205D1C368A6
:109A000003F5005393ED6B0A704710475D98020809
:109A10000F20704700487047304C170801207047EE
:109A20000120704790F8383063B1032B07D10B4BFE
:109A3000DFED0B7A93ED000A20EE270A70479FEDC9
:109A4000090A7047C26842F69C23DFED057A134489
:109A500093ED000A20EE270A704700BF60C700247C
:109A60000AD7233C0000000090F8383063B1032B84
:109A700007D10B4BDFED0B7A93ED000A20EE270A9E
:109A800070479FED090A7047C26842F69823DFEDE0
:109A9000057A134493ED000A20EE270A704700BFB1
:109AA00060C700240AD7233C0000000090F838303B
:109AB00033B9C26842F6A023134493ED000A7047FD
:109AC0009FED010A704700BF0000000090F8383099
:109AD00043B1032B03D1054B93ED000A70479FED73
:109AE000040A704790ED0B0A704700BF58C7002466
:109AF0000000000010B504460E4802F0F3FC78B9EF
:109B0000052384F83830E36842F2E8209FED0A0A22
:109B10001844C7F085F90023012084F8443010BDB3
:109B20000648FCF77FFF0028EAD0032384F838308A
:109B3000E9E700BFA02E0024000000002CC700248D
:109B400090F838300BB100207047C36842F2E8202B
:109B50001844C6F0C9BB00BF30B5012504462DED41
:109B6000028BF0EE408A87B0B0EE608A80F8385001
:109B7000CFF0A4F84FF0000CE06303AB6A4694F812
:109B800038100C48C4ED0D8A84ED128A84F83950DF
:109B9000CDED008ACDF804C0CDF808C08DED038A64
:109BA000CDF810C0CDF814C0FAF79AF807B0BDECA4
:109BB000028B30BDA02E0024022310B52DED028BA8
:109BC00080F8383086B00446F0EE408AB0EE608A05
:109BD000CFF074F801224FF0000CE06303AB84F87F
:109BE00039206A4694F838100B48C4ED108A84ED89
:109BF000128ACDED008ACDF804C0CDF808C08DEDF5
:109C0000038ACDF810C0CDF814C0FAF769F806B091
:109C1000BDEC028B10BD00BFA02E0024042310B5A4
:109C20002DED028B82B080F838300446B0EE608AA9
:109C30008DED010ACFF042F80346B7EE001AFFEEB1
:109C4000000A4FF4BF7023659DED010A2BF09EF8CA
:109C5000F0EE407AB7EE001A40F27F10FFEE000AF5
:109C6000B0EE480AC4ED157A2BF090F8012384ED8C
:109C7000160A84F84C3002B0BDEC028B10BD00BF58
:109C8000C16580ED180A704700220023C265036693
:109C9000704700BF10B50446CFF010F8034B606664
:109CA00004F1680C0FCB8CE80F0010BD7CBB0024C6
:109CB00010B5C36D044653B9DFED127A94ED187AEE
:109CC000B4EEE77AF1EE10FA0ADA002010BDCEF019
:109CD000F5FF626EE36D801A9842EDD3012010BD4E
:109CE000094804F168010EF09BF994ED187AB7EE7B
:109CF000C77AB4EEC70BF1EE10FACCBF01200020FA
:109D000010BD00BF000000347CBB002490F8383048
:109D10000BB101207047C36842F2E8201844C7F035
:109D2000E1B900BF70B590F838300446052B00F259
:109D3000F380DFE803F017334C93031290F84C30B4
:109D4000002B40F0A880784802F0CCFB28B177487F
:109D5000FCF768FE002840F095802046BDE8704082
:109D6000FDF7D0B8C36842F2E8201844C7F0BAF94A
:109D7000002800F08B8094F84430002B40F0B18034
:109D8000694802F0AFFB00286DD06848FCF74AFE36
:109D9000002868D0032384F8383067E090F8393021
:109DA000002BD0D0CEF08AFFE26B40F6B833801A99
:109DB000984200F29D8094F83930002BC3D0DFED3B
:109DC0005C0A204694ED0D0AFDF718FA30E090F891
:109DD0003930002BB7D0CEF071FFE26B40F6B833CC
:109DE000801A984200F2848094F83930002BAAD06F
:109DF000E368D4ED107A9FED4F7A03F580534A4A19
:109E000067EE877A93F8B0119FED4B0AD2EDD40A32
:109E1000C1F3400227EE800AA06A01F00101C5F0FB
:109E2000D5F9DFED467A204620EE270AFDF79AF9AC
:109E300094ED120A2046DFED427A2368B4EEE70A79
:109E40001D6EF1EE10FA94BF01210021FDF7EEF82E
:109E500020462B460121BDE8704018473348BDE835
:109E6000704000F067B92046FDF74CF8E36842F611
:109E70005821344819440EF0D3F8B7EEC00B84EDE6
:109E80000B0A70BD032384F8383070BD2046BDE84E
:109E90007040FDF78DBACEF011FF226D40F6B83359
:109EA000801A98422ED894F84C30002B3FF44BAFD8
:109EB00094ED150A41F2B015E0680021DFED1F7A3C
:109EC000284420EE270ACAF08DF994ED160AE068BE
:109ED000DFED1D7A284420EE270ABDE87040CAF065
:109EE00087B90021194884F8441072F0C9FD47E78A
:109EF00076F0AAF9164A04216CF040FB002384F89E
:109F0000393020E7002384F84C3076F09DF9104A70
:109F100004216CF033FBC6E776F096F90D4A042174
:109F2000BDE870406CF02ABBA02E00242CC7002492
:109F3000000000000AD7233C35FA8E3C00A08C4577
:109F4000000000B47CBB00240000C84214B9002407
:109F5000384C1708644C170890F838303BB1032B85
:109F600002D10648FCF7CEBB9FED050A7047C268D8
:109F700042F69423134493ED000A70472CC7002443
:109F80000000000038B590F838304BB1032B04D1F5
:109F90000C48BDE8384000F0C5B80025284638BD5B
:109FA000C36803F5005292F8785A002DF6D042F2B9
:109FB000E8200C461844C7F0A7F80FC884E80F0043
:109FC000ECE700BF2CC7002482B070B588B0C5682C
:109FD0000E460CAC84E80C0005F500530446D3F89B
:109FE000203F5B0633D50EAB93E803000CAB8DE846
:109FF000030042F2E82031460CCB2844C7F0E0F8D9
:10A0000060B300210125E368002084F8381002AA1B
:10A0100084F8445003F52A5396ED027AD6ED037A7C
:10A02000B8EEC77A1B68F8EEE77A0490059305ABA3
:10A03000069007900C488DED027ACDED037AF9F782
:10A040004FFE284608B0BDE8704002B0704742F2AB
:10A05000E8202844C6F082FE0028D2D1002008B0B3
:10A06000BDE8704002B07047A02E00240420704765
:10A0700000487047184517080020704700207047B7
:10A080000020704730B5002383B004461048019388
:10A09000FBF748FDB0B9E36842F6143041F2B01561
:10A0A000184401F04BFAE0689DED010A2844CAF01B
:10A0B0009FF8E06801219FED070A2844CAF092F852
:10A0C00003B030BD01A90248FBF7E6FCE3E700BF9F
:10A0D000A02E0024000000000520704700487047B3
:10A0E000504D170801207047DFED037A90ED0D0AFF
:10A0F00020EE270A704700BF0AD7233CDFED037A22
:10A1000090ED0D0A20EE270A704700BF0AD7233CC6
:10A110009FED010A704700BF0000000090ED0B0AA0
:10A12000704700BF38308C460FC88CE80F00012004
:10A13000704700BF30B5044683B0864804F138014B
:10A1400001910DF06DFFB7EEC00BE36842F61430DD
:10A1500084ED0B0A184401F017F80199002800F06B
:10A160009C80E068D4ED0B7A00F5005303F634329E
:10A1700092ED007AF4EEC77AF1EE10FA40F29A808E
:10A1800003F6145277EEC77A93EDBB7AD2ED006AEC
:10A19000704867EEA67AF4EE477AF1EE10FA48BFFF
:10A1A000B0EE677A84ED127A0EF0DEFBB6EE007B3D
:10A1B00063689FED666BA0EE067BBDEEC77BB8EED5
:10A1C000C77A84ED0D7A93ED800AB8EEC00A37EEB7
:10A1D000400A2AF029FDB0EEC07ADFED5F7AE3682D
:10A1E000B4EEE77A03F50053F1EE10FA93F9D931A2
:10A1F00050DD002B4ED1DFED597A94ED0D0A30EE93
:10A20000270A2AF011FD636884ED0D0AD3ED807AE8
:10A21000F8EEE77A30EE670A2AF006FDD4ED127AFE
:10A22000F1EE677AC4ED127A9FED4B7A3620B7EEE5
:10A23000001ADFED4B0AC0EE077AB0EEE70A2AF00B
:10A24000A5FDB6EE006AB7EE007AD4ED127AE068AA
:10A25000D4ED0D6AA0EE467A67EE877AC4ED127AE5
:10A2600042F61435B0EE660A284401F04DFB002892
:10A270004DD1DFED3B0A94ED0D0A2046FCF7BEFF01
:10A280002368012194ED120A1B6E204603B0BDE83D
:10A2900030401847022BC7D1ADE7E068D4ED0B7A08
:10A2A00000F5005393ED777AF4EEC77AF1EE10FAE9
:10A2B0003FF666AF42F61435284400F065FFDFED47
:10A2C000287A0028274B9FED280AA06A07FE800AFB
:10A2D000D3EDD40AC5F038F9E06884ED120A2844B9
:10A2E00000F052FF58BBE06800F5005393F9142BBF
:10A2F000002A28DDD3ED976ADFED1C7A9FED1C0A5A
:10A3000066EEA76A66EE806AC4ED0D6AA8E7E068AB
:10A3100094ED0D0A284401F063FBE06884ED0D0A1A
:10A32000284401F0C1FA0028A3D0E36803F50053E4
:10A33000B3F9F63200EE903AF8EEE00A9BE7E068F7
:10A34000D4ED0D6A8CE7D4ED0D6A89E700000000BA
:10A350009461B6407CBB002400A00C4600A08C4653
:10A3600000000000A02E0024CDCCCC3DE02E6542A4
:10A370000000C84238B5044642F2E820E36804F120
:10A3800038011844C6F030F8054608B9284638BDEB
:10A3900004F14801A06AC4F097FE08B90023A36441
:10A3A00063682846D3ED807AF8EEE77AC4ED0D7A3B
:10A3B00038BD00BF0020704700487047C44D1708E3
:10A3C0000120704700207047002070470020704730
:10A3D000034641F2B0109FED030ADB681844C9F050
:10A3E00023BF00BF0000000030B52DED028B87B009
:10A3F00004469FED318A01AA6946FCF75DFB2046C1
:10A4000002A9FCF783FCE26842F628739DED000A7E
:10A41000134480EE080AD3ED000A2BF0BBFA27485C
:10A4200020EE080A8DED000AFBF77CFB00283ED1E8
:10A4300004AA03A9204641F2B015FCF71DFD05A9A9
:10A440002046FCF735FDE0689DED030A2844C9F07D
:10A45000FBFEE0689DED040A2844C9F001FFE068B6
:10A460009DED050A2844C9F009FFE36842F614305F
:10A47000184400F017FFE0689DED010A2844C9F078
:10A48000B7FEE0689DED000A00F500532844D3F8BC
:10A49000241F01F00101C9F0A5FEE0689DED020A4C
:10A4A0002844C9F0C1FE07B0BDEC028B30BD01A944
:10A4B0000248FBF7F1FABBE700A08C45A02E002470
:10A4C0000B20704700487047384E1708012070472E
:10A4D0000020704790ED0B0A704700BF034642F220
:10A4E000E820DB681844C5F0FFBE00BF70B58AB035
:10A4F000044605F0F9FB90F87C32DB0734D5E268BE
:10A5000041F2587342F2E82006AD1344104493ED33
:10A51000000AB5EEC00AF1EE10FA48BF9FED140A2A
:10A52000C6F07EFC6368E66842F2FC1193ED9C0A7B
:10A5300002A8104A3144B8EEC00A5CF005F928467A
:10A540000DF082FB0AAB13E903008DE8030042F231
:10A55000E82002A995E80C003044C6F031FE18B19D
:10A56000012323870AB070BD00200AB070BD00BF70
:10A57000000000007CBB0024034642F2E820DB68B8
:10A580001844C6F0AFBD00BF10B5044642F2E82043
:10A59000E3681844C6F0A6FD90B394F8383003BBC6
:10A5A0001A4801F09FFFC0B194F8393073B11848D0
:10A5B000FFF7C0FDE36842F65821164819440DF034
:10A5C0002FFDB7EEC00B84ED0B0A10BD1048FCF751
:10A5D00029FA84F839000028E9D12046FCF792FCDA
:10A5E000E8E7002384F8383075F02EFE0A4A062189
:10A5F0006BF0C4FF054801F075FF0028D4D1ECE7EB
:10A600002046BDE81040FCF7D3BE00BFA02E0024BA
:10A610002CC700247CBB00243C4E170838B5C36807
:10A6200003F5005292F8785A0DB9284638BD42F227
:10A63000E8200C461844C6F067FD0FC884E80F00F8
:10A64000284638BD0720704700487047BC4E1708A1
:10A6500010B582B0044601AA6946FCF773FBE368B3
:10A6600003F5005393F91032FBB1DFED157A9DED40
:10A67000017AB4EEE77AF1EE10FA11DA94ED0F0AEE
:10A680008DED000A2046DFED0F0AFCF7B7FD2368C9
:10A6900001219DED010A1B6E2046984702B010BDB6
:10A6A0009DED000A84ED0F0AECE794ED0E0ADDED56
:10A6B000007A30EE270A2AF001FB8DED000AD4E77C
:10A6C00000000034000000004368D3ED807AF8EE0B
:10A6D000E77AC0ED0E7AD3ED807AF8EEE77AC0ED36
:10A6E0000F7A70470C20704700487047BCFA160874
:10A6F000012070470020704790ED0B0A704700BFA3
:10A7000090F83800A0F10200B0FA80F040097047DC
:10A71000034642F2E820DB681844C5F0E5BD00BFFF
:10A7200010B490F83830012B04D0002420465DF896
:10A73000044B7047C36803F5005393F8784A002C24
:10A74000F4D003F658238C460FCB8CE80F0020463C
:10A750005DF8044B704700BF10B584B004466846EE
:10A760000DF072FA6946606805F082FA28B3E26873
:10A7700002F5805393F8B416F9B103F5EB6342F296
:10A78000E82093ED000A1044B5EEC00AF1EE10FA8D
:10A7900016D4BDEEC00AB8EEC00AC6F041FBE368AD
:10A7A00042F2E8201844C5F07BFE30B1002384F863
:10A7B000383084F83A3004B010BD002004B010BD29
:10A7C0009FED010AE9E700BF0000000008490346C9
:10A7D000084A41F2A86010B4D1F8F44D0121DB68B9
:10A7E000A21A5DF8044B184418BF0122C7F0BCBC84
:10A7F000A0AE0024F0C7002470B590F8383086B0C1
:10A800000446012B25D010D8C36841F2A86000216E
:10A810001844C7F063F810B140F2011323872046B3
:10A8200006B0BDE87040FCF76DBB023B012B20D8A1
:10A8300001233F4884F8303001F054FE0028EED068
:10A8400094F83A306BB33B4806B0BDE87040FFF770
:10A8500071BC90F8393073B92046FCF7A9FDE36864
:10A8600042F2E8201844C6F03DFC10B1012384F800
:10A87000393006B070BDC06841F2A866002569464F
:10A880003044009501950295C7F0FCFA88B975F03F
:10A89000DBFC294A06216BF071FE022384F8383074
:10A8A000E7E72448FCF7BEF884F83A000028B6D061
:10A8B000C9E7E06803A90395304404950595C7F0FE
:10A8C00021FBE368C0B142F2E82003AA69461844BC
:10A8D000C5F04CFDB8B975F0B7FC184A06216BF00D
:10A8E0004DFE032384F8383065F014FF3D224FF409
:10A8F000801165F0C1FE06E042F2E8206946184486
:10A90000C5F00AFD18B1002384F83930A4E775F0CA
:10A910009BFC0A4A06216BF031FE032384F8383091
:10A9200065F0F8FE45224FF4801165F0A5FEEAE7D8
:10A93000A02E00242CC700243C4E1708304F1708C7
:10A94000032070470048704700191708012070471E
:10A95000002070470120704790ED0E0A704700BF3D
:10A9600030B52DED028B85B00446806A01A9C4F094
:10A97000ABFB00286AD0204603AA02A9FCF72EF9F7
:10A980009DED038ADFED567A41F2B010E368B4EE34
:10A99000E78A1844F1EE10FA94BF01250025C9F0AA
:10A9A000C9FC50B1DDED037A9FED4E7AF0EEE77A07
:10A9B000F4EEC77AF1EE10FA5FD4E368DDED017AC8
:10A9C00003F5B553DFED486A27EEA77AA26AD3ED07
:10A9D000007A92EDC21AF4EEE67AF1EE10FAB4EED5
:10A9E000E61A77FEA67A87EE270AF1EE10FA28DC3F
:10A9F0009FED3E1A2620DFED3C0A2AF0C7F99DEDB7
:10AA0000026ADFED3B6A29469FED357A2046C6EEA5
:10AA1000267AB4EEC78AF1EE10FA27EE800A98BFC4
:10AA2000B1EE400A84ED0E0AFCF714FC2368012104
:10AA30009DED030A20461B6E984705B0BDEC028BC6
:10AA400030BDDFED2C7A21EE271AD3E79FED2A8A5D
:10AA500041F2B015E068B0EE480A2844C9F0C8FBDE
:10AA6000E068B0EE480A01212844C9F0BBFB84ED40
:10AA70000E8A05B0BDEC028B30BDDDED027A0021FF
:10AA80009FED1B8AE36887EE887A1C4A03F58053A2
:10AA900003F2A46090ED006AA163B7EEC66A93F872
:10AAA000B011A06AD2EDD40AC1F3400201F0010155
:10AAB0009FED095B26EE056BB7EEC77A27EE067BA6
:10AAC000B7EEC70BC4F082FB204620EE080AFCF765
:10AAD00049FBABE7AFF30080000000A046DF913FE9
:10AAE000000000B400000034CDCCCC3DDD0C7B3F39
:10AAF00000A08C450AE81C4100000000A02E0024A4
:10AB000038B50446C0F03EF8036803210122002551
:10AB10009B68984744F254300B4B0C4A20441D600C
:10AB2000156059F03BF944F25030204459F036F9A1
:10AB300044F25530204404F5104459F02FF9044BE9
:10AB400084F8FD535D7238BD54C9002450C90024F7
:10AB5000F0CA002470B500F5104595F8FD3303B92F
:10AB600070BD0446CEF0AAF8304A314B12681B681B
:10AB7000801A984217D22F4B1B78012B33D0022B0F
:10AB80001AD0002BECD12C4A45F218502B4BB2F9BD
:10AB900000202044197800EE102AB8EEC00ACAF04E
:10ABA000C3F80028DCD195F8FD33002BD8D020461F
:10ABB000BDE87040FFF7A4BF204B1E7804F5E043CA
:10ABC000022E21D0D3F8443345F218503146B3F960
:10ABD0000830204400EE103AB8EEC00ACAF0A4F8DB
:10ABE0000028BDD1DFE7144A45F21850134BB2F9E3
:10ABF00000202044197800EE102AB8EEC00AC9F0EF
:10AC0000AFFB0028ACD1CEE7D3F8400377F048F88B
:10AC1000DFED0B7A45F21850314620EE270A20442A
:10AC2000CAF082F800289BD1BDE700BF50C90024BC
:10AC300054C9002458C900245AC900244CC900240E
:10AC40000000C8422DE9F04100F5004E0E469DF887
:10AC500018409EF8F07DBDF91C8097B31D46FAB9E7
:10AC6000334B344A1B68D86A0368DB69934242D18C
:10AC7000042D4AD8022C2CD840F69802A4F10103E6
:10AC80009045B3FA83F34FEA5313D8BF0023002B48
:10AC900045D114B9B8F1640F25DC3846BDE8F08120
:10ACA000844647F2C43001216044F7F727F9034690
:10ACB0000028D5D1204A022130461F4670F052F8B4
:10ACC000EBE730461D4A022170F04CF83846BDE8EB
:10ACD000F081002730462346194A022170F042F8DD
:10ACE0003846BDE8F0811F46164A434602213046E9
:10ACF00070F038F8D1E798470128B9D1124A0221FB
:10AD00003046002770F02EF8C7E7002730462B4664
:10AD10000E4A022170F026F83846BDE8F08143461D
:10AD20000B4A02213046002770F01CF8B5E700BF3F
:10AD3000982E0024591E02084C5017082C50170852
:10AD4000A8501708F05017086C50170888501708BB
:10AD5000D05017082DE9F04700F5104590461F46E2
:10AD60002DED028B82B095F8FD63B0EE408ABDF9FF
:10AD700030900EBB0446CDE9003913467A1E18BF49
:10AD80000122FFF75FFF002843D047F2C4364FF09F
:10AD9000010A264485F8FDA33046BDF04FFF88B375
:10ADA000002304F58044012284F8543384F850339E
:10ADB00084F855331A4B5A72CDF080FF9FED190A73
:10ADC000DFED197A28EE000A184B1860B4EEE70A96
:10ADD000F1EE10FA11D447F23051154B0020154A0C
:10ADE0001960154B177083F80080144BA3F800907E
:10ADF00002B0BDEC028BBDE8F087FCEEC07A17EE26
:10AE0000901AEAE7524630460321F7F7B5F90028D1
:10AE1000C6D1042002B0BDEC028BBDE8F08700BFB4
:10AE2000F0CA002400007A440060EA4650C90024B9
:10AE300054C9002458C900244CC900245AC900240C
:10AE4000B0F9DC1221B9B0F8DA3219B2A0F8DC326C
:10AE500089B20448B1F5C87FA8BF4FF4C871CAF0E1
:10AE600005BE00BF20B80024034648F6801000212C
:10AE70009FED020A1844CBF0C3BC00BF00000000E5
:10AE800070B544F26C3500F5E044064605442846AA
:10AE900076F0D2FD03462846C4F8403376F0F4FD40
:10AEA000C4F84403284676F003FE41F29411C4F836
:10AEB0004803D4F8400376F027FED4F84403642115
:10AEC00076F022FED4F8480310B1642176F01CFE1F
:10AED000C921284678F070F8CA21C4F84C032846E6
:10AEE00078F06AF80346D3212846C4F8503378F046
:10AEF00063F8D4F84C33C4F854034BB141F29411C5
:10AF0000184676F001FE1E21D4F84C0376F000FEC0
:10AF1000D4F8500340B141F2941176F0F5FD1E21B2
:10AF2000D4F8500376F0F4FDD4F8540340B141F264
:10AF3000941176F0E9FD1E21D4F8540376F0E8FD73
:10AF400046F67C60304400F093F947F2C430304458
:10AF5000BDF074FE80B10D4B4FF47A744FF4FA6279
:10AF600044F224701B68462130445B6ADC801A81FD
:10AF7000BDE8704078F0E4BD45F21854A019C9F05E
:10AF8000FFF8A019C9F0DCF8E5E700BF982E00240F
:10AF900010B500F5E0441E21D4F8400376F0B8FD6A
:10AFA000D4F844031E2176F0B3FDD4F8480320B151
:10AFB0001E21BDE8104076F0ABBD10BD2DE9F0417B
:10AFC00000F5E04595F9D4630EB9BDE8F08104467B
:10AFD000D5F8440376F022FF70B104F50043304900
:10AFE000D3F8F40D03685A698A4252D1DB68984756
:10AFF00080F00100C0B230B904F510440023C4F859
:10B00000DC33BDE8F08147F2C438A0444046BDF0CF
:10B0100015FE0746C8B9D5F84033B3F90830B3F583
:10B020007A6FE9DD04F51044CDF048FED4F8DC3346
:10B030009BB3C01AB0F5FA6FC7D301223946404618
:10B04000F7F79AF8C4F8DC73BFE7022EBDD145F2DA
:10B0500018502044CAF0C8FB06460028B5D1D5F8E0
:10B060004033B3F9083013F57A6FC5DA04F51044AC
:10B07000CDF024FED4F8DC337BB1C01AB0F5FA6F02
:10B08000A3D3012231464046F7F7A0F8C4F8DC63A9
:10B090009BE790470028AFD0B5E7C4F8DC0394E7FE
:10B0A0004D4A02082DE9F041044644F26C30204438
:10B0B00076F0EAFA38BB04F5804393F950230AB9D5
:10B0C000BDE8F08104F5E042B3F95263D2F84433AD
:10B0D000B3F90650CDF0F2FD04F50043D3F8083E75
:10B0E000C01AB0F5FA7F37D8ABB2B6B2B3422CBFB4
:10B0F000002301231D4920461D4A8B720121BDE812
:10B10000F041FBF751B9054604F50046CDF0D6FDF8
:10B1100004F58043C6F8080E93F95023BAB104F53C
:10B12000E042B3F95273D2F84433B3F90680CDF05C
:10B13000C5FDD6F8083EC01AB0F5FA7F0ED90B4906
:10B140002B460B4A20468D720121FBF72DF9204634
:10B15000BDE8F041FFF732BF0123CBE71FFA88F5C6
:10B16000BFB2BD422CBF00250125E8E7F0CA00248C
:10B170001851170810B50446024958F0C3FF20467D
:10B1800010BD00BFC851170890F90030002B13DD27
:10B1900010B5036C0446022B0CD0012B08D1DFED57
:10B1A000107A90ED067AB4EEE77AF1EE10FA05DA4D
:10B1B000012010BD002010BD002070470948C7F0D5
:10B1C000B7FF0028F4D0084BD4ED067A93ED007A4F
:10B1D000B4EEE77AF1EE10FA54BF0120002010BD62
:10B1E000000000341C940024C094002410B590F991
:10B1F000003082B00446002B0EDD00230DF1070164
:10B2000017488DF807305BF019F8236C154A023B9C
:10B2100018BF012382F8A23D2046FFF7B5FF38B9D9
:10B220001148C9F087F880B10123236402B010BD32
:10B2300001230E480DF107018DF807305AF0FEFF8B
:10B240000948C9F077F80028EED1462078F0E4F9F3
:10B250000028E9D1034B93F94035002BE4D1E5E711
:10B2600048930024A08E0024B8830024E193002496
:10B2700010B5044676F030FCCF2177F09DFE48B142
:10B280006062642176F040FC606A1E21BDE81040D7
:10B2900076F03EBC024BD3F84433636210BD00BF6E
:10B2A000A09E0024264B10B593F8FC3DDB0736D456
:10B2B000436A04469BB3B3F90830B7209FED211AC7
:10B2C00000EE103ADFED200AB8EEC00A29F05EFD6C
:10B2D0001E48C8F0E1FF636A9FED1A1AB820B3F95F
:10B2E0000830DFED1B0A00EE103AB8EEC00A29F074
:10B2F0004DFD1648C8F0E2FF636AB9209FED111AB0
:10B30000B3F90830DFED120A00EE103AB8EEC00AC9
:10B3100029F03CFD0D48BDE81040C8F0E1BF9FEDAD
:10B32000090A0A48C8F0B8FF9FED070A0748C8F0A5
:10B33000C5FF9FED050A0548BDE81040C8F0D0BF25
:10B34000A0AE00240000C84200000000B883002422
:10B350000000C8C238B50446DFED6A7A6A4D6B4812
:10B36000D5EDD40A2DED068BB0EE409A94ED040A8B
:10B37000BFEE00AA9FED668A20EE270AC3F028FEE2
:10B3800046F2BC539FED636AB7EE007A2B44DFEDC3
:10B39000626ADFED627A60EE089A93ED001A21EEA0
:10B3A000061AB4EEE61AF0EEC18AF1EE10FAB4EE27
:10B3B000E79A88BFB0EE47AAF1EE10FA5DDAB0EE78
:10B3C000480A5748C8F068FFDFED537AB7EE007AB5
:10B3D0005348B4EEE79ADFED4E7ABFEE000AF1EE85
:10B3E00010FAF4EEE79A88BFB0EE470AF1EE10FAD1
:10B3F0004CBF77EEE97ADFED4B7A6AEE277A27EEDB
:10B40000800AC8F05BFFDFED457AB4EEE79AF1EE13
:10B4100010FA06DBD4ED037AF4EEE87AF1EE10FAD6
:10B4200008DD9FED400A3E48BDEC068BBDE8384084
:10B43000C8F056BF9FED3C8A37EE887AB4EEE87AC2
:10B44000F1EE10FA3ADCDFED397AF4EEE78AF1EE4C
:10B4500010FA47DC2AEE081A94ED022ADFED2C0AD6
:10B46000F1EE421A9FED320A29F056FB2C48BDEC52
:10B47000068BBDE83840C8F033BF94ED030AD320F3
:10B4800094ED021AD4ED010A38EEC00A29F07EFCD0
:10B49000F0EE480AB0EE401A94ED022AD4ED011AFB
:10B4A0009FED200A29F038FBB0EE481A39EE800AE9
:10B4B000D820DFED1C0A29F069FC82E7B7EE007A9C
:10B4C000DFED1C6AB0EE681AA9EEE67AB5EEC07A36
:10B4D000F1EE10FAD8BF9FED137AA7EEC71A2AEE45
:10B4E000011AB9E7892078F0A1FADFED0B7A9FED18
:10B4F000121AB4EEE70AF1EE10FA88BFB0EE481A5D
:10B50000AAE700BF35FA8E3CA02E00244484002414
:10B510000000C842E02E6542000000B40000003484
:10B52000B8830024000000000000B442000007437C
:10B530000000C8C20AD7233C0000B4C208B52DEDF4
:10B54000028B9FED0A8A0A489FED0A0AC8F0A4FE02
:10B55000B0EE480A0648C8F0B1FEB0EE480A04480A
:10B56000BDEC028BBDE80840C8F0BABE0000000088
:10B57000B88300240000C84238B500232DED028BAB
:10B580000B6090F90030002B3BDD036CB0EE408A7D
:10B5900004460D46022B0DD0012B08D0B0EE480A10
:10B5A0002046BDEC028BBDE83840FFF7D3BE90F8D3
:10B5B0003C30CBB3294BB0EE480A9FED291A03F576
:10B5C000A042D3EDD41A03F58043264892F818150B
:10B5D000D3EDCE0A93F94633C1F3C002C1F3800123
:10B5E00007EE903AF8EEE77A27EE811AC4F020F8D9
:10B5F000DFED1D7A20EE270A85ED000A236C022B71
:10B60000CCD19FED190A1948C8F046FE9FED180AE3
:10B610001648C8F053FE9FED160A1448BDEC028B85
:10B62000BDE83840C8F05CBEDFED127A90ED067AD6
:10B63000B4EEE77AF1EE10FAB0DB0F48C7F078FD10
:10B640000028DBD00D4BD4ED067A93ED007AB4EEF2
:10B65000E77AF1EE10FAADD4D0E700BFA02E0024B7
:10B660000AD7233C448400240000C842B883002445
:10B6700000000000000000341C940024C09400244A
:10B6800010B582B01C4801A9C3F01EFD48B31B4C85
:10B69000D4F8F40D0368DB68984718B99DED010AEA
:10B6A00002B010BD164A174B92ED007ADFED167A04
:10B6B000234427EE277A93ED000A9FED0D6BB7EE3A
:10B6C000C77AB7EEC00A97EE060B29F01FFBB7EE5C
:10B6D000C00B3AF14BFBDDED017A20EE270A02B0F8
:10B6E00010BD9FED0A0A02B010BD00BFAFF300808D
:10B6F000000000A046DF913F44840024A0AE002457
:10B70000A49C00248CA6FFFF0AD7233C0000000065
:10B7100090F90030002B37DD10B52DED028B036C56
:10B720000446022B2DD0012B08D1DFED207A90EDBD
:10B73000067AB4EEE77AF1EE10FA26DA94F82830B9
:10B74000FBB901211A4A1B4B84F8281092ED008A9C
:10B7500093ED000A30EE480AB7EEC00A29F0D6FA97
:10B76000B0EE006BB7EEC88AA0EE068BB0EE480BC9
:10B7700029F0F4FAB7EEC00B84ED0B0ACDF09EFA77
:10B780002063BDEC028B10BD70470B48C7F0D0FCA6
:10B790000028D3D0094BD4ED067A93ED007AB4EEAD
:10B7A000E77AF1EE10FAECD4C8E700BF00000034ED
:10B7B0002C550024649400241C940024C09400247C
:10B7C000194B10B5D3ED007A044690ED0B0A30EE1C
:10B7D000670AB7EEC00A29F099FAB7EEC00B9FEDE1
:10B7E000107BB0EEC00AB7EEC00AB4EEC70BF1EEA4
:10B7F00010FA07D4CDF062FA226B41F28833801A36
:10B80000984208D9002384F8283084F83C30236318
:10B81000CDF054FAA06394ED0B0A10BDAFF3008095
:10B82000000000481857C63F2C55002490F90030FE
:10B83000002B16DD10B5036C0446022B10D0012B33
:10B8400008D1DFED107A90ED067AB4EEE77AF1EEEA
:10B8500010FA07DA94F8283013B9CDF02FFA2063E4
:10B8600010BD70470848C7F063FC0028F2D0074BB2
:10B87000D4ED067A93ED007AB4EEE77AF1EE10FAA1
:10B88000E8D510BD000000341C940024C0940024AE
:10B89000002310B5044680F8283080F83C3003635C
:10B8A000CDF00CFAA06310BD90F90030002B23DD21
:10B8B00010B5036C0446022B1CD0012B08D1DFED20
:10B8C0000F7A90ED067AB4EEE77AF1EE10FA02DA2A
:10B8D00094F8280010BD0A48C7F02AFC0028F7D0C9
:10B8E000084BD4ED067A93ED007AB4EEE77AF1EEE8
:10B8F00010FAEDD5002010BD002070470000003484
:10B900001C940024C094002490F90030002B54DDD6
:10B9100010B5036C82B00446022B4BD0012B08D12A
:10B92000DFED297A90ED067AB4EEE77AF1EE10FABF
:10B930002DDA94F8280000283DD1DFED247A244B3D
:10B9400067EEC07A9FED237A93ED000AA7EE870A8F
:10B95000B7EEC00A29F0DAF9F2EE047A94ED057A2E
:10B96000B7EEC00B37EE277AB0EEC00A9FED146B2E
:10B97000B7EEC77AB7EEC00A27EE067BB4EEC70B68
:10B98000F1EE10FA94BF0120002002B010BD124861
:10B990008DED010AC7F0CCFB9DED010A0028C8D04F
:10B9A0000E4BD4ED067A93ED007AB4EEE77AF1EE21
:10B9B00010FABED5002002B010BD0020704700BFB5
:10B9C000000000A046DF913F000000340AD7233C6E
:10B9D0006494002435FA8E3C1C940024C094002406
:10B9E0002DE9F0412DED088B0446B0EE408AFFF7BB
:10B9F000CBFB28B9B0EE480ABDEC088BBDE8F0815E
:10BA0000C54E0546DFEDC57A06F2C4539FEDC47AF4
:10BA100067EEC87A96F83C8693ED00AAB0EE4A9A93
:10BA2000A7EE879AB7EEC99AB0EE490B29F06EF9E6
:10BA300094ED056AB7EEC07BB7EEC66A9FEDB25BC8
:10BA4000B0EEC77A26EE056BB7EEC77AB4EEC67BCA
:10BA5000F1EE10FA04DD94F82830002B00F0B880E5
:10BA6000CDF02CF9256B07465DB194F82830002BFA
:10BA700040F02281451B2363B5F5FA7F2CBF0025DA
:10BA8000012506F60866D4ED077A96ED007AF0EE09
:10BA9000C76AF4EEE76AF1EE10FA26DBF0EEE77A19
:10BAA000DFEDA06AF4EEE67AF1EE10FA1DD4002D77
:10BAB0004BD194F82830002B40F00381B4EEE67AA5
:10BAC000DFED997AF1EE10FAB4EE677AACBF01259A
:10BAD0000025B8F1010F14BF002505F00105F1EEB6
:10BAE00010FA02D8B8F1000F2FD0B7EECAAA94ED21
:10BAF000057A9FED85BBB7EEC77AB0EE4A0BA7EE8D
:10BB00000B0B29F02BF994ED057AB7EEC09BB7EE3D
:10BB1000C77AB0EE4A0BA7EE4B0B29F01FF9B7EE30
:10BB2000C08B75BB94F82830002B79D1B8F1000F89
:10BB300042D19FED7E8ADFED7E7A29EE080ABDECC8
:10BB4000088B20EE270ABDE8F081B7EECA8A94ED93
:10BB5000057A9FED6DABB7EEC77AB0EE480BA7EE56
:10BB60000A0B29F0FBF894ED057AB7EEC09BB7EE0F
:10BB7000C77AB0EE480BA7EE4A0B29F0EFF8B7EE04
:10BB8000C08BA36B41F28832FB1A9342CAD974F07E
:10BB90005BFB684A06216AF0F1FCB8F1000F00F087
:10BBA000AD80B8F1010F40F0898084ED0B9A01233C
:10BBB000676384F8283035E09FED5C0ADFED5C7A3E
:10BBC00028EE000ABDEC088B20EE270ABDE8F081C4
:10BBD000B0EE490B29F09AF8B7EEC00BDFED527AC0
:10BBE000B4EEE70AF1EE10FA8CBF0123002398456A
:10BBF0003FF400AF06F2BC53B0EEC00A9FED4E7AA0
:10BC0000D3ED007AF0EEE77A37EE800AB4EEC70A99
:10BC1000F1EE10FA7FF5EEAECDF050F8074630E7C2
:10BC200094ED0B9A454B93ED000A39EE400AB7EEBE
:10BC3000C00A29F06BF8B7EEC07B9FED356BB0EE14
:10BC4000C77AB7EEC77AB4EEC67BF1EE10FA29D9FF
:10BC5000606B41F288333F1A9F420FD9236C012B4E
:10BC60001AD107EE907A9FED367AF8EE677AF4EE05
:10BC7000C77AF1EE10FA0FD584F83C3094ED0B0A38
:10BC8000DFED2A7A9FED2A8A20EE270A20EE080AA5
:10BC9000BDEC088BBDE8F08174F0D6FA294A062184
:10BCA0006AF06CFC002384F8283084F83C3023636D
:10BCB000CDF004F8A063E1E70025E2E694ED0B9AED
:10BCC00075E7B7EECAAA94ED057A9FED0FBBB7EE04
:10BCD000C77AB0EE4A0BA7EE0B0B29F03FF894EDB4
:10BCE000057AB7EEC09BB7EEC77AB0EE4A0BA7EE67
:10BCF0004B0B29F033F8B7EEC08B13E7B0EE489A40
:10BD000084ED0B8A53E700BF000000A046DF913F9F
:10BD1000000000481857C63FA08E00240AD7233CD5
:10BD200035FA8E3C00000034000000B4E02E65427D
:10BD30000000C84220511708DB0F49402C55002451
:10BD400000606A463451170870B505460C4609B9BB
:10BD50002C6470BD0C481646C8F0ECFA0028F7D1E8
:10BD6000462077F059FC0028F2D1084B93F9403572
:10BD7000002BEDD1002EECD074F066FA044A0421B9
:10BD8000BDE870406AF0FABBB8830024A08E00249E
:10BD90005051170800F63C100DF076BD10B5044662
:10BDA0000EF0ACF890F925302BB190F8443313B174
:10BDB00094F9643903B910BD47F2C4302044BCF093
:10BDC0003DFF0028F7D104F63C10BDE810400DF00F
:10BDD000F5BB00BF2DE9F04300F5A0482DED028B27
:10BDE00098F8E03283B023B903B0BDEC028BBDE814
:10BDF000F08345F26C27064607443846B1F0CAF88E
:10BE000098F8E032002B68D0002542F2F8492C4621
:10BE100021464C4438460135B1F0D0F906EB840197
:10BE2000ECB281ED000A98F8E0329C42F0D306F5BE
:10BE3000104494F8E823002A59D094F8FC130131F7
:10BE4000C9B2994284F8FC134CD23846B1F096F945
:10BE500094F8FC133846B0EE408AB1F009FA054672
:10BE6000CCF02CFF94F8FC1306EB810303F5104390
:10BE7000D3F8F42393EDFB0AA5EB020883EDFB8ACC
:10BE800038EE408A08F1FF3CBCF1630F02D9A0EB09
:10BE900002080546C3F8F4533846B1F065F9024686
:10BEA00094F8FC1338460192B1F052F907EE908AEB
:10BEB000DFED230AB0EE401A019AF8EE677A2946C0
:10BEC000B0EE480A06F5125067EEA00A03B0BDECCA
:10BED000028BBDE8F04334F0D7BB06F5104494F86C
:10BEE000E8334BB30023194684F8FC33ADE7012156
:10BEF00084F8E813002B3FF477AF9146144606EB25
:10BF000084052146384609F1010905F51045B1F0CF
:10BF100035F92146384685EDFB0A5FFA89F4B1F020
:10BF2000A7F9C5F8F40398F8E032A342E7D803B0C4
:10BF3000BDEC028BBDE8F083012384F8E83353E7BE
:10BF40006F12833A10B5044641F2E87020445AF06B
:10BF50009BFE2046BDE81040F7F730BEF8F772B8F8
:10BF60000148FAF7F9B900BFA02E002400F5A0435C
:10BF700070B52DED048B93F9C42A0446022A57D0DC
:10BF800000F58042F6EE008AF2EE0E7A45F2A456F3
:10BF900092F9462303F5A365064408EE102A95EDB1
:10BFA0000A9A3046B8EEC88A28EE288AB4EEE78AA4
:10BFB000F1EE10FA58BFB0EE678AC3F09DFA88B967
:10BFC000B4EEC98AF1EE10FA22D4002104F5104231
:10BFD00004F500540B46C2F8D81384F88937BDEC39
:10BFE000048B70BD3046C3F097FAB4EEE80AF1EE68
:10BFF00010FAE5DDB4EEC98AF1EE10FA08D4DFEDEF
:10C00000177A95ED0A7AB4EEE77AF1EE10FADCDBF6
:10C01000CCF054FE04F51042D2F8D83383B904F5BD
:10C020000054C2F8D80384F88937BDEC048B70BD86
:10C03000002304F5005484F88937BDEC048B70BDEF
:10C04000C31A04F50054B3F5FA6F94BF002301231B
:10C0500084F88937BDEC048B70BD00BF000000344C
:10C0600038B5044648F67420144A0621204404F5E5
:10C0700012556AF083FA124B64211B68986A0368B0
:10C080005B689847284601F0ABFF04F50053012296
:10C0900004F6884083F8892783F89426B4F9DC12E3
:10C0A00021B9B4F8DA3219B2A4F8DC3289B226F038
:10C0B000E9FE2846BDE8384002F094B868521708F7
:10C0C000982E002470B50B68054608460C46DB68C0
:10C0D00098470A4E03462046337423681B689847E6
:10C0E00003462046F37023685B689847014642F296
:10C0F00030402844BDE8704052F032B8F0CA002405
:10C100002DE9F84300F50047D7F8F46D8E4264D06E
:10C11000022A04460D4690460DD10B6808461B685E
:10C1200098470C230146384A204664F013F800284B
:10C1300058D1D7F8F46D2846FAF774FC8146A8B3B5
:10C1400043F69C60C7F8F45D04F58045204494F004
:10C150002FF9D7F8F40D03681B689847034630465B
:10C16000A3F10A03B3FA83F35B0987F85C3DFAF79E
:10C1700055FC85F83881D7F8F40D03681B6898479B
:10C18000014641F6982095F83821204465F00AFDD3
:10C1900048F674200021204470F05AFC2046D7F85D
:10C1A000F41DFFF78FFF4846BDE8F88366F042FCB8
:10C1B00003462A6828461D46136898470A21024606
:10C1C000284666F059F948F67420104A04212044A4
:10C1D0006AF0D4F94846BDE8F8834FF001094846B3
:10C1E000BDE8F8832B6828464FF000095B68984744
:10C1F000034648F67420064A052120446AF0BEF939
:10C200004846BDE8F88300BFF4521708D852170813
:10C2100098521708F8B5064609480F461546FBF729
:10C2200059F8044630B12A4601460548BDE8F840B1
:10C23000FFF766BF3046394663F0E8FE2046F8BD9A
:10C24000A02E002470B50A480E461546FBF742F8AA
:10C25000044630B12A4601460548BDE87040FFF764
:10C260004FBF3146024863F0D1FE204670BD00BF8B
:10C27000A02E00242DE9F041044642F2304086B061
:10C28000802704F50045204451F0B6FE2046D5F83D
:10C29000F41D04F5F468FFF715FF48F6406004F557
:10C2A0008056204407F084F947F26030204478F04B
:10C2B0005FFB41F6C830204479F096F942F26C31C8
:10C2C00046F27C5021442044C6F038FF404606F038
:10C2D00021FA48F67420204470F03EFC47F2684092
:10C2E00020449AF023FC0DF009FE4FF400634363F1
:10C2F0000DF004FE0FF04CF904F5405341F2E870E4
:10C300000021C3F8BC7A4FF480632044C6F8943A05
:10C310005BF0DCF945F6C82020448EF06FF945F259
:10C32000B0102044BBF032FA01214046C4F8B47783
:10C3300006F0D0FD042304F55670C4F8F43316F06B
:10C3400045FB4FF400232046C6F8983404F5144604
:10C35000FEF71EFE04F5C04345F2185093F8401551
:10C360002044C8F00FFC77F0FFFE77F049F845F263
:10C370006C202044B0F0CCFD47F284002044B8F09B
:10C3800085F947F228404FF40011204454F0FCFA9C
:10C3900042F2DC30204485F085F848F66C502044A9
:10C3A0007AF070F848F6EC40204409F0DDF82046B9
:10C3B000FEF746FD364B4FF47A7236491B68986A91
:10C3C0000368DB6A984745F610202044C5F0F0F971
:10C3D00046F6C060204495F0B1FF1A22314620464F
:10C3E000FFF78EFE2046FFF73BFE49F290502044B7
:10C3F0002FF04EFA04F510434FF4807241F6982066
:10C40000C3F8D8272044244A244BCDE9042306ABA3
:10C4100013E9060065F0BEF904F58043204693F861
:10C420003113FAF757FF1A22002814BF014631468C
:10C430002046FFF765FE44F26C3099222921204402
:10C4400004F5A044019076F0FFFD9B2205210198A0
:10C4500076F0FAFD019875F027FA1148FEF7C6FE4E
:10C4600094F9C43A022B05D0012385F8F03D06B0BB
:10C47000BDE8F08101230DF10F010A488DF80F305E
:10C4800059F0DCFE012385F8F03D06B0BDE8F081EF
:10C49000982E002461BF0208A02E00245DBF020870
:10C4A0001C9D0024E49400240A4B002270B51D68F2
:10C4B0000C46E86903685B689847E86921460122F1
:10C4C00003681B699847E86921460368BDE8704026
:10C4D000DB681847982E0024034641F6982018443C
:10C4E00066F04AB800F5A04090F9C40AA0F1020035
:10C4F000B0FA80F040097047002070470020704774
:10C50000002070472DE9F84F4FF0010A0446074616
:10C5100000F1740800F5AE792DED028B9FEDAF8A26
:10C5200097ED070A4046F3F0F9FFFB690AF1FF3681
:10C530005FFA8AFBC8F83C304FF07E53F6B2C8F879
:10C54000483097F92830013B0F2B00F24381DFE898
:10C5500013F03500E000EC00A800B500C200D200E6
:10C56000400049005600630070007D008C00980078
:10C57000100034200CF016FB054618B13246214657
:10C58000F2F06EFAC9F800505DB12B6828469B683E
:10C590009847002800F0E680D9F800300BB184F805
:10C5A00057B1BAF1020F07F1180708F1840809F131
:10C5B000040900F0C7804FF0020AB1E748200CF0F0
:10C5C000F1FA05460028DDD032462146F2F0B8FCEB
:10C5D000D8E731467A692046F1F0A2FF0546C9F84E
:10C5E0000000D1E748200CF0DDFA05460028C9D04C
:10C5F000B2EE040A32462146F1F014FDC2E74820AB
:10C600000CF0D0FA05460028BCD0B3EE040A32463E
:10C610002146F1F007FDB5E748200CF0C3FA0546C6
:10C620000028AFD0B3EE0E0A32462146F1F0FAFCF4
:10C63000A8E748200CF0B6FA05460028A2D0B0EED4
:10C64000480A32462146F1F0EDFC9BE760200CF0F1
:10C65000A9FA0546002895D032462146F1F00CFC97
:10C660005F4B2B6000236B628CE734200CF09AFA4E
:10C670000546002886D0324600232146F3F06CFAA6
:10C6800080E744200CF08EFA054600283FF47AAF8C
:10C6900032462146F1F0F0FB524B2B6000232B6415
:10C6A00070E768200CF07EFA054600283FF46AAF78
:10C6B000324600232146F2F04FFF63E768200CF07A
:10C6C00071FA054600283FF45DAF3246012321464A
:10C6D000F2F042FF56E744200CF064FA05460028C9
:10C6E0003FF450AF32462146F1F0C6FB3E4B2B6083
:10C6F00000232B6446E748200CF054FA0546002836
:10C700003FF440AFB1EE040A32462146F1F08AFC14
:10C7100038E728200CF046FA054600283FF432AFEF
:10C7200032462146F3F0BEFE2CE768200CF03AFAC0
:10C73000054600283FF426AF3246FF232146F2F09B
:10C740000BFF1FE7D4F85C21A2B3D4F860210AB331
:10C75000D4F85C31E3B1D4F86031A3B1BDEC028B05
:10C76000BDE8F88F73F070FD5346204A032169F04D
:10C7700005FFD9F8000010B103685B6898470023F3
:10C78000C9F800300DE7E362BDEC028BBDE8F88F1D
:10C790006361E0E794F94030082BD9D101212046AC
:10C7A000F1F0BEFEC4F860010028D1D0022384F865
:10C7B0005731CDE794F92830082BC6D111462046D1
:10C7C000F1F0AEFEC4F85C010028BED0012384F86D
:10C7D0005731BAE7D9F80050D6E600BF00007042E2
:10C7E0004456170888A61A0884AA1A08005317087E
:10C7F00010B5044682B0143000F0C0FF04F12C00E4
:10C8000000F0BCFF04F17400F3F066FE04F1F800E0
:10C81000F3F062FE4FF0FF3315492046C4F858315B
:10C8200057F070FC00230DF1070104F128008DF88A
:10C83000073059F003FD01230DF1070104F1290030
:10C840008DF8073059F0FAFC0F230DF1070104F1C0
:10C8500025008DF8073059F0F1FC064B1A681AB91B
:10C8600020461C6002B010BD0348CCF0F5F900BFB3
:10C87000E45417085CC90024185317082DE9F04345
:10C880008DB003A957F04CF9002845D00023244A65
:10C89000244C07AE176840F6CA728DF82C3004F1AC
:10C8A000A009DFF888C0DFF888800696CDE9073355
:10C8B000CDE90933012314E0022531461A4B112238
:10C8C000CDE9005C23F0AAFBB7EE000A002103A823
:10C8D00058F024F94C451FD0237E10342268D4F838
:10C8E0000CC001258DF81430EBB2F86A0492012BCC
:10C8F000E2D11122CDF800C04346314623F08EFB31
:10C90000B7EE000A002103A858F008F954F82520D2
:10C91000D4F80CC00135E7E70DB0BDE8F08300BFE7
:10C92000982E002484551708445317086458170894
:10C930003853170810B5044682B0FFF79FFF204612
:10C9400057F098FB28B994F9283073B994F940301E
:10C950005BB994F90030002B05DD94F9283013B150
:10C96000D4F85C3153B102B010BD01230DF10701C1
:10C9700020468DF8073059F08FFCEAE7204602B0D8
:10C98000BDE81040FFF7BEBD90F90030002B29DD57
:10C99000012930B50C4683B003D99FED140A03B0CA
:10C9A00030BD01EB4103054600EBC30393F928308A
:10C9B000002BF2D000EB81039FED0C0AD3F85C0151
:10C9C0008DED010A0028EAD0036804EB441401A9A4
:10C9D000DB6805EB840498479DED010A84F8650047
:10C9E00003B030BD9FED010A704700BF000000009A
:10C9F00090F90030002BD4BF00230123012988BF08
:10CA000000230BB90020704701EB410300EBC30387
:10CA100093F92830002BF5D000EB8100D0F85C01B1
:10CA20000028EFD0036811461B69184790F90020D1
:10CA3000002A4DDD2DE9F84F354B0446884635492F
:10CA40001B682DED028BD86A03685B688B4248D166
:10CA5000264604F1440725464FF0010B9FED2E8A30
:10CA6000DFF8BC90DFF8BCA0002A1FDD96F9283063
:10CA7000E3B195F864308BBBB8F1000F29D1D7F83A
:10CA80001831002B3CD0CCF019F90023A866A5F88A
:10CA90007030A5F87230012385ED1B8A3B6073F07E
:10CAA000D3FB5B464A46062169F068FDBBF1020FE5
:10CAB00006F1180605F1840507F1040703D1BDEC62
:10CAC000028BBDE8F88F94F900204FF0020BCBE702
:10CAD000704796F92630002BD1D0E7E786ED068A1D
:10CAE000E4E7984710B994F90020B1E773F0ACFB84
:10CAF0000A4A0621BDEC028BBDE8F84F69F03EBD45
:10CB000073F0A2FB5B465246032169F037FDCDE787
:10CB1000982E0024FDC4020800000000505317089E
:10CB200090531708685317082DE9F04190F9003029
:10CB300086B0002B8DED030A02DD01290C4602D9D7
:10CB400006B0BDE8F08101EB4107054600EBC707E1
:10CB500097F92830002BF3D001EB41164FEA41182A
:10CB600000EB8606B36E002BEAD0CCF0A7F8B36ECC
:10CB70009DED030AC01AB0F57A7F70D3B6F8723013
:10CB80000F2B6CD9B6F87030002B00F0898007EEBF
:10CB9000903AD6ED1B6AD5F86421F8EEE77A86EE76
:10CBA000A77A8DED057A002A78D095F90230002B0E
:10CBB00074DD07EE903A9FED445AB2F90C30F8EE6E
:10CBC000E76AD7ED065AF7EE007A06EE103A37EE2E
:10CBD000657AB8EEC66AE6EE857AF6EE006AB0EEE1
:10CBE000C77A67EE867A67EEA77AE6EE467A67EE50
:10CBF000A67AB4EEE77AF1EE10FA4FDDF0EEE55AE0
:10CC0000661CF5EEC05AF1EE10FA06DD73F01CFB5F
:10CC10002E4A0421334669F0B1FCF0B205A900EBBD
:10CC2000400005EBC00059F0CDFA022205EB840369
:10CC30005A646B68DB063FD573F006FB9DED057A01
:10CC40003346234AB7EEC77A06218DED007B69F0A3
:10CC500095FC4444002305EB8404A36670E708EBCD
:10CC6000040305EB830393F8652072B1B3F87220D7
:10CC7000052A0AD9D3ED1B7AB3F8702037EE800A63
:10CC8000013283ED1B0AA3F87020444405EB8404B1
:10CC9000B4F872300133A4F8723051E7661CBCE777
:10CCA00073F0D2FA631C0B4A042169F067FC03227B
:10CCB00005EB84035A64CCE773F0C6FA3346064AA0
:10CCC000062169F05BFCC4E70AD7233CC853170868
:10CCD000F8531708B0531708205417080346406C40
:10CCE000012807D0032805D0986C012802D003281A
:10CCF00018BF0220704700BF2DE9F84F2DED028BC1
:10CD000090F90030002B02DD01290C4603D9BDEC5F
:10CD1000028BBDE8F88F01EB410605464FEA410959
:10CD200000EBC60696F92830002BF0D000EB810B03
:10CD30000FFA81F8DBF85C31002BE8D004EB4417E4
:10CD4000CBF0BCFF05EB87074FEA441A3866DBF8E7
:10CD50005C0103685B69984768B1DBF85C0184217A
:10CD6000036801FB04519B69503198473B6D87F87C
:10CD70006500FB64CBE72146284697F865B0FFF7CE
:10CD800003FE96ED068ABB6E30EE488A87ED178A61
:10CD9000002B61D1BBF1000F5BD00AEB0403DFED88
:10CDA0006E7A9FED6E7A05EB830368EE277AD3EDFA
:10CDB000166AE6EE877AA1440AEB040305EBC9097B
:10CDC00005EB8303C3ED167A99F92720002A76D064
:10CDD000012A49D1B5EEC08A08EB4808B1EE488A6D
:10CDE000DFED5F7A05EBC808F1EE10FA83ED158AE6
:10CDF00098ED070A58BFB0EE678A28EE008AB4EEB5
:10CE0000678AF1EE10FA00F19280B1EEC80A0AEBDF
:10CE1000040305EB8303D3ED167A83ED130AF5EED5
:10CE2000C07AF1EE10FA4CBFB1EE670A9FED4C0AE2
:10CE3000D8ED077A20EE270AB5EE400AF1EE10FA97
:10CE400038D4F1EEC07A544405EB8404C4ED147A6E
:10CE50005DE7F0EE487AAEE721462846FFF764FE2C
:10CE6000BBF1000FF5D098E708EB4808B0EEC80A10
:10CE700005EBC80883ED150A98ED078A20EE080A2D
:10CE8000B5EE400AF1EE10FA56D4F1EEC07A0AEB94
:10CE9000040305EB830393ED160AC3ED137AB0EE9A
:10CEA000C00AD8ED077A20EE270AB5EE400AF1EE67
:10CEB00010FAC6D53AF154F8F0EE407AC3E7B5EE71
:10CEC000C08A08EB480883ED158A05EBC808F1EE27
:10CED00010FA98ED070AD8BF9FED218A28EE008A44
:10CEE000B5EE408AF1EE10FA30D4B1EEC80A0AEB82
:10CEF000040305EB8303D3ED167A83ED130AF5EEF5
:10CF0000C07A98ED070AF1EE10FAD8BFDFED147A77
:10CF100067EE807AF5EE407AF1EE10FA11D4B1EEB8
:10CF2000E70A544405EB840484ED140AEFE6B0EEFE
:10CF3000480A3AF115F86AE73AF112F8F0EE407A49
:10CF4000A5E7B0EE670A3AF10BF8EAE7B0EE480A57
:10CF50003AF106F8CBE700BF9A99993E3333333F55
:10CF60000000000090F90030002B15DD70B50B7843
:10CF70000D46012B0FD80446D0F85C0110B10368B0
:10CF8000DB699847D4F8600128B103682946DB695A
:10CF9000BDE87040184770BD704700BF08B590F9F4
:10CFA0000030002B0BDD90F85531024683F0010371
:10CFB00001298CBF002003F0010010B908BD00203A
:10CFC00008BD01EB410102EBC10292F92830002BB0
:10CFD000F5D092F9243083B1022BEFD1462076F0C0
:10CFE00025FDB0EEC00ADFED067AB4EEE70AF1EEF9
:10CFF00010FA4CBF0120002008BD184608BD00BF34
:10D000000000003490F900300246002BD4BF00200D
:10D010000120012988BF002000B9704701EB4101C0
:10D0200002EBC10191F92800003818BF01207047B8
:10D0300090F900300246002BD4BF002001200129C6
:10D0400088BF002000B9704701EB41034FEA410C53
:10D0500002EBC30393F928000028F4D001EB41133D
:10D0600002EB830300B593F865004FEA411E30B12F
:10D0700002EB8103D3F85C01003818BF01208C4417
:10D0800002EBCC0CDCED067AF0EEE77AF5EEC07A36
:10D09000F1EE10FA01DD5DF804FB714402EB810151
:10D0A00091F86430002BF6D19CF92630002B0CBF90
:10D0B000002000F00100EEE790F90030002B15DDB4
:10D0C00010B590F9283004461BB10021FFF7B0FFDE
:10D0D00048B194F940303BB101212046FFF7A8FF49
:10D0E000003818BF012010BD012010BD012070477D
:10D0F0002DE9F04F04464FF000092DED028B9DB055
:10D10000DFED618ACBF0E2FD264604F5AE7783467B
:10D110008A4625469FED5D8A94F900205FFA89F8DA
:10D12000002A5EDD95F92820002A5AD03A68002AA4
:10D1300057D00DAA41462046FFF75AFC00285ED082
:10D14000DDED0D7A67EEA87AFDEEE77A17EE903AFC
:10D150001BB20B931D22002114A83CF17DFDA322DC
:10D16000CDF847B08DF844209522CDF84BA08DF82E
:10D17000452072228DF84F808DF8462094F90020CA
:10D18000002A40DC424A0B9B149218EE102AADF89C
:10D190005830CDF85A204146AA692046CDF85E2085
:10D1A000FFF7FCFE41468DF862002046FFF740FF86
:10D1B000D6F8BC308DF863001993D6F8C0301A93B6
:10D1C00094F856318DF86C3065F034FC292211A9A1
:10D1D00064F00CFB38680368D3F824802D4B984525
:10D1E0001ED1843618350437B9F1000F02D14FF043
:10D1F000010991E71DB0BDEC028BBDE8F08F0B90EB
:10D200008DED0D8AA6E70B9B95F92820ADF85830D7
:10D21000002A33D0F26C1492726D1592F26DB8E759
:10D2200010AB0FAA0EA9C0470028DAD00E9AD6F884
:10D23000CC309A42D5D065F0FDFB8046CBF046FD60
:10D240009DED0F6A9DED107A134BB7EEC66AB7EEEF
:10D25000C77A124A0193124BCDF810900093114BEC
:10D26000CDE902018DED086B40460F498DED067B3F
:10D2700064F06CFF0E9BC6F8CC30B2E7044A1492FF
:10D2800018EE102A85E700BF0000C8420000000029
:10D29000000080BF01C502080C0B17084054170896
:10D2A00084EC16083854170858541708F8B590F944
:10D2B0000030002B38DD04460021FFF71DFD012161
:10D2C0002046FFF719FD94F90030002B02DD94F998
:10D2D00040306BBB6678204694F856713146FFF7B4
:10D2E000A7FE054608BB01462046FFF7A1FEB8BBD6
:10D2F00001212046FFF79CFE88BB2046F1F08AFD05
:10D3000094F85631BB4204D065F094FB5A2165F085
:10D3100081F8D4F85831013306D065F08BFBD4F88E
:10D32000581165F029F990B9F8BD84F85661E4E721
:10D3300072F08AFF94F90030002B0DDD94F9403033
:10D3400053B194ED350A084969F078FCC2E72046EC
:10D35000BDE8F840FFF7CCBEBFEE000AF3E70125B9
:10D3600084F85651C9E700BF6054170890F900309F
:10D37000002B01DD012902D9BFEE000A704701EB45
:10D38000410300EBC30393F92830002BF4D001EBE9
:10D39000411100EB810191ED140A704790F90030C2
:10D3A000002B01DD012902D9BFEE000A704701EB15
:10D3B000410300EBC30393F92830002BF4D001EBB9
:10D3C000411100EB810191ED130A704790F9003093
:10D3D000002B01DD012902D99FED080A704701EBFE
:10D3E000410300EBC30393F92830002BF4D001EB89
:10D3F000411100EB810191ED150A7047000000001A
:10D40000014B1868704700BF5CC9002400207047BA
:10D41000704700BF704700BF012070470346406A55
:10D42000C8B1B3F850201AB95B6D01200B6070478A
:10D4300007EE902AD3ED136A4FF0000C0022F8EEAD
:10D44000E77A012086EEA77A81ED007A83ED157ADE
:10D45000A3F850C0DA64704770B5044661F0F2FD7D
:10D4600000222221054661F06FFA606240B300237A
:10D4700006201A46194622F001F901462046F0F02E
:10D4800037FD666A00222221284661F031FB014601
:10D49000304622F043FC94F82030E269002103EB8F
:10D4A000430302EBC30383F82410012194F82030D6
:10D4B000E269084603EB431302EB830383F864102D
:10D4C00070BD00BF034B10B504460360F0F0E4FCF0
:10D4D000204610BD44561708054B10B5044603609E
:10D4E000F0F0DAFC20460BF069FB204610BD00BFCF
:10D4F0004456170870B590F8455082B00446DDB91F
:10D5000090F8383063B990F82830413B192B04D893
:10D5100090F82930413B192B46D9284602B070BDFE
:10D5200090F84820DAB9012BF7D1294628303DF18F
:10D5300039FF84ED100AF0E70122002390F828005B
:10D540000DF1060184F846208DF806308DF807307D
:10D550000AF0B0FA90B90025284602B070BD072B3A
:10D5600008BF012AD9D1294628303DF11BFFDFED44
:10D57000197A20EE270A84ED0F0ACEE70DF1070194
:10D5800094F829000AF096FA0028E4D09DF80620C5
:10D590009DF8073094F8445043EA0213DBB2ED1AC9
:10D5A000B5FA85F56D09B8E700F12A060A49304653
:10D5B000F3F7BEFE40B109493046F3F7B9FE30B982
:10D5C000012384F84830A8E784F84850A5E784F898
:10D5D0004750A2E7E4388E3E3456170838561708ED
:10D5E000A1F10A0330B5044683B0222B1FD8DFE82F
:10D5F00003F0181E1E181E1E1E1E1E1E1E1E1E1EA0
:10D600001E1E1E1E1E1E1E1E1E1E1E1E501E1E1E08
:10D610001E1E181E120090F8443083F02C0380F870
:10D62000443094F84650BDB1002003B030BD90F8AE
:10D6300037300D2B05D85A1C034480F8372083F867
:10D64000281094F845000028EED194F84430594051
:10D6500084F8441003B030BD94F84730002BE3D079
:10D6600094F8373020460191234483F82850FFF77F
:10D6700041FF019994F83830A1F12A0184F837501C
